:020000040000FA
:040000006FD00400B9
:101000006F00907E00000000000000009020002093
:10101000AA220020A9BDF9F56C23002000000000E1
:10102000000000006C230020902000200000000041
:101030000000000090200020000000009020002010
:101040000000000090200020902000209020002030
:101050009020002090200020582F00209424002071
:101060000000000090200020902000201E2400207E
:1010700090200020D22300209020002090200020EB
:101080009020002090200020902000209020002020
:101090009020002001A04111B7170040985F3AC688
:1010A000945F3247E39CE6FE3245410182800111A4
:1010B00013078008F337078093F787083EC20100C3
:1010C0000100B7170040930570052380B70413068D
:1010D00080FA2380C7040100010083C6B70493F699
:1010E000F60DA385D704238007049246F3A6068055
:1010F0000100010093760502D5CEF336078093F602
:10110000860836C4010001002380B7042380C70489
:1011100001000100B70614007D89558D88C70100C4
:1011200001000100010023800704A246F3A6068007
:101130000100010073370780137787083AC6010062
:1011400001002380B7042380C704010001000100CF
:1011500001003727004093061005A303D7802380A2
:101160000704B247F3A70780010001009307800836
:10117000F3B7078093F787083ECE01000100B71749
:101180000040130770052380E704130780FA2380CB
:10119000E7040100010003C7B70413670708A3852C
:1011A000E70423800704F247F3A70780010001004A
:1011B0000561828093760504BDC6F336078093F6F9
:1011C000860836C8010001002380B7042380C704C5
:1011D00001000100B7061400938606047D89558D31
:1011E00088C7010001000100010023800704C246F6
:1011F000F3A6068001000100733707801377870884
:101200003ACA010001002380B7042380C70401000B
:1012100001003727004093062005A303D7802380D1
:101220000704D24781B773370780137787083ACC12
:10123000010001002380B7042380C70401000100DE
:1012400098471367070C98C723800704E24719BF24
:101250000111814601468145114506CE97000000E7
:10126000E780605893078008F3B7078093F78708F3
:101270003EC601000100B717004013077005238028
:10128000E704130780FA2380E7040100010003C785
:101290006704136717002383E70423800704B2471A
:1012A000F3A7078001000100F2400561828041112F
:1012B000814601468145114597000000E780A05214
:1012C00013078008F337078093F787083EC40100AF
:1012D0000100B7170040130670052380C70493066A
:1012E00080FA2380D70401000100FD552396B70240
:1012F00023800704A245F3A5058001000100733790
:101300000780137787083AC6010001002380C704CD
:101310002380D7040100010003C767041367170087
:101320002383E70423800704B247F3A70780010063
:10133000010001A0BD473305F50201007D1575FDD3
:101340008280411122C426C206C6AA8401446317C2
:101350009400B24022449244410182800504130566
:10136000803E420497000000E78000FD4180C5B741
:101370009305000273A04580824573901534924016
:101380002242B2424243D2436244F2440255925551
:101390002256B2564257D2576258F25806499649D9
:1013A000264AB64A464BD64B664CF64C065D965DD1
:1013B000265EB65E465FD65F09617300203041113C
:1013C000B7170040985F3AC6945F3247E39CE6FE49
:1013D000324541018280B71700401307000323887C
:1013E000E702854717170000232EF74673002030C9
:1013F000411122C42D6426C24AC006C637190040D6
:101400001304A4AAB704002023208900977000E0E9
:10141000E780C0459C408297977000E0E7800045D8
:10142000E5B737370040834747009146BD8B639E41
:10143000D702B73600401306F00F973500009385AA
:1014400065219737000083D7E73003C7A6001377DD
:10145000F70F1DE3B7E70400BC4F09468945171590
:1014600000000345A5F7829731A099466394D70001
:10147000834757007300203003C786001377F70FA8
:10148000E365F6FC13851700AE97173800002313A9
:10149000A82C2380E70075B7B787004003C7670013
:1014A000098B6309071003C77700930600031377BE
:1014B0000703630DD7081748000003483880173624
:1014C00000001306A67C0547B30606012380E6004C
:1014D00083C57700173700001307477D429793F5C0
:1014E000F50F2300B70003C58700973500009385EB
:1014F000E57AC2951375F50F2380A5000347070011
:1015000089451377F703630CB70C63E7E50A6306B5
:10151000071A8545630CB7129737000083C7177AFF
:101520003307F600034707001377F70F19CB85073A
:1015300093F7F70F3D476363F71A17370000A30FC0
:10154000F776B787004009472383E700B787004055
:1015500083C77700E207E18763DE0704973700005F
:1015600083C7D77517370000130747723E97854624
:101570002300D70017370000130747733E979306E1
:1015800000032300D70017370000130727713E9789
:10159000A14685072300D70093F7F70F3D47636403
:1015A000F71417370000A30BF770B78700400947FF
:1015B0002383E70073002030930610026300D70EE8
:1015C000930620026305D70693060002E316D7F4BC
:1015D00003C727021377C70F13672700D5A803C7D0
:1015E00067001377070465CB03C7A702173800000D
:1015F0001308484B173500001305854213470708A9
:101600002385E70203C7A7021377370F1367870005
:101610002385E702814713070004B305F5008C41D9
:10162000B306F80091078CC2E399E7FEF5B503C74E
:10163000A702134707042385E70203C7A70213770E
:10164000C70F136727002385E702F9B503C76700B3
:101650001377070449C303C767021738000013084C
:101660002838173500001305652F13470708238313
:10167000E70203C767021377370F136787002383D7
:10168000E702814713070004B305F5008C41B30658
:10169000F80091078CC2E399E7FEBDBD03C767025E
:1016A000134707042383E70203C767021377C70FB3
:1016B000136727002383E70285B503C76700137705
:1016C000070411CB03C727021377370F136787006F
:1016D0002381E70291B5238006003DBD97370000C6
:1016E000A38E075CB9BD97370000A389075C75BD61
:1016F0002303048015472303E48001002302A48010
:10170000828083076480E3CE07FE23030480828007
:1017100083076480E3CE07FE03454480828083070D
:101720006480E3CE07FE2302A4808280411126C498
:101730004AC24EC006C61377F50BAD47AA892E895B
:101740009544630CF700194597000000E78080FA84
:1017500097000000E78020FB8D444E859700000035
:10176000E78040F9FD59FD1463983401B240A2446A
:101770001249824941018280135509011375F50F01
:1017800097000000E780E0F92209F1BF011126CCA3
:1017900006CEB704080097000000E780C0F61545A4
:1017A00097000000E78000F597000000E78080F6D2
:1017B00097000000E78000F62AC697000000E78047
:1017C00080F432459377150089EB13651500137586
:1017D000F50FF240E24405618280FD14E9F0014515
:1017E000CDBF397126DC4ADA4ED852D656D45AD2F9
:1017F0005ED006DE62CE66CCB7E700E07D5783AAF6
:10180000070022C603AA470023A0E71823A2E7186F
:10181000B7170040130770052380E704130780FA09
:101820002380E70483C74704930B75FFB684E20760
:1018300093FBFB0F8546AA892E8B32893724004003
:10184000E187015763FA76016308D50089461307DB
:1018500000026313D5000157D98F93F7F70FB71C18
:1018600000402382FC0411472303E4801305F00F9A
:1018700097000000E78000E8094C97000000E7802F
:1018800080E863657C15B7050700DA9537870700A0
:10189000795563FEE504B3879500636AF704370B57
:1018A0000800A94733EB65016395F90881E8814495
:1018B00097000000E78020E5268515A8DA85094510
:1018C00097000000E780C0E605090345F9FFFD1415
:1018D000050B97000000E780C0E481C49377FB0FFD
:1018E000E5F797000000E780A0EA69F17D55B7179A
:1018F0000040130770052380E704130780FA238054
:10190000E70403C74704418B2382E704F250B7E79B
:1019100000E023A0571123A24711E2543244525948
:10192000C259325AA25A125B825B724CE24C21615C
:101930008280A547639BF90685691309F00FB306FA
:101940009900B3742B01B6941349F9FFB37499004D
:10195000856B33796901416B9387F9FFB3F72701F1
:1019600099E363FC340193D94900C147E3E637FFAB
:101970003DBF0569C1697D19D9B71305800D63881D
:101980006901130500026384790113051008CA85F3
:1019900097000000E780C0D997000000E78040DF93
:1019A00031D54E99B38434416DBFDA852D4597000A
:1019B0000000E780E0D7CA94E30B99EE0509970091
:1019C0000000E78020D5A30FA9FEFDB79387F9FF9C
:1019D00093F7F70F636DFC0C83C71C0413073008E3
:1019E0006315F706370708006361EB06B3079B0032
:1019F000B706100063FBD704334BEB0089476399AC
:101A0000F9068980D549E38404EADA850945970017
:101A10000000E780E0D111090327C9FF9147232087
:101A2000E48003076480E34E07FE23033481FD173F
:101A3000EDFBFD14110B81C49377FB0FE9FF9700B9
:101A40000000E780E0D461F155B5B717004003C747
:101A50005704B70708001377070219E3B787070091
:101A60007955E376FBE833079B00E3F9E7F841B5E6
:101A70008547E380F9F0DA852D4597000000E7807F
:101A800020CB9389F4FFE38404E297000000E78011
:101A900060C893F7390091EB83260480032709007F
:101AA00093074900E396E6E03E89CE84D9BFB54767
:101AB0006399F9001305900B97000000E78080C33D
:101AC000FDB3B1471305B00AE388F9FE9947639760
:101AD000F904B7050800B365BB002D459700000069
:101AE000E78000C581448D4BA14997000000E78045
:101AF00060C263967401832704802320F900850463
:101B0000E39534FF8327048013172B0163550700E7
:101B10002312F90069BB2322F90051BB9D47639F43
:101B2000F90281451305B00497000000E78040C02A
:101B3000BD442320090023220900FD59970000001D
:101B4000E78040BD93F77400CA9703C70700FD14F0
:101B5000398D2380A700E39334FF91BBA14763979E
:101B6000F90697000000E780A0C28144630D0B00D6
:101B70008D479304C0036308FB00930400056304CE
:101B80008B01930440041375C507E30295D21945F0
:101B900097000000E78000B697000000E780A0B63D
:101BA000054597000000E780E0B426859700000017
:101BB000E78020B7094597000000E78080B69700CE
:101BC0000000E780E0BCE31405CE0DB39147639FAE
:101BD000F9001305600697000000E780A0B19700A8
:101BE0000000E78040B213059009F9B5E38109CC04
:101BF000F1547DB9BD66014717360000130646381B
:101C0000938606A685458347060093F7F70F91C391
:101C100082800507E3F9E6FE973700002382B73696
:101C2000DDB77D166206618693178601E18763D46E
:101C3000070001458280931726003307F500AE9711
:101C400018439C4363E7E7007D16E37FF7FC7D556F
:101C5000828005458280FD15E205E18513978501A7
:101C6000618793F7F50F63480700FD15139725006B
:101C70002A97584365D713851700620561858280CE
:101C80003308B5021C4283A80600B335B502C297DB
:101C900033B50701AE98469585486367B5006394F0
:101CA000A50063E3070181480C43C6950CC388C2B5
:101CB0001CC2828081471397870161876343B70005
:101CC0008280139727002A97232007008507E5B70E
:101CD0008147014793968701E18663C5B6001335B6
:101CE0001700828093962700AA9694428507558F05
:101CF000D5B793D755408A07AA979C430545331516
:101D0000B5007D8D828017F3FFDFE702833D2A84D3
:101D100097000000E78060F405C5931725003E9406
:101D20000327C4FF814711EB7D1516053E9542053B
:101D3000418517F3FFDF6700033D05838507E5B79E
:101D40000145C5BF81471397870161876343C7007A
:101D5000828013972700B386E50094422A9785076F
:101D600014C3D5B77D1662066186014793178601B5
:101D7000E18763D50700133517008280931726008B
:101D8000B306F500AE9794429C437D16B58F5D8FE8
:101D9000F1BF8A05AA9501476363B500828083A6D7
:101DA000C5FFF11593D71600D98F9CC11397F60183
:101DB000E5B72A830148014701456343D700828084
:101DC000B387050183A80700B30706019C43C697A4
:101DD000AA976384F80033B517010507B308030118
:101DE000620723A0F80061871108C1BF2A83014759
:101DF0008147014563C3D70082803388E50083288B
:101E00000800330EE600032E0E003388A840330886
:101E1000C8416384080133B508018507B308E300AE
:101E2000E20723A00801E1871107E9B717F3FFDFF5
:101E3000E702232B0111B286B2842E86AA850A8579
:101E400097000000E780C0FA2A84A6850A859700DB
:101E50000000E78020E833348000060413351500C5
:101E6000018D056117F3FFDF6700E32917F3FFDF3B
:101E7000E702A3244111AA89AE8A328BB68402C23A
:101E800002C402C60144131C8401135C8C416349E3
:101E90009C02939B1400FD1B0549138CF4FFF15C1D
:101EA00033048901620461846340740792478E049D
:101EB000CE9423AEF4FE410117F3FFDF67006323E6
:101EC00013192400B30B2B01014A93172A00D6974C
:101ED00083A50B0088437800340050009700000071
:101EE000E78040DA050A93178A01E187F11BE35E78
:101EF000FCFC92474E9905042320F900A2473EC2FC
:101F0000B24702C63EC441B7131A8901135A8A4127
:101F1000131D240093178A01E18763CF970092472E
:101F20000A044E941CC0A24705091379F90F3EC25A
:101F3000B24702C63EC4ADB7B3079A0313152A00D1
:101F400056950841780034005000050AEA97DA9760
:101F50008C4397000000E780E0D26DBF197106C284
:101F600012C416C61AC81ECA22CC26CE2AD02ED219
:101F700032D436D63AD83EDA42DC46DECAC0CEC2C9
:101F8000D2C4D6C6DAC8DECAE2CCE6CEEAD0EED2F9
:101F9000F2D4F6D6FAD8FEDA971500009385058CB0
:101FA0008841E700050092402242B2424243D243B8
:101FB0006244F244025592552256B2564257D257C5
:101FC0006258F25806499649264AB64A464BD64BBD
:101FD000664CF64C065D965D265EB65E465FD65F45
:101FE0000961730020300000972100209381810156
:101FF000175100201301018117F5FFFF1305C500DC
:102000009705002093850500171600201306C6FDCE
:1020100063FAC5008322050023A055001105910530
:10202000E3EAC5FE171502001305852B971500205E
:102030009385C5FB171600201306C66563FAC50015
:102040008322050023A0550011059105E3EAC5FE92
:102050001715002013050564974500209385053E5C
:102060006377B500232005001105E36DB5FEFD4241
:10207000739002BC8D4273904280B722000093821D
:10208000828873900230970200209382A2F793E235
:10209000320073905230975200009382C2C3739003
:1020A00012346FB0F47573002030397101436EC67D
:1020B00019A0397141536AC866CA62CC5ECE19A0B4
:1020C000397101535AD056D252D44ED64AD826DA54
:1020D00022DC06DE33016140828241114AC026C201
:1020E00022C406C68282B24D4101024D924C224C5E
:1020F000B24B4101024B924A224AB2494101024984
:1021000092442244B240410182803D432A87637356
:10211000C3029377F700BDEFADE5937606FF3D8AE6
:10212000BA960CC34CC30CC74CC74107E36BD7FE30
:1021300011E28280B306C3408A0697020000969699
:102140006780A6002307B700A306B7002306B700E1
:10215000A305B7002305B700A304B7002304B70005
:10216000A303B7002303B700A302B7002302B700FD
:10217000A301B7002301B700A300B7002300B700F5
:10218000828093F5F50F93968500D58D9396050182
:10219000D58D61B7939627009702000096968682A8
:1021A000E78086FA9680C1171D8F3E96E374C3F8C8
:1021B000A5B73367B500FD530D8B79E7B7877F7FF0
:1021C0009387F7F710419441B372F6003363F6003A
:1021D000BE92B3E262006397720C6318D606504158
:1021E000D441B372F6003363F600BE92B3E26200EC
:1021F0006398720A631BD60410459445B372F600C7
:102200003363F600BE92B3E262006391720A631E0A
:10221000D6025045D445B372F6003363F600BE9241
:10222000B3E26200639A72086311D60210499449BE
:10223000B372F6003363F600BE92B3E262006393BA
:1022400072085105D105E30FD6F6131706019397CF
:102250000601631CF7001357060193D706013305E7
:10226000F7409375F50F91E982804183C18333056F
:10227000F7409375F50F91E182801377F70F93F78D
:10228000F70F3305F74082800346050083C605003B
:10229000050585056313D60065FA3305D6408280AF
:1022A00011059105E312D6FE014582802105A105A5
:1022B000E31CD6FC014582803105B105E316D6FC4E
:1022C000014582804105C105E310D6FC01458280AD
:1022D000B717004003C777051377E70FA38BE70411
:1022E000130700F8A38DE7043D47238CE704130789
:1022F0005003A38CE70403C7A7051377D70F238DDB
:10230000E7048280B717004003C7E7020D89411137
:102310001377C70F498F93068008F3B6068093F6AC
:10232000860836C601000100930670052380D70495
:10233000930680FA2380D704010001002387E70277
:1023400023800704B247F3A7078001000100410181
:10235000828041112A83014E930E407E130F001993
:10236000930F400663E56E129308001913034006AD
:10237000B3781503854E0D4FA14F337365020D8958
:102380001335150063EFBE121308F6FF79467298F5
:102390004208135808013307C70213D61700BE07B7
:1023A00032976146B3F6C60213068070B386C60242
:1023B0003697A166F58F42075D8FB716004083C739
:1023C000F60293F70708A303F1000346710083C7E1
:1023D000F60293F70708E394C7FE83477100B71628
:1023E000004093F7F70F6388071293078008F3B74D
:1023F000078093F787083EC401000100B71700402B
:10240000930670052380D704930680FA2380D704AF
:102410000100010023AA070383C6170393E60608F9
:10242000A388D70223800704A247F3A707800100EF
:1024300001001166B71700407D16D45BC85F938515
:102440004703A98EF18EF5FA93068008F3B606804D
:1024500093F6860836C601000100930670052380B6
:10246000D704930680FA2380D7040100010098C1A5
:1024700003C7170313670704A388E7022380070431
:10248000B247F3A7078001000100410182807D135C
:102490003368E3039308E016630E08003368F30320
:1024A0009308D016630808009378330093B8180097
:1024B0009388D81633081E01131E0801135E0E01FF
:1024C00055B56393E5030548638608000148630337
:1024D00003002A8871087298FD15131E0801C205B1
:1024E000135E0E01C18179BD13F8150063F4BF00BE
:1024F0007908D5B713381800E5BF83C7F60293F7FC
:102500000708A303F1000346710083C7F60293F79F
:102510000708E394C7FE8347710093F7F70FF1DFD5
:10252000E9B531714AD966CB06DF22DD26DB4ED70D
:1025300052D556D35AD15ECF62CD6AC96EC7AA8C26
:1025400002D897100000E78020B12A8993078008FD
:10255000F3B7078093F787083EDA01000100B71749
:102560000040130770052380E704130780FA2380D7
:10257000E7040100010003C7F7021377770FA38771
:10258000E70203C7F70213678700A387E7022380E8
:102590000704D257F3A70780010001000545970003
:1025A0000000E78060D6130780C13347E902116A53
:1025B00093070AE893065002BD69930BA004814A71
:1025C000014B13048008930470057D1AB347F90288
:1025D0003307D7023EC0FD873ECC938709A69309F7
:1025E000803E3347F7023AC27D873AC43347390306
:1025F0008549B399990193D93940B306D702B30BF2
:102600007703B3C6F602B3CBFB0236C6FD8636C8E7
:1026100093D6FB4136CEB7460F0093860624334946
:10262000D9028566938606FAB3969601B389E902C4
:10263000130760553309D90293060010B389E902E4
:102640003349D902B3C9F9029316390036CA37198A
:102650000040FD8636D0930D090493D7F9413ED250
:10266000F336048093F6860836DC010001009307F8
:1026700070052380FD00930680FA2380DD000100B1
:1026800001008346390593F6860FA309D9048346D2
:10269000390593E61600A309D90423800D00E256FC
:1026A000F3A6068001000100130C80FA116DF336C9
:1026B000048093F6860836DE01000100930770055A
:1026C0002380FD0023808D01010001008346390530
:1026D000216693E60602A309D90483560905B3E6E9
:1026E000A6012318D90483560905D18E2318D904CD
:1026F00023800D00F256F3A60680010001008346F8
:10270000390593F606026381061A03463905218AC4
:102710006DDE081897100000E7800098733604807B
:1027200013768608B2C20100010023809D00238039
:102730008D0101000100B717004003C6370513766D
:10274000F60DA389C70403C6370513660602A389DD
:10275000C704835609052166B3E6A6012318D904E8
:1027600083560905D18E2318D90423800D0096467F
:10277000F3A60680010001008346390593F60602A0
:10278000638B061483463905A18AEDFE970000206D
:10279000E7806090AA8636D497000020E780A08F5B
:1027A000A256E30AD5FE835609054255B3E6A601B3
:1027B0002318D90497100000E780C08F834639059D
:1027C000A18AEDDE03560905834629058247337643
:1027D000CA00B306DA0293D5F641B296B388F64042
:1027E000E24733B8C6002E983308F840A247B3B684
:1027F00016013308D84063C70701631DF8009247EC
:1028000063FA1701C247634FF80E63950701B24799
:1028100063EAF80E894663E9660FF24693151800DD
:1028200013D3F8015E8613951800B365B30042D642
:1028300046D497D00100E780E0E53258050B137BC2
:10284000FB0F63470001631A0838A25863870838F2
:1028500013081500B336A800B69513D6F5013298C3
:10286000B336C800AE9613581800FE06B3E606014C
:102870007336048013768608B2C6010001002380F7
:102880009D0023808D01010001000356C902B2960C
:10289000C206C1822316D90223800D00B646F3A6D4
:1028A00006800100010021B5F336048093F6860806
:1028B000B6C00100010023809D0023808D0101002E
:1028C00001008346390593E60602A309D904238053
:1028D0000D0086460DB5F336048093F68608B6C41F
:1028E0000100010023809D0023808D010100010073
:1028F0008346390593E60602A309D90423800D0017
:10290000A646BDB5E30B0BF0F336048093F68608BC
:10291000B6C801000100930680FA23809D00238041
:10292000DD00010001008346390593F5FC0F93F6A5
:10293000860FA309D90483463905CD8EA309D9048E
:1029400023800D00C646F3A6068001000100130592
:1029500080FA03463905930639051D8A631C9629BA
:102960007336048013768608B2CC0100010013068A
:1029700080FA23809D002380CD000100010003C662
:1029800006001376F60D2380C60003C60600136604
:1029900006022380C600835609051166D18E2318CE
:1029A000D904835609052166D18E2318D9042380C2
:1029B0000D00E646F3A6068001000100130680FA2A
:1029C0008346390593F60602638006268346390559
:1029D000130C3905A18AFDDA081897000000E7807A
:1029E000A06BF336048093F68608B6D00100010090
:1029F000930680FA23809D002380DD000100010002
:102A000083460C00116693F6F60D2300DC00834626
:102A10000C0093E606022300DC0083560905D18EE4
:102A20002318D904835609052166D18E2318D904A9
:102A300023800D008656F3A60680010001001306D0
:102A400080FA8346390593F60602638A0620834698
:102A50003905A18AEDFE97F0FF1FE780C0632A8C3D
:102A600097F0FF1FE7802063E30C85FF835609057D
:102A700011664255D18E2318D90497000000E780D3
:102A800060638346390513063905A18AFDDAF336FA
:102A9000048093F68608B6D401000100930680FAFC
:102AA00023809D002380DD00010001008346060095
:102AB00093F6F60D2300D60023800D00A656F3A64C
:102AC0000680010001008356090503462905D24707
:102AD000B376DA003306CA021305800C9355F6412B
:102AE0003696330DF6408257333CD6002E9C333653
:102AF000A601330CFC40330CCC40330885039256BE
:102B00004E86B335A5033305A503C29597D00100C2
:102B1000E78040B863468001631E0C16630C0D16F7
:102B2000130615003335A6002E959356F5013696FB
:102B3000B335D600AA959396F50105828585D18E89
:102B40006346B000639D051A638B061A0356C902DB
:102B500015823305D6003336C500B2956348B00000
:102B6000639105241306F00F637DA622894663F363
:102B7000561593078008F3B7078093F78708BED6EA
:102B80000100010037170040930770052300F70488
:102B9000930780FA2300F704010001008356C7025F
:102BA00089678117D58FC207C1832316F7022300D7
:102BB0000704B657F3A7078001000100FA506A54D2
:102BC000DA544A59BA592A5A9A5A0A5BFA4B6A4C49
:102BD000DA4C4A4DBA4D296182801308F5FF33352E
:102BE000A800FD152E951356F5013298B336C8008E
:102BF000AA9695B9F336048093F68608B6CA010002
:102C0000010023809D002380AD0001000100834668
:102C10003905CD8EA309D90423800D00D646F3A62D
:102C200006800100010035B3F336048093F6860870
:102C3000B6CE0100010023809D002380CD0001005D
:102C400001008346390593E60602A309D9042380CF
:102C50000D00F646F3A606800100010095B3F33699
:102C6000048093F68608B6D20100010023809D00FF
:102C70002380CD00010001008346390593E606025A
:102C8000A309D90423800D009656F3A606800100FF
:102C9000010045BB9306F5FF33B5A600FD152E9543
:102CA0009355F501AE96B3B5B600AA951396F50106
:102CB000858269B5F336048093F68608B6D801009C
:102CC0000100930680FA23809D002380DD0001002F
:102CD00001008356C9020566011693F6F60FD18EE0
:102CE000C206C1822316D90223800D00C656F3A660
:102CF000068001000100850A93FAFA0F95B233E6C7
:102D0000B60045C20356C9023305D0403338A0008F
:102D1000B305B040B385054115826345B000D1E1EC
:102D20006371A608894663F0560593078008F3B7D8
:102D3000078093F78708BEDA01000100B71700404B
:102D4000130770052380E704130780FA2380E70444
:102D50000100010003D7C7027D8B2396E702238081
:102D60000704D65781BDF336048093F68608B6DC97
:102D700001000100930680FA23809D002380DD007E
:102D8000010001008356C9020566011693F6F60F8D
:102D9000D18EC206C1822316D90223800D00E656C9
:102DA000B9B793078008F3B7078093F78708BEDEAB
:102DB0000100010037170040930770052300F70456
:102DC000930780FA2300F704010001000356C702AD
:102DD00093975600B297C207C1832316F7022300C8
:102DE0000704F657C1BB914763EEB70217E701002E
:102DF000130747288A05BA959C41BA978287B71767
:102E0000004003A7470B1345F5FF698F23AAE70A84
:102E100003A7070B698F23A8E70A03A7070A798D81
:102E200023A0A70A8280B717004083A6470B134749
:102E3000F5FFF98E23AAD70A83A6070B558D23A881
:102E4000A70A83A6070A758F23A0E70A8280B7170F
:102E5000004003A7470B498F23AAE70A03A7070BE4
:102E60001345F5FF45BFB717004083A6470B13472F
:102E7000F5FF758F23AAE70A03A7070A598D4DB7F7
:102E8000B717004003A7470B498FEDB7914763EE93
:102E9000B70217E701001307271F8A05BA959C415F
:102EA000BA978287B717004003A7470D1345F5FF70
:102EB000698F23AAE70C03A7070D698F23A8E70CE6
:102EC00003A7070C798D23A0A70C8280B7170040B9
:102ED00083A6470D1347F5FFF98E23AAD70C83A6C7
:102EE000070D558D23A8A70C83A6070C758F23A06B
:102EF000E70C8280B717004003A7470D498F23AA2C
:102F0000E70C03A7070D1345F5FF45BFB7170040B2
:102F100083A6470D1347F5FF758F23AAE70C03A778
:102F2000070C598D4DB7B717004003A7470D498FC0
:102F3000EDB7797122D43714004026D24AD0035914
:102F400024028354040206D64209C2044ECE52CC57
:102F500056CA13590901C1802DE11379F9F793F489
:102F6000F49F4209C20413590901C18093078008E4
:102F7000F3B7078093F787083EC401000100930769
:102F800070052300F404930780FA2300F404010081
:102F90000100231124032310940223000404A247F8
:102FA000F3A7078001000100B25022549254025945
:102FB000F249624AD24A45618280B7F507008146EC
:102FC0003000B105194597000020E7808081A247B5
:102FD00013972701E34A07FC1369090893E40440A7
:102FE00093098008F3B7098093F787083EC0010072
:102FF0000100930A700523005405130A80FA230088
:10300000440501000100231124032310940223002E
:1030100004048247F3A7078001000100294597F0C7
:10302000FF1FE7802031F3B9098093F989084EC268
:1030300001000100230054052300440501000100A4
:103040008357040293E707202310F40223000404AB
:103050009247B9B7B7170040884742054181937737
:10306000050491EB9377F5013755E80113050580C9
:103070003345F50282809377050C130700046397AC
:10308000E7009377F50137459C1CCDB72165130503
:1030900005D0828037E700E01C435443A183E20659
:1030A000D58F1CC1FD572320F7182322F7188280E3
:1030B00013178500B7E700E023A0E710618123A282
:1030C000A7108280B7F700E08847CC47828081470D
:1030D00037370040A14663C4C7003285828003456C
:1030E000B740E38EA6FE3385F5000345050085074E
:1030F0002304A740CDB797070020938727EF9C4371
:1031000017370020130787333E95636EE5001737A6
:1031100000201307273F6368A70017070020232715
:10312000A7EC3E858280FD57EDBF8280411122C40D
:1031300006C62A8497000000E78000F22947B307FB
:10314000E502B2408D83B3D7870222449507B3D7F7
:10315000E70237370040C207C1832316F700410159
:103160008280411137150E0006C697000000E780E7
:1031700020FCB7370040130770F82381E7000D47A4
:10318000A381E70013070004A380E7000547238716
:10319000E700B24041018280373700408347270073
:1031A0001A0593F7F703C98F93F7F70F2301F70079
:1031B0008280B737004003C7170019C9D98DA38093
:1031C000B70003C70700136787002380E7008280EA
:1031D00093C5F5FFF98DA380B7008280AE872A875B
:1031E000B736004021463738004089E71703000012
:1031F0006700E3F383C8B600E30916FF05078348B9
:10320000F7FFFD17C20723041801C183F9BF41115D
:1032100022C406C62A8497000000E780E0E329471D
:10322000B307E502B2408D83B3D7870222449507E6
:10323000B3D7E70237370040C207C1832316F740F0
:1032400041018280716541111305052006C6970072
:103250000000E78000FCB7370040130770F82381B7
:10326000E7400D47A381E74013070004A380E74030
:1032700005472387E740B24041018280CC4141119C
:1032800006C6328503C6150083C5050022064D8E8D
:1032900042068D654186138875A2630C0611634B47
:1032A000C804138845A26300060D634AC8009385CD
:1032B00035A26301B6082390060029464DA0138865
:1032C00055A26305060D938565A2E316B6FE8D45EE
:1032D0001D4663E6E5081146198E63F3C7003E8676
:1032E000B7E704002390C600FC4797E501009385EB
:1032F000E5DB9DA0138895A263030611634E060DBE
:103300001388A5A263000613938505A5E315B6FAF5
:1033100099451D4663E5E504198E63F3C7003E86B3
:10332000B7E704002390C600FC479705002093856B
:1033300025D61DA09D451D4663E3E5022146198E55
:1033400063F3C7003E86B7E70400FC472390C6003E
:103350009705002093858534BA9582970146B2403F
:10336000328541018280AD451D46E3EAE5FE3146E6
:10337000198E63F3C7003E86B7E704002390C600AA
:10338000FC4797E501009385E5D4F9B7B1451D46A3
:10339000E3E7E5FC3546198E63F3C7003E86B7E7E1
:1033A00004002390C600FC4797E50100938585D370
:1033B00065B78D451D46E3E4E5FA1146198E63F3C2
:1033C000C7003E86B7E704002390C600FC4797E598
:1033D0000100938565CE49B78D451D46E3E1E5F8CB
:1033E0001146198E63F3C7003E86B7E704002390A9
:1033F000C600FC4797E50100938585D0B1BFA54580
:103400001D46E3EEE5F42946198E63F3C7003E86B8
:10341000B7E704002390C600FC4797E501009385B9
:1034200065CA1DBFB5451D46E3EBE5F23946198E69
:1034300063F3C7003E86B7E704002390C600FC474D
:1034400097E50100938585C501BFB7E7040003A395
:103450000713970600209386A6C24146A545170587
:1034600000201305E5B802832D455DE703C505007F
:103470000947631FE50803A84500411106C6034735
:10348000180032850346080022074168518F9308CF
:1034900028FE6307170563E9E800051863030703BF
:1034A00023900600294591A8130648FE630AC70425
:1034B0001518E31707FF15463E87637BF60015478F
:1034C00001A8130600023E876374F600130700028A
:1034D000B7E704002390E600FC471316070111A884
:1034E0003E8691C30546B7E70400FC472390C6001B
:1034F0004206CC45418282970145B240410182801B
:10350000130600083E87E375F6FC13070008C9B7E9
:103510002390060005458280828041677917630405
:10352000E504411122C406C685472A84639FF5003D
:10353000B7E7040022852244B24003A3871397050E
:1035400000209385E52F4101028389476399F500A7
:10355000B7E7040083A7070B8545829771D9B2406E
:103560002244410182808280797126D252CCAE847D
:103570002A8A97E501009385A5BA17E5010013058E
:10358000A5BC06D63AC622D44AD0368432894ECE5D
:1035900097C00100E780405BA28517E50100130595
:1035A000A5BB97C00100E780205A294597C00100BC
:1035B000E780605E83C7840093F70702F9E383C95D
:1035C00004008947054532476396F908D44083C70C
:1035D000160083C60600A207D58FC166138616FEA5
:1035E000638CC7028D16638FD7068D6693862690EF
:1035F00029456391D706B7E70400A286225403A3A6
:103600004714B250F2494A86A6850259925452850F
:10361000624A8547456102832D450DEF93070002FD
:10362000354563E98702B7E70400FC47C844130641
:103630000002CA8582978149970700209387072156
:103640009C43014581CB9C4391C74E852286CA8508
:1036500082970145B250225492540259F249624A6B
:10366000456182802D457DF79307700F3545E3E373
:1036700087FEB7E70400FC47C8442286CA858297C4
:1036800065BF2145C1BF411122C437E4040083272F
:10369000841326C2AA84416506C697050020938537
:1036A000251A7D1582978327C40A17050000130584
:1036B00005E78588829795C0032304132244B2400E
:1036C000924497060020938626AE4146C5451705CD
:1036D00000201305659C41010283B24022449244BC
:1036E00001454101828019C59707002023A0A71634
:1036F00001458280454582801147636AA70A97E6A3
:1037000001009386A6A00A0536951841411106C608
:103710003697AE87B2850287130700026145639D25
:10372000E700B7E70400FC47130600021705002076
:10373000130545F782970145B24041018280054754
:103740006145E39BE7FEB7E70400FC470546170524
:103750000020130525F7F9BF1307700F6145E39D9E
:10376000E7FCB7E70400FC471306700F17050020BD
:10377000130585F5C1B7130700086145E39EE7FA15
:10378000B7E70400FC4713060008170500201305DF
:1037900025034DB715476145E390E7FAB7E7040005
:1037A000FC471546170500201305C50961B70945F3
:1037B0008280411126C2B7E4040083A7C41322C447
:1037C0004AC006C62E8497050020938565072A897E
:1037D0008297058905C5970700209387E78B83D7D4
:1037E000A70BA28503A3440D2310F4002244B2408A
:1037F00092444A850249014641010283B240224473
:103800009244024949454101828097070020238163
:1038100007049707002023AF0702B717004003A74C
:10382000070CB706C0FFFD16758F23A0E70C03A792
:10383000070DB7064000558F23A8E70C03A7070C18
:103840003D9B23A0E70C03A7070D1367070123A8DF
:10385000E70C8280B717004003A5470C83A7470CED
:10386000598113451500C18B058999E3136525001E
:103870009707002083C7C7FD6380A7029707002032
:103880002388A7FC11C9970700209387A7FC03A3EF
:1038900007006303030002838280114517F3FFFFD3
:1038A000670063C8011122CC06CE3714004026CA37
:1038B0004AC84EC652C483447405034AB4058349BA
:1038C00084050349940597F0FFFFE780A0A0834794
:1038D000A40593F4F40F137AFA0F93E71700230D5E
:1038E000F40493F9F90F1379F90FB717004003C7E0
:1038F000A705058B6DFF03D5C705A38D4705238C51
:103900003705A38C2705A38B9704F2406244D24469
:103910004249B249224A05618280411193970501CB
:1039200022C406C626C2C1872E8463DC0700B7E422
:103930000400FC54829719C1BC5482972165218DE3
:1039400015A893F7150013C515008DE793F725000B
:103950009DC797000000E78020F0B7E70400BC4F48
:103960001306000A894517050020034525EF8297B5
:1039700013452400B240224492444101828093972F
:10398000250163D80702B7E4040083A7C41E829709
:1039900097000000E780A0F0BC4C375607001306E4
:1039A0000630896517050020034545EB82970965B8
:1039B00079B7939715010145E3DE07FA17E5010092
:1039C0001305858197C00100E780E02FB7E7040069
:1039D000BC4F13060064916517050020034505E8F8
:1039E00082971165A9BF1D71A2CC37E404005C5C0D
:1039F000485886CE494697D50100938565798297C8
:103A000011E917D501001305E57997C00100E7809A
:103A1000802B01A0B7F600E0795798CAFD57DCCAA1
:103A20000567B7E700E023A0E7101306F00290C295
:103A300023A0E718010001003707002018471306EC
:103A4000000481459706002023A8E6E04157A38A99
:103A5000E7403C4408088297970700209387077F38
:103A60003EC8856713870740938757D1231AE10023
:103A70002312F1021307B00F97F7FFFF9387C76474
:103A80002310E1023ED81547970700009387C7E14E
:103A9000B7F50700A30FE1003EDC054797070000DC
:103AA0009387E7DF81463000E10519452301E102F4
:103AB0003EDE97F0FF1FE780C0D218088147994685
:103AC00030003E960346060085070507A30BC70096
:103AD000E398D7FEC24791C70357410185676373D7
:103AE000F70001A0B7E7040083A7470A08088297F8
:103AF000AA8511C917D501001305056C97C00100EF
:103B0000E780800401A0F64066442561828041116F
:103B100026C2B7E4040083A7040806C622C417051A
:103B200000001305C5DF829717040020130404D397
:103B30002300A40097000000E780800297000000A7
:103B4000E780E0CC03450400224403A38405B2408F
:103B5000924413060032896541010283797106D6C9
:103B600022D413078008F337078093F787083EC2F3
:103B700001000100B7170040930570052380B704CA
:103B8000130680FA2380C7040100010083C6F702F0
:103B900093F6A60FA387D702238007049246F3A6C5
:103BA00006800100010073370780137787083AC445
:103BB000010001002380B7042380C7040100010035
:103BC00003C7F70213672700A387E70223800704D0
:103BD000A247F3A7078001000100054597E0FFFF1A
:103BE000E780807297000000E78060CB0147814644
:103BF0008147054685451305407E97E0FFFFE78036
:103C0000807537E404003C44680051468145829742
:103C1000B707C0A83EC8B787E803938707D03ECA56
:103C200097E7FF1F9387A7793EC67C586800829765
:103C3000B250225445618280411197E5010093857D
:103C4000A5BD17D501001305255006C697C0010074
:103C5000E78080EF17E501001305C5D397C0010089
:103C6000E78080EEB2402945410117C3010067009B
:103C700083F2411197E50100938545BB17D50100FB
:103C80001305854C06C697C00100E780E0EB17E5F9
:103C900001001305E5CE97C00100E780E0EAB240DD
:103CA0002945410117C301006700E3EE411122C419
:103CB00006C6834705002A849DC797E501009385C2
:103CC000A5BC17D501001305254897C00100E78062
:103CD000A0E74C4017E501001305C5E097C00100BF
:103CE000E78080E63DA058410DEF97E50100938500
:103CF000A5B917D501001305254597C00100E78038
:103D0000A0E417E50100130565DF97C00100E78017
:103D1000A0E32244B2402945410117C301006700D6
:103D200083E7A1679386D7036313D70297E5010062
:103D3000938585B517D501001305054197C001008E
:103D4000E78080E017E50100130545DC7DBFED0746
:103D500097E50100938545B317D501001305C53ECE
:103D6000631BF70097C00100E78000DE17E5010044
:103D7000130505DB59BF97C00100E780E0DC4C402C
:103D800017E501001305C5DB91BF411197E501005F
:103D9000938505AB17D501001305053B06C697C0F3
:103DA0000100E78060DAB2402945410117C30100F4
:103DB000670063DE797122D426D24AD02E842A8904
:103DC000B28481457146480006D697E0FFFFE78040
:103DD000003497F7FF1F9387275EDC4783D70700E0
:103DE000231421012313F10097600000E78020F1E4
:103DF0008547A305F1009307401F2305A1003EC698
:103E00002686FD57A2854800230AF100976000002E
:103E1000E780C0F1B2502254925402594561828029
:103E20004111972700202396079297270020238F80
:103E3000078006C6170700200347C7319307F00A1B
:103E40006315F7029307F0F889451705002013055D
:103E5000653017070020230FF72E97070020A38B4C
:103E6000072E97700000E780C0AA97700000E780D7
:103E700080D797700000E780C0D8814537050400DF
:103E80009707002023AE072A970700202389072AD7
:103E9000970700202390072097070020239E071CE8
:103EA000970700202393072697070020239C0728C5
:103EB00097400000E780803C014597700000E78054
:103EC00040AED14717070020231AF726B7E70400B2
:103ED000BC4F13060014894517050020034585983B
:103EE000829797E501009385259817D50100130562
:103EF000A52597C00100E78020C59705002083D540
:103F0000E52317E501001305E5C997C00100E78027
:103F1000A0C3B2402945410117C301006700A3C7F0
:103F20004111814617F6FF1F1306464685451705C2
:103F300000200355251406C697D00000E780803284
:103F400015C997E501009385E59217D50100130582
:103F5000A51F97C00100E78020BF17E501001305EA
:103F600065B497C00100E78020BE294597C00100D5
:103F7000E78060C297E501009385C58F17D50100E2
:103F80001305851C97C00100E78000BC17E5010000
:103F9000130585B297C00100E78000BB294597C093
:103FA0000100E78040BF97F7FF1F9387E740DC479A
:103FB000054797E501009385E58B2390E70017D52A
:103FC00001001305651897C00100E780E0B717E509
:103FD00001001305A5AF97C00100E780E0B6B2402D
:103FE0002945410117C301006700E3BA411122C40A
:103FF00097E501009385858A2A8417D5010013056A
:10400000A51406C697C00100E78000B44C4017E530
:1040100001001305A5A697C00100E780E0B229457D
:1040200097C00100E78020B7034704009307F00F13
:10403000631FF70297E501009385458617D50100B8
:104040001305851097C00100E78000B04C4017E5CC
:1040500001001305A5A397C00100E780E0AE22444C
:10406000B2402945410117C301006700C3B2B24005
:10407000224441018280411122C426C22A84AE8496
:1040800017D501001305450C97D501009385C57C14
:1040900006C697C00100E78020AB17E501001305B5
:1040A000E5AE97C00100E78020AA294597C001002E
:1040B000E78060AE97D501009385057A97070020C9
:1040C000239A87FA17D501001305050805449707B9
:1040D0000020239F97F897070020239C87F89717C5
:1040E00000202398976697C00100E780E0A5971508
:1040F000002083D5056617E501001305A5A997C023
:104100000100E78060A4294597C00100E780A0A8CE
:1041100097170020238C875297F7FF1F9387C72993
:10412000DC4717F5FF1F0345E57303D70700C16799
:10413000FD17631EF700B7E7040003A38705130606
:10414000000A85452244B240924441010283B7E708
:10415000040003A387051306001493050010DDB7C0
:10416000B1C1411122C417D501001305E5FD2E840C
:1041700097D501009385856D06C697C00100E7803D
:10418000A09CA28517E501001305859F97C001003B
:10419000E780809B2244B2402945410117C30100BA
:1041A0006700639F8280011122CC26CA4AC836C6A6
:1041B00006CE2A84AE84328997000000E780C0BF13
:1041C000F157B246631EF50089CE97600000E78084
:1041D00000CA4A86A685228597000000E780C0BDF8
:1041E00005C59707002083D747EC850717070020F0
:1041F000231DF7EA97070020239AA7EAF2406244BA
:10420000D2444249056182809707002083D727EA7C
:10421000850717070020231CF7E8CDB7011122CC32
:1042200037E404005C5C06CE26CA354697D501000B
:104230009385857717E5010013054570829711E98D
:1042400017D50100130505F697C00100E780A0A768
:1042500001A097F7FF1F9387A7613EC4B7F507003A
:10426000856793870780814617F6FF1F1306C65F91
:10427000E10519453EC697E0FF1FE78080567C4464
:10428000194697F5FF1F9385255E17050020130536
:10429000A5E08297340017F6FF1F1306E65C97E54A
:1042A0000100938525BB17E50100130525BC978008
:1042B0000000E780E0EBAA8421C197D50100938537
:1042C000256117D50100130525E897C00100E78097
:1042D000A087A68517D501001305056E97C00100BC
:1042E000E7808086294597C00100E780C08AF240B8
:1042F0006244D2440561828097F00000E780C0519B
:1043000017D501001305456297700000E78000E0B3
:1043100097C00000E78000A697700100E780800A40
:1043200017F5FF1F1305C50597700100E78020F3FF
:1043300017D501001305456097700100E780000B59
:10434000AA8497700000E780404697200100E7802C
:1043500060E297900100E780807B97900000E78003
:1043600020A297800000E78040BC97500100E780C2
:10437000C0A397D501009385A55517D50100130556
:10438000A5DC99C897B00100E780007CA68517D509
:1043900001001305A56499B797B00100E780C07AC2
:1043A00017D501001305C56597B00100E780C079F6
:1043B000294597B00100E780007E97400100E78023
:1043C000A07F97100100E780609E6DC58545370589
:1043D000040097400000E78060EA97D501009385CC
:1043E000254F17D50100130525D697B00100E780AA
:1043F000A07517D501001305256297B00100E7806D
:10440000A074294597B00100E780E07897F7FF1F77
:10441000938707EA83D7070017170020231BF7327B
:104420008547171700202303F72297F7FF1F93876D
:10443000A7F8DC4703D70700C167FD176316F7002D
:1044400097000000E78000AE97800000E780601DC5
:104450008567938707E33E9597800000E780201DDE
:1044600097200000E780602F171500200355652E68
:1044700097600000E780601F054597600000E780B7
:10448000405297600000E780C07797D50100938580
:10449000254417D50100130525CB97B00100E7800F
:1044A000A06A17D501001305255C97B00100E780CD
:1044B000A0690DBDD14797D501009385654117D5FA
:1044C0000100130565C8170700202319F7C697B028
:1044D0000100E780606717E60100130666B89705DC
:1044E000002083D5A5C517D501001305255597B024
:1044F0000100E7806065294597B00100E780A06969
:104500003C4C1306000A894517F5FF1F0345853506
:104510008297014597600000E780A048BDB7411130
:1045200022C437E404008327041A06C682979760E2
:104530000000E780401783270408171500001305C3
:10454000053D829797F7FF1F238EA73017F5FF1FB2
:10455000130585E697600000E78020C82244B2403A
:104560004101170300006700A3CBB7E70400FC4735
:104570001171A2DDCAD986DFA6DBCED72E8432899F
:104580002E86AA85170500201305C5BC829717073C
:104590000020130727BC83470700930680029387F8
:1045A000E70793F7F70FE3ECF610BA898A0717D7F6
:1045B00001001307A7C2BA979C43BA9782878D4719
:1045C00097D501009385053317D501001305C5B7AD
:1045D000630FF40097B00100E780005717D5010082
:1045E000130505F097B00100E7800056BDA497B011
:1045F0000100E780605517D501001305E5EF97B07E
:104600000100E7806054294597B00100E780A05879
:10461000930720F81146970500209385A5B34A8596
:10462000170700202308F7B297070020A38507B2D9
:1046300097F0FFFFE78040782A841DC997D50100D5
:104640009385452B17D50100130505B097B00100E0
:10465000E780804FA28517D501001305A5ED97B01F
:104660000100E780604E294597B00100E780A05225
:1046700097D501009385052817D501001305C5AC12
:1046800097B00100E780404C17D501001305C5EB3A
:1046900097B00100E780404B294597B00100E780C3
:1046A000804F4165930730FA0546970500209385B2
:1046B00065AA7D1517070020230EF7A897F0FFFFC6
:1046C000E780806F2A841DC997D5010093858522D4
:1046D00017D50100130545A797B00100E780C04634
:1046E000A28517D501001305E5E497B00100E78026
:1046F000A045294597B00100E780E049B7E70400ED
:10470000BC4F0566130606C8A14517F5FF1F0345F4
:1047100065158297FE506E54DE544E59BE59116194
:10472000828091476303F40297D501009385851C2D
:1047300017D50100130545A197B00100E780C040DF
:1047400017D50100130585E371BDB7E70400FC4FE1
:10475000914517F5FF1F0345E510829797D5010096
:104760009385451917D501001305059E97B00100E3
:10477000E780803D17D50100130505E297B00100E1
:10478000E780803C294597B00100E780C040975002
:104790000000E780C06D914535A485476303F402AE
:1047A00097D501009385051517D501001305C59907
:1047B00097B00100E780403917D50100130545DFA8
:1047C00015B5970700202397278DB7E704000566E6
:1047D000BC4F130606C8C1450DBF8D476303F402E5
:1047E00097D501009385051117D501001305C595CF
:1047F00097B00100E780403517D50100130505DDAE
:10480000D5B3930740F8114697050020938585940A
:104810004A8517070020230FF79297070020A38CE3
:10482000079297F0FFFFE78020592A84E30405EE02
:1048300097D501009385050C17D501001305C59088
:1048400097B00100E7804030A28517D5010013051D
:1048500065CE97B00100E780202F294597B0010071
:10486000E780603345BD9147E31CF4F6B7E70400E9
:10487000FC4F9305000217F5FF1F0345A5FE829725
:1048800097D501009385050717D501001305C58B42
:1048900097B00100E780402B17D50100130585D4A0
:1048A000F1BD894763E3870297D5010093858504AD
:1048B00017D501001305458997B00100E780C0288E
:1048C00017D50100130545D331BB9704002083C4DD
:1048D00084889707002083C7F78797D501009385C1
:1048E0006501A20417D5010013050586DD8C97B07C
:1048F0000100E7806025A28517D50100130505D1C9
:1049000097B00100E7804024C204294597B0010018
:10491000E7806028C1849305D4FF93960401C18287
:104920004A8693F5F50F170500201305D5829740A9
:104930000000E7806098E35F90DC930750F817076A
:1049400000202309F78083C73900228697050020BD
:104950009385458085074A8517F7FF1FA30DF77ECE
:1049600097F0FFFFE78040452A84E30505DA97D5F5
:104970000100938525F817C501001305E57C97B064
:104980000100E780601CA28517D501001305451EB4
:10499000C9B5894763E3870297D50100938585F5FB
:1049A00017C501001305457A97B00100E780C019CB
:1049B00017D50100130545C735B197500000E780B2
:1049C000004BA28517F5FF1F1305C57897600000FF
:1049D000E78020F481B38D476303F40297D501008B
:1049E000938545F117C501001305057697B00100C1
:1049F000E780801517D501001305C5C4E5B6B76675
:104A000002000146B7750200054597E0FF1FE780E9
:104A100040DD930760F817F7FF1F230DF77297F734
:104A2000FF1FA38A07729307000617F7FF1F2305CE
:104A3000F772894717F7FF1FA300F77297F7FF1F59
:104A4000238D077097F7FF1FA3890770C14717F7DA
:104A5000FF1F2305F770930720F917F7FF1FA30F18
:104A6000F76E314697F7FF1FA38BA76E97F5FF1FD1
:104A70009385456E4A8597F7FF1F2382076E97F04F
:104A8000FFFFE78060332A84E30605C897D501005D
:104A9000938545E617C501001305056B97B0010026
:104AA000E780800AA28517D50100130525BB55B301
:104AB000B1476303F40297D501009385A5E317C5B9
:104AC00001001305656897B00100E780E00717D57E
:104AD0000100130565BA39B6B7E70400FC4F93052A
:104AE000000417F5FF1F0345E5D782979750000094
:104AF000E780E037B145F9B5914763E3870297D581
:104B00000100938525DF17C501001305E56397B004
:104B10000100E780600317D501001305A5B7D9B4DC
:104B200097F4FF1F83C4446397F7FF1F83C7B762DF
:104B3000A204DD8C8E04B77702006D14BE94228629
:104B4000A68517D50100130525B697B00100E780AB
:104B5000A0FFB7E70400FC47228697F5FF1F938567
:104B6000B55F2800829793160401C1823000A685A4
:104B7000094597E0FF1FE780C0C62A8409C917D5F9
:104B80000100130525B497B00100E780C013930717
:104B900070F8194697F5FF1F9385C55B4A8517F78F
:104BA000FF1F2309F75A97F7FF1FA387875A97F02C
:104BB000FFFFE78060202A84E30E05B497D501004B
:104BC000938545D317C501001305055897B001001B
:104BD000E78080F7A28517D501001305A5AF95B929
:104BE0009947630BF41297D501009385A5D017C59B
:104BF00001001305655597B00100E780E0F417D573
:104C000001001305A5AEF9BA914763E3870297D572
:104C10000100938525CE17C501001305E55297B015
:104C20000100E78060F217D501001305A5AD5DBA5C
:104C300097F4FF1F83C4445297F7FF1F83C7B751F0
:104C4000A204DD8C8E04B77702006D14BE94228618
:104C5000A68517D50100130525AC97B00100E780A4
:104C6000A0EEB7E70400FC47228697F5FF1F938567
:104C7000B54E2800829793160401C1823000A685A4
:104C80000D4597E0FF1FE780C0B52A8409C917D5F5
:104C90000100130525AA97B00100E780C002930721
:104CA00080F8194697F5FF1F9385C54A4A8517F77F
:104CB000FF1F2301F74A97F7FF1FA38F874897F03D
:104CC000FFFFE780600F2A84E30605A497D5010063
:104CD000938545C217C501001305054797B001002C
:104CE000E78080E6A28517D501001305E5A595B6F6
:104CF00099476303F40297D501009385A5BF17C5B3
:104D000001001305654497B00100E780E0E317D583
:104D100001001305E5A4F9B0B7E70400FC4F9305C3
:104D2000000417F5FF1F0345E5B382979750000075
:104D3000E780E013994579B18D476303F40297D575
:104D40000100938525BB17C501001305E53F97B00A
:104D50000100E78060DF17D501001305E5A159B018
:104D600017D50100130545A297B00100E780A0F513
:104D70001305C01297D0FF1FE780A05C014597E0A4
:104D8000FFFFE78060310D4597100000E780A01716
:104D9000294597D0FF1FE780C05A97D0FF1FE780B3
:104DA000204B8DBA99476303F40297D50100938590
:104DB00065B417C501001305253997B00100E780D8
:104DC000A0D817D501001305E59C29B817F7FF1FD8
:104DD0000347973897F7FF1F83C7073822075D8F70
:104DE0009166BA96C2061166C1821306F6EF8D4728
:104DF0006365D60297E7FF1F9387075C9C4B17F606
:104E0000FF1F034656359386C7002DC203D6070001
:104E100069CA8907E39CD7FE89471307A0F81146A2
:104E200097F5FF1F938505334A8597F6FF1F238368
:104E3000E63217F7FF1FA300F73297F0FFFFE78076
:104E4000A0F72A84E308058C97D50100938585AAED
:104E500017C501001305452F97B00100E780C0CEAC
:104E6000A28517D5010013052594E5B203D60700E6
:104E7000630EE60A8907E39BF6FE8D4779BF9147EB
:104E80006304F40297D501009385C5A617C50100F8
:104E90001305852B97B00100E78000CB17D50100E3
:104EA000130505926FF00FF4B7E70400FC4F93056C
:104EB000000817F5FF1F0345E59A8297C9B897D5F3
:104EC0000100938525A317C501001305E52797B0B9
:104ED0000100E78060C717D501001305E58F6FF06B
:104EE0006FF02390E70017E5FF1F1305E54C97408F
:104EF0000100E780E0F197D501009385A59F17C5D4
:104F000001001305652497B00100E780E0C317D5C1
:104F100001001305658D97B00100E780E0C22945C7
:104F200097B00100E78020C78147C5BD23900700E7
:104F300017E5FF1F1305454897400100E78040ED46
:104F400097D501009385059B17C501001305C51F63
:104F500097B00100E78040BF17D501001305458ACF
:104F60005DBFB7E70400FC4741112E8606C622C488
:104F700026C24AC02E842A89AA8517F5FF1F130569
:104F8000651D829797D501009385859817C5010007
:104F90001305851B97B00100E78000BB97F5FF1F45
:104FA00083C5451B17C501001305853E97B0010059
:104FB000E78080B9294597B00100E780C0BD97F42C
:104FC000FF1F9384241983C7040041479387070672
:104FD00093F7F70F6369F75A17C701001307472ABA
:104FE0008A07BA979C43BA9782879D476307F40262
:104FF00097D501009385C59117C501001305C51408
:1050000097B00100E78040B417C501001305C5380B
:1050100097B00100E78040B3A1AC97F7FF1F83C7AB
:105020007713DDCB17F7FF1F0347F71297F7FF1F23
:1050300083C7671222075D8F97F7FF1F83C7C711CA
:10504000C2075D8F97F7FF1F83C71711E207D98F3C
:1050500017F7FF1F2326F70E83C7640097D50100BB
:105060009385058B17C501001305050E17F7FF1F64
:105070002307F70C97B00100E78000AD97F7FF1FFB
:105080009387070C8C4317F6FF1F0346460B17C583
:1050900001001305253297B00100E780E0AA2945F9
:1050A00097B00100E78020AF97F7FF1FA384070A9E
:1050B0002244B24092440249930700F817F7FF1FB9
:1050C000230AF7089D4517F5FF1F1305A5084101A1
:1050D000176300006700E38397700000E780A05328
:1050E00097F7FF1F2389A7069357850017F7FF1F20
:1050F000A303F706935705012A8417F7FF1F230D13
:10510000F70493578501014517F7FF1FA306F7041E
:1051100097700000E780805497F7FF1F238FA70246
:1051200097C501009385C57E17C501001305C5010C
:1051300097B00100E78040A117F6FF1F0346E60184
:10514000A28517C5010013056528B1B7CD476303D4
:10515000F40297C501009385A57B17C501001305CF
:10516000A5FE97B00100E780209E17C5010013053A
:10517000652779BD97F7FF1F83C7E7FEA20717F7DB
:10518000FF1F034737FED98FC207C1876357F0025D
:1051900017F7FF1F2314F7FAB7E7040003A38705E7
:1051A0001306000A89452244B2409244024917E599
:1051B000FF1F0345256B41010283D147D1BF8D47B6
:1051C0006303F40297C501009385857417C5010038
:1051D000130585F797B00100E780009717C5010018
:1051E0001305053035B517F4FF1F0344C4F697F7D0
:1051F000FF1F83C737F697C50100938565712204A9
:1052000017C50100130545F45D8C97B00100E780D8
:10521000A093A28517C501001305451E97B0010094
:10522000E7808092294597B00100E780C0960D463F
:1052300097F5FF1F938505F2228597F0FFFFE78022
:10524000A0B7AA8421C197C501009385656C17C5D5
:105250000100130565EF97B00100E780E08EA68599
:1052600017C501001305C51A97B00100E780C08D6E
:105270002244B240924402492945410117B301003A
:105280006700639197F7FF1F239687E0B7E7040055
:10529000116603A38705130606E8914529B78D47D4
:1052A0006303F40297C501009385856617C5010065
:1052B000130585E997B00100E780008917C5010053
:1052C0001305C530B1B317F4FF1F0344C4E897F7C3
:1052D000FF1F83C737E897C50100938565632204E4
:1052E00017C50100130545E65D8C97B00100E78006
:1052F000A085A28517C501001305C51297B001004E
:10530000E7808084294597B00100E780C0880D467A
:1053100097F5FF1F938505E4228597F0FFFFE7804F
:10532000A0A9AA841DC197C501009385655E17C514
:105330000100130565E197B00100E780E080A685D4
:1053400017C501001305450F05B797F7FF1F2395F4
:1053500087D2B7E70400116603A38705130606E8A2
:105360009305000289B5894763E3870297C5010069
:105370009385055A17C50100130505DD97A00100A7
:10538000E780807C17C501001305052751B197F40C
:10539000FF1F83C444DC97F7FF1F83C7B7DB97C5A4
:1053A00001009385E556A20417C501001305C5D970
:1053B000DD8C97A00100E7802079A68517C5010044
:1053C0001305050997A00100E7800078294597A0FB
:1053D0000100E780407C228697F5FF1F938585D7E3
:1053E000268597F0FFFFE780209D2A84630E051A2B
:1053F00097C501009385C55117C501001305C5D494
:1054000097A00100E7804074A28517C5010013052D
:10541000650599BD854763F98718834519002244BE
:10542000B24092440249B335B00097F7FF1F238D75
:10543000B7C617C5010013052504410117A30100D4
:1054400067008370A2852244B24092444A85024993
:10545000410117130000670043B199476303F40249
:1054600097C501009385C54A17C501001305C5CD31
:1054700097A00100E780406D17C501001305853135
:1054800041BE17F4FF1F034404CD97F7FF1F83C7E6
:1054900077CC97C501009385A547220417C5010065
:1054A000130585CA5D8C97A00100E780E069A2859D
:1054B00017C501001305C5FD97A00100E780C0686E
:1054C000294597A00100E780006D194697F5FF1F59
:1054D000938545C8228597F0FFFFE780E08DAA8479
:1054E0001DC197C501009385A54217C5010013058D
:1054F000A5C597A00100E7802065A68517C5010016
:10550000130505FA95B397F7FF1F239D87C2B7E7E9
:105510000400116603A38705130606E89305000837
:1055200059B1854797C501009385853E17C5010090
:10553000130585C1630BF40097A00100E780C060EC
:1055400017C50100130505F7E1B497A00100E78036
:10555000A05F17C50100130565F797A00100E7805C
:10556000A05E294597A00100E780E0622244B24096
:105570009244024997F7FF1F239207BC410117731A
:1055800000006700C3F997C501009385653817C50A
:105590000100130565BB97A00100E780E05A17C51D
:1055A000010013056523ADB4B24022449244024980
:1055B00041018280411106C622C426C239C12A8413
:1055C00097F00000E780807EAA8411EDB7E7040021
:1055D000BC474146814522858297B24022442685B8
:1055E00092444101828041657D1597F00000E7807B
:1055F000C07CB7E7040001E9BC47414681452285EC
:1056000082978144D9BF0347E501FC479305900881
:1056100019E393050003AA954146228582978544A4
:105620006DBF93170501C1876350F00817F6FF1F80
:105630001306C6AF97F6FF1F83C606B0B2850147B3
:10564000B287639BE60215476367D700850617F7A5
:10565000FF1F2303D7AE17F7FF1F0347E7AD7D17E3
:105660001377F70F0607BA976381C70203D7E7FFDF
:10567000F9172391E700CDBF890503D8E5FF631132
:10568000A8020607BA976397C70097F7FF1F239FE3
:10569000A7A8828003D7E7FFF9172391E700E5B7B2
:1056A00005071377F70F71BF8280011122CC06CE58
:1056B00026CA4AC8834705002A849DC797C50100AA
:1056C0009385051F17C50100130505A897A00100C4
:1056D000E78080474C4017C501001305655097A02F
:1056E0000100E780604605A25841B707CF009387C5
:1056F000777D6319F70C0359C500854704450356A8
:10570000E50063F8270903C7040083C51400F17698
:1057100093178700CD8FC207C1879386C6556392C2
:10572000D702328597000000E780E0EF6244F24044
:10573000CA8526854249D2440561172300006700C7
:10574000E36E954763F72705930730056313F70466
:1057500093075004639FF50283C624009307100447
:105760006399F60283C734006395E70203C74400D8
:105770009307B004631FF70003C754009307900515
:105780006319F700CA85328597200000E780E05B47
:1057900071BF9707002083D7C7FB638AC700CA85FC
:1057A000268532C697E0FFFFE78080A33246624439
:1057B000F240CA8526854249D244056117F3FFFFAE
:1057C0006700E3DAB707CC009387777D6317F704A8
:1057D00097C501009385C50D17C501001305C59632
:1057E00097A00100E78040361C448356E4008355AF
:1057F000C40003C6070017C501001305E53F97A0C5
:105800000100E78060346244F240D24442492945B5
:10581000056117A3010067000338B707CE0093871F
:10582000777D6304F70297C501009385650817C566
:1058300001001305659197A00100E780E0304C401E
:1058400017C501001305C52F59BDF2406244D2446B
:1058500042490561828017F5FF1F0345E58D82806F
:1058600097F7FF1F83C7478D637BF50097F7FF1FEF
:105870009387C78B06053E95035505008280014539
:1058800082800111854622CC4AC84EC652C406CE3B
:1058900026CA2A8A2E89328497F0FFFFE780E0909B
:1058A000AA89630B09049307F4FFC207C1835D470C
:1058B0006364F704B7E40400FC442286CA8517F544
:1058C000FF1F1305E584829797F7FF1F239F8784A7
:1058D00097F7FF1F239C4783894717F7FF1F23056F
:1058E000F784BC4C8565130600329385058017E567
:1058F000FF1F034525F78297F24062444E85D2444C
:105900004249B249224A056182805D71A2C486C6BD
:10591000A6C2CAC04EDE93F715002E84B5CB97E021
:10592000FFFFE7802060930710F817F7FF1F23039E
:10593000F78297E7FF1F83D7A77317F7FF1FA30B04
:10594000F7809145A18317F5FF1F1305A58017F771
:10595000FF1F2302F78097E7FF1FA38E077E975054
:105960000000E78000FBB7E70400BC4F13060014FB
:105970009305001017E5FF1F0345C5EE82971345F9
:105980001400B640264496440649F259616182806B
:10599000856493840480B3F79500A5CB97E7FF1F38
:1059A00083C78778A1CF17E6FF1F0356067839C64D
:1059B000854697E5FF1F9385A57517E5FF1F0355DE
:1059C000E57497E0FFFFE780407E97E7FF1F93872E
:1059D000A77583C70700FD1793F7F70F17E7FF1F9A
:1059E0002304F77481CFB7E70400BC4F13060032DD
:1059F000A68517E5FF1F0345E5E6829705651305B4
:105A00000580218D42054181ADBF93F70540B9C79F
:105A1000814797C501009385E58A9306300231A03E
:105A200070003E962300E60085073387B700030722
:105A3000070013960701418209C7E393D7FE1306B7
:105A4000300217E5FF1F0355456F11C56C00970025
:105A50000000E78040E31345044025B793F7052095
:105A600081CB97E7FF1FA389076C13C5052011BFE2
:105A700093F70510B1C3054597500000E78060F229
:105A8000170500200355E5CC97500000E780E0BDE6
:105A900097100000E78060CC97E7FF1F83C7D77A95
:105AA00089E797500000E780001497500000E780D6
:105AB000401513450410F1B593F72500E9CF17E71A
:105AC000FF1F0357A76769C7AD64B71900409384E8
:105AD000A4AA23A0990097E6FF1F938666669442C6
:105AE00097C701009387C70D17E6FF1F034626657A
:105AF000814517C501001305A50D97700000E780CB
:105B0000209223A0990097D7FF1F239BA77A2A8969
:105B100041C197C501009385A5DC17B501001305A8
:105B2000A56297A00100E7802002CA8517B5010091
:105B30001305057B97A00100E7800001294597A088
:105B40000100E780400597E7FF1F2399075E930751
:105B500010F817E7FF1F230FF75E97E7FF1F83D7A4
:105B6000275117E7FF1FA307F75EA18317E7FF1F62
:105B70002303F75E91458D4717E5FF1F1305855DEC
:105B800017E7FF1FA309F75C97500000E78060D874
:105B900013452400FDB393F74500D1C397C5010019
:105BA000938505D417B501001305055A97A0010088
:105BB000E78080F917B501001305457497A001002F
:105BC000E78080F8294597A00100E780C0FC930793
:105BD00020F817E7FF1F230FF75697E7FF1F83D71C
:105BE000674B17E7FF1FA307F756A18317E7FF1FB0
:105BF0002303F756854717E7FF1FA30EF754974077
:105C00000000E780C02617E5FF1F1305A554914546
:105C100097500000E780E0CF134544009DB393F711
:105C20008500A9C797C50100938585CB17B50100ED
:105C30001305855197A00100E78000F117B5010019
:105C40001305056D97A00100E78000F0294597A096
:105C50000100E78040F497E7FF1F2391074E9770FC
:105C60000000E780C08B1345840021BB93F705013A
:105C7000D1C3854517E5FF1F0355C5419750010066
:105C8000E780804197C50100938585C517B5010060
:105C90001305854B97A00100E78000EB17B50100C5
:105CA0001305456897A00100E78000EA294597A001
:105CB0000100E78040EE930730F817E7FF1F230B42
:105CC000F74897E7FF1F83D7E73C17E7FF1FA303BA
:105CD000F74817E5FF1F1305E547A1838D4517E733
:105CE000FF1F230AF74697500000E78080C2134544
:105CF000040141B993F70502D1C797C50100938507
:105D000025BE17B501001305254497A00100E780C3
:105D1000A0E317B501001305256397A00100E780F4
:105D2000A0E2294597A00100E780E0E6930740F84C
:105D300017E7FF1F2300F74297E7FF1F83D7C733FB
:105D400017E7FF1FA308F740A18317E7FF1F2304EE
:105D5000F740854717E7FF1FA30FF73E97E7FF1FA1
:105D6000239C073097400000E780601017E5FF1F75
:105D70001305453E914597500000E78080B91345D3
:105D8000040201B193F70504FDC397C50100938593
:105D900025B517B501001305253B97A00100E78045
:105DA000A0DA17B501001305A55B97A00100E780F5
:105DB000A0D9294597A00100E780E0DD97E7FF1F04
:105DC00083C747391307700A6386E7061307800AFB
:105DD000638CE7081307600A6393E704930760F88E
:105DE00017E7FF1F2308F73697E7FF1F83D7E73131
:105DF00017E7FF1FA300F736A18317E7FF1F230C48
:105E0000F734854717E7FF1FA30BF734B14517E5B4
:105E1000FF1F1305253497500000E78080AF97409F
:105E20000000E780C0041345040497E7FF1F239E8A
:105E3000072C81BE930770F817E7FF1F230CF7307C
:105E400097E7FF1F83D7672C17E7FF1FA304F730DF
:105E5000A18317E7FF1F2300F730854717E7FF1FD0
:105E6000A30CF72E994565B7930780F8F1B793F720
:105E700005080145E38707B097C50100938545A64E
:105E800017B501001305452C97A00100E780C0CB92
:105E900017B501001305454E97A00100E780C0CA61
:105EA000294597A00100E78000CF9307A0F817E7E6
:105EB000FF1F2301F72A97E7FF1F83D7A72817E7BC
:105EC000FF1FA309F728A18317E7FF1F2305F72862
:105ED000854717E7FF1FA300F72897E7FF1F2393C6
:105EE000072697400000E78080F817E5FF1F13059D
:105EF0006526914597500000E780A0A1134504084E
:105F000049B4411122C491462A8417E6FF1F1306A3
:105F100066329D652D4506C697D0FF1FE780608CD1
:105F2000B7F7070003C70701A5476313F70001A0F0
:105F30009306001001469D65254597D0FF1FE78019
:105F4000408A97E7FF1F2387872E2244B24091465D
:105F500017E6FF1F1306062E9D652945410117D33D
:105F6000FF1F670003881171CED7B7E9040083A72C
:105F7000C904CAD917E9FF1F1309C91DA2DD2E865E
:105F800086DFA6DB2E84AA854A85829797E7FF1FC6
:105F900083C7471C1307700A6385E710636DF7001A
:105FA0001307600A6385E704FE506E54DE544E59B1
:105FB000BE59116182801307800A6385E7161307B3
:105FC000900AE393E7FE8D476306F41C97C5010032
:105FD000938505CE17B501001305051797A001009D
:105FE000E78080B617C501001305C5C925A08D47F8
:105FF000630CF40297C50100938585CB17B50100AA
:106000001305851497A00100E78000B417C50100AF
:10601000130585C097A00100E78000B3294597A02C
:106020000100E78040B749B7854717C50100130550
:1060300065C017E7FF1F2309F70697A00100E78057
:1060400080C8B7750200B76602000146054597C0D3
:10605000FF1FE7800079930760F817E7FF1F230B06
:10606000F70E97E7FF1FA388070E9307002617E791
:10607000FF1F2323F70EE5779387072117E7FF1FFD
:10608000231EF70CB14597E7FF1F238A070C97E7FC
:10609000FF1FA386A70C4A8597000000E780E01643
:1060A00021B7914763E3870297C50100938545C0F7
:1060B00017B501001305450997A00100E780C0A8A6
:1060C00017C50100130505B9B1B797E4FF1F83C4D5
:1060D000A40897E7FF1F83C71708A204DD8C83A7D6
:1060E000C9046D14228697E5FF1F9385F5062800E5
:1060F00082978E0493160401B7750200C1823000A6
:10610000A695094597C0FF1FE780A06D930770F81B
:1061100017E7FF1F2300F704994597E7FF1FA38D9B
:10612000A70295BF914763E3870297C50100938556
:1061300025B817B501001305250197A00100E780D8
:10614000A0A017C50100130565B2E9B597E4FF1FCC
:1061500083C4840097E7FF1F83C7F7FFA204DD8C89
:1061600083A7C9046D14228697E5FF1F9385D5FE8A
:10617000280082978E0493160401B7750200C1822D
:106180003000A6950D4597C0FF1FE78080659307F7
:1061900080F8BDBF17C50100130505B097A0010029
:1061A000E78060B2930790F82304F1008347190059
:1061B0008D452800A304F100834729002305F10041
:1061C00097000000E78060041305C01297C0FF1F0E
:1061D000E7802017014597D0FFFFE780E0EB0D45F2
:1061E00097000000E78020D2294597C0FF1FE78075
:1061F000401597C0FF1FE780A0057DB397E7FF1FFD
:1062000023A2A704828097E7FF1F9387A70303A316
:106210000700630303000283174300006700636FF6
:1062200041114AC097F6FF1F83D6A652328917D66E
:10623000FF1F0356861A22C426C206C62A84AE84CD
:1062400097000000E780A06629C921C8994763F636
:1062500097048347140003470400A207D98F1397BC
:106260008700A183D98FC2073167C1831307C75540
:106270006395E70297D7FF1F83D72716A301F40082
:10628000A1832302F40097F7FF1F83D7874C91C7A0
:10629000A302F400A1832303F400630D090297F71E
:1062A000FF1F83C7A73A9DE797E7FF1F83C7C7F97B
:1062B00095C38DC097E7FF1F83C707DF81EF228556
:1062C0002244B2400249A68592444101174300008E
:1062D00067002364B2402244924402494101828013
:1062E000834755008345450017C501001305059FE9
:1062F000A207DD8D17A301006700038517C5010004
:106300001305C59C17A301006700E39B8D4763F647
:10631000B708011126CA06CE22CC0344350097E403
:10632000FF1F83C474F297C501009385659CB33742
:10633000800017E7FF1FA309F7F009C497C5010004
:106340009385C59B17C501001305C59B9790010058
:10635000E780807F97E7FF1F83C717EF638697006B
:1063600097000000E780804397500000E780608935
:106370009967938757EE2316F1006800854791458A
:10638000A30781002307F10097000000E780E0E702
:10639000F2406244D244056182808280894763F77B
:1063A000B708011122CC06CE26CA834425008547B2
:1063B0002A84639DF404914763F5B70403454500BF
:1063C0008347340022055D8D97D7FF1F2397A700D1
:1063D00097000000E78080569967938767EE231443
:1063E000F1008347340023059100A305F1008347A2
:1063F0004400954528002306F10097000000E7803F
:10640000C0E0F2406244D24405618280FDF89967A1
:10641000938767EE2314F10097D7FF1F83D7E7FB1D
:10642000A305F10023050100A183E1B782800111DA
:10643000996722CCD51717F4FF1F130424212314C6
:10644000F1008347040026CA97F4FF1F9384643049
:106450002305F10083D7040028009545A305F1002A
:10646000A18306CE2306F10097000000E780E0D963
:1064700003D604008345040017C501001305858970
:1064800097900100E780406CF2406244D24405617D
:1064900082809D677971D9172316F10097F7FF1F46
:1064A0009387C71A83C707001305F10006D6230791
:1064B000F10097F0FFFFE780201009E9B7E704003B
:1064C000BC47414681451305F10082976800CD45E0
:1064D00097000000E78060D397F5FF1F83C505177D
:1064E00017C501001305058697900100E780C06578
:1064F000B25045618280630C0516011126CA06CE92
:1065000022CC4AC84EC697E7FF1F83C7F7D397F43C
:10651000FF1F83C4A41399C393E424002A84972003
:106520000000E780E08193E9C40119E193E9C40028
:1065300037E9040083278904228513062003814557
:106540008297930750FA2300F4009307A005A30055
:10655000F4008D472301F4009147A301F400930751
:106560001005A302F40097F7FF1F83D7871E2304AB
:10657000F400A183A304F40097D7FF1F83D7E7E5B6
:106580002305F4009304C400A18323020400230321
:106590003401A305F400268597F0FFFFE780C001D2
:1065A00019E583278904414681452685829797D737
:1065B000FF1F83D727E0230EF400A183A30EF4006E
:1065C00093070002230FF400930710FAA30FF400BF
:1065D0009D472300F402A3000402B7E70400FC4730
:1065E00013052402194697D5FF1F9385E527829747
:1065F00097E7FF1F83D7A7AB2304F402A183A3046B
:10660000F40297E7FF1F83D747AA2305F402A1836B
:10661000A305F40297E7FF1F938747A98397070015
:106620002285930500032306F402C207C183A183D8
:10663000A306F40297D7FF1F938787C883970700A5
:106640002307F402C207C183A183A307F4029700C2
:106650000000E780C0212308A4022181A308A4022E
:10666000F2406244D2444249B2490561828082804C
:106670005D71E17793C777FF1305E10086C62316A6
:10668000F10097000000E78040E7680093054003B1
:1066900097000000E78060B7B640616182805DC905
:1066A000411122C426C206C6930750FA2300F50002
:1066B0009307A005A300F50089472301F500914742
:1066C000A301F50093071005A302F50097F7FF1F3C
:1066D0009387C7F783C707009304C5002A84230361
:1066E000F50097E7FF1F938737B683C7070023029C
:1066F0000500A303F50097F7FF1F83D78705230441
:10670000F500A183A304F50097D7FF1F83D7E7CC3B
:106710002305F500A183A305F500268597F0FFFF6B
:10672000E78080E901E9B7E70400BC4741468145BD
:10673000268582972285F14597000000E780201387
:10674000230EA4002181A30EA400B240224492444F
:106750004101828082805D710A8586C6A2C497004D
:106760000000E78000F437E404007C448A850810C8
:10677000794682973C441305E10309468145829797
:10678000101093050002014597D0FFFFE78000F746
:10679000B6402644616182800111B7C7A55A22CC58
:1067A0009387C73317E4FF1F130414AA3EC483471B
:1067B0000400856601469965254506CE3EC697C00C
:1067C000FF1FE78000023000A1469965294597C068
:1067D000FF1FE78000018345040017B50100130582
:1067E000E56097900100E7802036F2406244056141
:1067F00082800111A146300099652D4522CC06CE3C
:1068000097C0FF1FE780E0FDA24737C4A55A1304D5
:10681000C43363958702B24517B501001305C5540B
:10682000B335B00097E7FF1FA380B7A29790010090
:10683000E7808031F2406244056182809165A14623
:106840003000938505F02D4597C0FF1FE78060F964
:10685000A247E38287FC97E7FF1FA387079E814536
:1068600017B5010013058552D1B7C1676976814616
:10687000FD1705061397060141836364B7003E8543
:1068800082803307D50003470700B98F214713F8EB
:106890001700858363050800B18FC207C1837D1788
:1068A0001377F70F6DF78506F1B741C5A547054783
:1068B00063F2B70883471500034705003168A20754
:1068C000D98F13978700A183D98FC207C18313087B
:1068D000C855054763900707411106C622C426C262
:1068E00003442500914763F087049307540063EC49
:1068F000F502A301C50021822302C50093043400E0
:1069000091C6A302D500A1822303D5002A84A685BF
:1069100097000000E780A0F526942300A4002181C1
:10692000A300A4000147B240224492443A854101A9
:10693000828005473A8582800111B7C7A55A22CCCB
:106940009387E7342A842AC68566014695652545DE
:1069500006CE3EC497C0FF1FE780A0E83000A146E6
:106960009565294597C0FF1FE780A0E7A28517B569
:1069700001001305A54997900100E780E01C9700EE
:106980000000E78080DDF2406244056182800111F1
:10699000A146300095652D4522CC06CE97C0FF1F3D
:1069A000E78020E4A24737C4A55A1304E434639572
:1069B0008702B24517B501001305453F97D7FF1F62
:1069C000239DB7A0C205C18197900100E780C01741
:1069D000F2406244056182809165A1463000938552
:1069E00005EE2D4597C0FF1FE780A0DFA247E38299
:1069F00087FCD14717D7FF1F2311F79ED14517B545
:106A000001001305A53CC9B721C1411126C206C624
:106A100022C4AE848DC52A8497100000E78000410F
:106A200097E7FF1F83C7478299CB22852244B24054
:106A3000A6859244410117430000670083EDB240F0
:106A40002244924441018280828001114EC606CECA
:106A500022CC26CA4AC893F71500AE899DCBAD67F4
:106A6000371700409387A7AA1CC3B7E70400BC4FA1
:106A700013060019854517D5FF1F0345E595829735
:106A800013C51900F2406244D2444249B24905613B
:106A9000828093F725000145F5D717F7FF1F0357AD
:106AA00027CB954763F9E70C014417F6FF1F130640
:106AB00026BA9306300513055004130810049308F2
:106AC000B00413039005930764006374F7043A84D9
:106AD0007D5997F4FF1F83C4A4B797F7FF1F83C79F
:106AE00037B7A204DD8CAD679387B755638BF41479
:106AF00063E3970AA9679387A755638EF414A28569
:106B000017F5FF1F1305C5B497000000E78000F0DC
:106B1000E9A0B307860083C50700639AD50483C53F
:106B200017006396A50483C527006392050583C5F6
:106B30003700639ED50283C54700639A150383C758
:106B400057006396670222890DE897F5FF1F83D5EA
:106B500025C0B3852541C20517F5FF1F130545AFB5
:106B6000C1814A9597000000E78040EAE1A0050452
:106B70004204418089BF3A847D598547E3EB87F41D
:106B80005DC4854517F5FF1F130585AC9700000010
:106B9000E780C0E769A8B1679387C7556389F404A4
:106BA000B5679387D755E39CF4F4A28517F5FF1FCB
:106BB000130505AA97400000E780A0D58947630E1A
:106BC000F4009305E4FFC205C18117F5FF1F13050B
:106BD00045A897100000E7806025A68517B501003D
:106BE0001305852497900100E78000F689A097306F
:106BF0000000E78060C797100000E780601411C9AB
:106C0000A28517F5FF1F1305A5A497100000E780C4
:106C1000E0210546A28517F5FF1F130565A397F030
:106C2000FFFFE780206097300000E780E0C3FD575A
:106C3000E31DF9F097F7FF1F239C07B013C5290048
:106C400091B5A28517F5FF1F130585A097F0FFFFEB
:106C5000E780406959B7A28517F5FF1F1305459FC7
:106C600097F0FFFFE780C0698DBF411122C437E470
:106C700004005C5C06C6354697B501009385C5D215
:106C800017C50100130585CB829711E917B50100DF
:106C90001305C51A97900100E780E00201A0832741
:106CA000041C82972A84054597D00000E78020B60F
:106CB00097700100E780403B97700100E78040102B
:106CC00097C00000E780A0C72285B240224441015E
:106CD00082804111054506C622C426C297C0FFFF27
:106CE000E78060251305A00497B0FF1FE780203CD4
:106CF000757585457D1597C0FFFFE780000F7D7591
:106D000085451305F53697C0FFFFE78060183714F7
:106D100000408327840A8D451305002093E7072050
:106D20002324F40A97C0FFFFE780200CB7E4040097
:106D300097C0FFFFE7804051C85897900100E78057
:106D400080F817C50100130565BF97900100E78023
:106D500080F78327840C8545414593E70708232462
:106D6000F40C97C0FFFFE780A0128D4513050008C3
:106D700097C0FFFFE780C01197C0FFFFE780A03EEC
:106D800037A507001305051297C0FFFFE780403ABB
:106D9000014597C0FFFFE78060409545054589475D
:106DA00017F7FF1F2308F79A97C0FFFFE780A0405F
:106DB000B7E700E013070006238DE740370700041C
:106DC00023A0E71097D0FFFFE78020C297D0FFFFF6
:106DD000E78020D497000000E78060E9970000007A
:106DE000E78060A197000000E780A0BA97D0FFFF7E
:106DF000E780207397100000E78080049700000070
:106E0000E780801083A7040817050000130525C438
:106E1000829797C7FF1F2381A75CBC4C13060064B1
:106E20008545829797B0FF1FE780805C014582808F
:106E3000AD67371700409387A7AA1CC3B7E700E0E8
:106E40003707400023A0E71801000100B7F707004B
:106E500003C70701A5476316F7009397450191C340
:106E600001A04111AE860146AA85254506C697C0F8
:106E7000FF1FE7800097B240B7E700E03707400008
:106E800023A0E710410182804111B2862E86AA8597
:106E90002D4506C697C0FF1FE780A094B24001456C
:106EA000410182809307000463ECC7041D71A2CCEA
:106EB0002A840808A6CACAC886CE32C6979001009E
:106EC000E78020BDAD67371700409387A7AA1CC392
:106ED000B7E400E03709400023A0241901000100B5
:106EE000B2461008A285294597C0FF1FE780608F32
:106EF000F640664423A02411D64446492561828089
:106F00003955828041110D658D4506C697C0FFFF3A
:106F1000E780A0EDB71700408D6623A6D70A17F5C6
:106F2000FF1F130565831387C70A9387870A1CC150
:106F30005CC5856689675CC958C114C518C9B7E7BF
:106F40000400B24003A3871E4101028303870600A9
:106F500009E763E0C5022E85828093871500C2078A
:106F6000C183E3F8C7FEAA952380E5008506BE85A8
:106F7000F1BF2E9523000500F9BF8145B307B50089
:106F80008387070089E7173300006700839485052E
:106F9000C205C181E5B7011106CE2307010001ED4D
:106FA00017B501001305053597000000E78020FDA7
:106FB000F240056182805800A947BA8529462548D4
:106FC000B376C502FD1793F7F70F93860603A30464
:106FD000D700B356C5026375A8007D173685EDF35B
:106FE0003385F500D1B797B701009387E730135782
:106FF000C5003E9703470700011106CE2304E100B8
:10700000135785003D8B3E97034707002306010079
:10701000A304E100135745003D8B3D893E97AA9795
:107020000347070083C7070028002305E100A305E5
:10703000F10097000000E78080F4F2400561828053
:1070400081473307F600030707000DE363E4F50209
:107050004111B2853E8606C697900100E78000A1E7
:10706000B240133715003A85410182808507C20777
:10707000C183C1BF3A858280797117B501001305BC
:10708000A52006D622D426D24AD04ECE97000000A4
:10709000E780E0EE17E5FF1F0355A56B97000000A2
:1070A000E780A0F497E7FF1F83C7475A17B5010091
:1070B0001305051B89C717B501001305E5199700CE
:1070C0000000E780C0EB17B501001305251C9700F1
:1070D0000000E780C0EA17B501001305A51B970063
:1070E0000000E780C0E9114597000000E780E0EA72
:1070F00017B501001305857897000000E78020E8A8
:10710000014597000000E78040E917B5010013052D
:10711000E57697000000E78080E6130510059700EC
:107120000000E78080E797D7FF1F83C7F71117B5E7
:1071300001001305651389E717B501001305451311
:1071400097000000E780A0E317B5010013050515BF
:1071500097000000E780A0E237A50700130505129D
:1071600097000000E78060E317B501001305851361
:1071700097000000E780A0E097E7FF1F83C7475F05
:1071800017B501001305450F89E717B50100130571
:10719000250F97000000E78080DE17B5010013057A
:1071A000251197000000E78080DD17B50100130569
:1071B000A51097000000E78080DC17B501001305DB
:1071C000251097000000E78080DB17C5FF1F0355DF
:1071D000651E97000000E78040E117B50100130528
:1071E000650E97000000E78080D917C5FF1F035583
:1071F000C51E97000000E78040DF17B501001305AA
:10720000E50C97000000E78080D717D5FF1F0355D6
:1072100005EA97000000E78040DD17B5010013057F
:10722000650B97000000E78080D517D5FF1F035539
:10723000C5E797000000E78040DB17B501001305A4
:10724000E50997000000E78080D317D5FF1F03559D
:10725000E5E597000000E78040D917B50100130568
:10726000250897000000E78080D117C5FF1F035550
:10727000250597000000E78040D717B501001305EA
:10728000A50697000000E78080CF014497C9FF1F43
:107290009389895D97B40100938404061949B30763
:1072A000340183C707000A85050413D74700BD8B47
:1072B0002697A6970347070083C70700230101000D
:1072C0002300E100A300F10097000000E78020CB3D
:1072D000E31724FD17B50100130585019700000091
:1072E000E780E0C90A8597E0FFFFE780E02C0A8489
:1072F000040883470400034514000904A2075D8DB8
:1073000097000000E78060CEE39584FEB2502254DF
:1073100092540259F24945618280411126C2E977AF
:1073200097E4FF1F9384045922C49387A7552E84A2
:107330002381B4002E86AA8517E5FF1F1305C557C4
:1073400006C62390F400A381040097800100E78023
:10735000407493052400C205C18117E5FF1F130582
:10736000855597F0FFFFE7808050B3878400238224
:10737000A7002181A382A700930564002244B240A4
:1073800026859244C205C181410117230000670090
:10739000435409C99307000463E6B70017030000CC
:1073A0006700E3F78280011106CE2307010081EE1A
:1073B00097B60100938606F497000000E78040B975
:1073C000F2400561828058002A88AE883283A9473E
:1073D0003A85A945254E33F6B602FD1793F7F70F08
:1073E00013060603A304C70033D6B6026375DE0096
:1073F0007D17B286EDF3B306F5001A86C685428581
:1074000065BF5971A2D4A6D2CAD02E842A89B2846B
:1074100097B60100938686B2130680058145280041
:1074200086D697000000E780A0B2AA85CA86130618
:107430008005280097000000E78080B1AA8597B6F4
:107440000100938666B013068005280097000000AF
:10745000E78000B0AA85A68613068005280097005D
:107460000000E78080F4AA8597B60100938606AEF7
:1074700013068005280097000000E78060AD130721
:107480008002A2859307800263639700A687AA976C
:10749000C207C183130670051308E005631AF502DD
:1074A000AA8597B601009386A6AA13068005280030
:1074B00097000000E780C0A9AA8528009720000057
:1074C000E7802041B6502654965406596561828063
:1074D0001307250042074183E364E6FC03C7050068
:1074E000930607FE93F6F60F6374D8001307E002C5
:1074F00080109306150022952304E5FA13950601E2
:107500008505418161BF3571B706400022CD06CFA8
:1075100026CB4AC94EC752C517E7FF1F1307872559
:1075200001445946A506631FA4000145FA406A4478
:10753000DA444A49BA492A4A0D6182800504420464
:107540004180D5B783470700BA84D91793F7F70F5F
:107550006367F600B3D7F600858B0507E5F33304C0
:10756000854042044180BD4763E5870201476319B6
:10757000F40C3D4697B50100938505A726859780B5
:107580000100E780A04E31E117B501001305C5A643
:1075900005A0414697B50100938585A22685978071
:1075A0000100E780A04C71F517B50100130585A215
:1075B00097000000E780A09C97000000E78000ACE7
:1075C00017A501001305C516A9A4C14763F98706CD
:1075D000454697B50100938565A3268597800100F0
:1075E000E780C048014729ED97E0FFFFE780E026EC
:1075F000AA8417B501001305A5A297000000E78033
:107600000098268597000000E7802099014417C95B
:107610000100130929C9E38584FA4A85970000000F
:10762000E780E095228597E0FFFFE780A02305042F
:1076300097000000E780609B1374F40FE9BF0147D7
:10764000B70640005946A506B387E40083C7070084
:10765000131507014181D91793F7F70F636FF600F0
:10766000B3D7F600858B91CB050705059317070166
:107670004205C1834181E3E987FCB309A440C20903
:1076800093D90901A14763FC37113389A40025462A
:1076900097B501009385459A4A8597800100E78058
:1076A000E03C75EDA547638DF900834799003547A8
:1076B0006388E70029476385E70093F7F70DE5E363
:1076C00097B60100938606981306000481450818B2
:1076D00097000000E780C087AA8597B601009386CF
:1076E000A69713060004081897000000E78040865C
:1076F000AA8597B601009386E6961306000408183B
:1077000097000000E780C084AA8591461306000414
:10771000081897000000E78040C9AA8597B60100C5
:107720009386C61513060004081897000000E7802A
:107730002082AA8597B601009386C6BB1306000473
:10774000081897000000E780A080AA8597B601007E
:107750009386C61213060004081897F0FFFFE7800F
:10776000207FAA85930610051306000408189700C9
:107770000000E78080C3AA8597A60100938646FB98
:1077800013060004081897F0FFFFE780607CAA85C5
:10779000081897200000E780C013054541BB17B6C5
:1077A00001001306A68CA285268597000000E780BD
:1077B00060892DC5930724FFC207C1830D47637CF1
:1077C000F7021389E400114697A501009385C57B54
:1077D0004A8597800100E7806029630005181146FB
:1077E00097A50100938505774A8597800100E7807A
:1077F000E027630D051617B50100130525882286BD
:10780000A68597000000E78000C017B501001305AA
:10781000E58797F0FFFFE780807641B717B6010054
:1078200013060689A285268597000000E7808081DF
:107830006317051417B6010013068688A2852685EE
:1078400097000000E7800080631B051217B6010057
:1078500013064688A285268597F0FFFFE780807E85
:10786000630E054617A901001309097417AA010040
:10787000130A0A74A68517B501001305A58622868A
:1078800097000000E78020B8814713051004930596
:107890004004130820059308D0031387570093165C
:1078A0000701C182636ED412B386F40003C60600DA
:1078B0001376F60D631BA61203C616001376F60D9B
:1078C0006315B61203C626001376F60D631FB610B5
:1078D00003C636001376F60D6319061183C64600FB
:1078E000639516111D8C420441809307B4FFC207B3
:1078F000BA94C18305476375F70283C60400130772
:107900000003639FE60003C7140093068005137706
:10791000F70D6317D7006514931704018904C18319
:10792000814601441148A5489545139706014183B6
:1079300013F5F60F6385E70A639C060593170401A8
:10794000C187635FF00897E7FF1F83C727D0D5E3A0
:1079500017A501001305057C6DBD17A901001309CA
:10796000A96217AA0100130AAA6229B717A9010080
:107970001309495E17AA0100130A4A5EE5BD17A95B
:1079800001001309295F17AA0100130AEA5EDDB599
:107990003387D40003470700130607FD1373F60F60
:1079A00063E868001204518C420441808506B5BF2B
:1079B0001306F7FB1376F60F63E9C50012041307ED
:1079C00097FC418F13140701CDB71306F7F913760F
:1079D000F60F63E6C5001204130797FADDB739FD09
:1079E00017A50100130585702DB58507C207C18352
:1079F0006DB597E7FF1F83D7C7D517A501001305FE
:107A00006573E38887E0C16797C9FF1F83D9899AA7
:107A1000FD1781445D4717A501001305A573E38A8F
:107A2000F9DEB3079A0083870700139604014182A9
:107A300081C7639BE4285D462C08228597E0FFFF01
:107A4000E78060E497A6010093860673130600059D
:107A500081452A8A081897F0FFFFE780604FAA85C2
:107A600097A601009386C67213060005081897F0C2
:107A7000FFFFE780E04D1C01B386A7001357C40049
:107A800097B70100938747873E9703470700AA856A
:107A9000130600052386E6FA135784003D8B3E97B4
:107AA000034707000818A386E6FA135744003D8BE6
:107AB0003E97034707002387E6FA1377F400BA9747
:107AC00083C70700A387F6FA97A601009386C66CC2
:107AD00097F0FFFFE780C047AA85CA861306000516
:107AE000081897F0FFFFE780A046AA8597A6010037
:107AF0009386067D13060005081897F0FFFFE780C0
:107B00002045AA8597A6010093868668130600057E
:107B1000081897F0FFFFE780A0431C01B386A70079
:107B200013D7C90097A701009387077D3E970347A6
:107B30000700AA85130600052386E6FA13D78900F5
:107B40003D8B3E97034707000818A386E6FA13D734
:107B500049003D8B93F9F9003E97BE9983C7090010
:107B600003470700A387F6FA2387E6FA97A60100E2
:107B70009386066397F0FFFFE780803D2AC60145A4
:107B800097E0FFFFE78000CEB245AA8997A60100E3
:107B90009386066013060005081897F0FFFFE7803C
:107BA000203B13D7C9001C014207B386A7004183BD
:107BB00097A70100938747743E9703470700AA855C
:107BC000130600052386E6FA13D789003D8B3E97FE
:107BD000034707000818A386E6FA13D749003D8B30
:107BE00093F9F9003E97CE970347070083C7070034
:107BF0002387E6FAA387F6FA97A601009386C63490
:107C000097F0FFFFE780C034AA85A686130600051B
:107C1000081897F0FFFFE7804079AA8597A6010032
:107C20009386865813060005081897F0FFFFE78033
:107C30002032AA8563500A0A97A601009386465708
:107C400013060005081897F0FFFFE7806030B306C1
:107C5000404113060005AA85081897F0FFFFE7804A
:107C6000C074AA8597A60100938686AC130600050A
:107C7000081897F0FFFFE780A02DAA850818972025
:107C80000000E78000C517A501001305A552E31207
:107C90000AB817A501001305255497F0FFFFE780E8
:107CA000002E228597F0FFFFE780203417A5010002
:107CB0001305854E97F0FFFFE780602C4A8597F00B
:107CC000FFFFE780C02BEDB83408A6962380F600AE
:107CD000850481BBD28613060005BDBFC147E3F60C
:107CE0008784414697A50100938585502685978016
:107CF0000100E780A0D7E31A058283C704011307B8
:107D00001003639CE700854717E7FF1F2302F7A6D0
:107D100017A501001305054FEDBC1307000317A5B8
:107D2000010013052551E396E7AE97E7FF1F238176
:107D300007A417A501001305654EE1BC17E5FF1F59
:107D4000034505A38280397122DC26DA97A601005B
:107D500093868615130600032A84AE840A8581451E
:107D600006DE97F0FFFFE780A01EAA8597A6010018
:107D700093860642130600030A8597F0FFFFE7800B
:107D8000201D8D47AA8563F6A7041C18B386A7009B
:107D90001357C40097A70100938707563E970347E0
:107DA00007002386E6FC135784003D8B3E9703476C
:107DB0000700A386E6FC135744003D8B3D883E97A1
:107DC000A2970347070083C707002387E6FCA38722
:107DD000F6FC97A6010093862617130600030A8572
:107DE00097F0FFFFE780C016A686AA85130600035A
:107DF0000A8597F0FFFFE780405BAA8597A6010000
:107E000093860693130600030A8597F0FFFFE78029
:107E10002014AA850A8597200000E78080ABF250E5
:107E20006254D2542161828097E7FF1F83C747A81D
:107E300089E7172300006700C3A9828097E7FF1F27
:107E400083C7A7AB99EF411106C697200000E780D2
:107E500020A0B240854717E7FF1F2300F7AA410182
:107E60008280828063090540638705401D71CAC80E
:107E7000CEC686CEA2CCA6CAD2C4D6C2DAC05EDE38
:107E800062DC66DA6AD86ED6B947AA892E8963FFA2
:107E9000B708394697A501009385C5029780010070
:107EA000E780C0BC41E583C7E90013071003639670
:107EB000E704854717E7FF1F230CF79E17A501006E
:107EC0001305450197E7FF1F2393079E97E7FF1FC1
:107ED000239A078E97F0FFFFE780600AF64066441A
:107EE000D6444649B649264A964A064BF25B625C3E
:107EF000D25C425DB25D256182801307000317A545
:107F0000010013052500E397E7FC97E7FF1F238196
:107F1000079A97E7FF1F239C079897E7FF1F239374
:107F2000078A17A50100130565FC6DB797E7FF1FCA
:107F300083C707986394072C8144B54A17EAFF1F4B
:107F4000130A4A8317AB0100130B0BFEA94B130C4A
:107F5000E00497AC0100938CACFD93970401C183BE
:107F600017E4FF1F0354048663E8272B25D817A6C0
:107F700001001306A60FA28517D5FF1F1305857FE5
:107F800097F0FFFFE780000C31F917A601001306F8
:107F90002612A28517D5FF1F1305C57D97F0FFFF99
:107FA000E780400A05FD17A6010013066611A285A9
:107FB00017D5FF1F1305057C97F0FFFFE7808008AA
:107FC00011FD17A601001306E610A28517D5FF1FA5
:107FD0001305457A97F0FFFFE780C00601F122857F
:107FE00097F0FFFFE7806052E30A05EE97D7FF1F87
:107FF000239A077CE5B5B387490183C6070097E755
:10800000FF1F83D7C78A8DE79307A005639BF60000
:10801000854717E7FF1F231CF78897D7FF1F238586
:10802000D77A050A93170A01C183E3E627FD7DB5D8
:10803000854D639BB7039307500A639EF6008947FB
:1080400017E7FF1F2315F786930750FA17D7FF1F6F
:10805000A30CF776F9B79307A005E384F6FC97E73E
:10806000FF1F2396078475BF138717004207DA970F
:1080700041832380D70017E6FF1F231AE6828D472E
:10808000E3F1E7FA17D4FF1F0344347497D7FF1FB7
:1080900083C7A77322045D8C9307F4FFC207C183D3
:1080A0009306F00DE3EDF6FA93076400C207C1836F
:1080B000E319F7F693052400C205C18117D5FF1F08
:1080C0001305A57097E0FFFFE780607A33078B0008
:1080D0008347570003474700A207D98F17D7FF1FD1
:1080E0002317077C6311F5108144630CB40197D406
:1080F000FF1F83C4A46DA20497D7FF1F83C7176D0A
:10810000DD8C17F5FFFF1305052997E0FFFFE780DA
:10811000200F6385740963EF9B026388A4059307AE
:10812000EC656383F40697D7FF1F83C7276A05476B
:108130006380E70881CB1387A7051377F70F8D4678
:1081400063F9E6081307F0072300E100A300F1003C
:10815000894595A8638994059387FA77E395F4FC9C
:1081600097E0FFFFE780005111A8A28517D5FF1FF8
:108170001305C56597E0FFFFE7808019014597E08B
:10818000FFFFE780E00771BDA28517D5FF1F13052C
:10819000E56397E0FFFFE780A020CDB797E0FFFF02
:1081A000E7802029E1BF97E0FFFFE780C02EF9B705
:1081B000930710F8130511002300F10097E0FFFF6B
:1081C000E780204EFD450A8597F0FFFFE7802015E8
:1081D00075B7A28517D5FF1F1305455F97E0FFFF11
:1081E000E780A0D861BF9307F00789450A8523106F
:1081F000F10097F0FFFFE780801225B5BD6A396C6A
:10820000014A17DBFF1F130B2B5C938BFA55938CE2
:10821000FA66130DEC5539B5B387990083C707008B
:10822000638457016398770329C0228597F0FFFF85
:10823000E780A02D19E917D6FF1F0356A658D2854F
:108240005A8597F0FFFFE780001C97D7FF1F239BFD
:10825000075621A8636D8C0013071400529497D61B
:10826000FF1F2391E6562300F4008504FDB122860A
:10827000D2856685F9B78280411126C2AE848D45CC
:1082800022C406C62A8497B0FFFFE78060C0B717F4
:10829000004099C803A5C70C418D23A6A70CB24086
:1082A000224492444101828003A5870C418D23A47E
:1082B000A70CF5B78347050003471500A207D98F20
:1082C000C2076177C18713072720639AE7008345B8
:1082D00025003705040017030000670023FA828099
:1082E00017D6FF1F1306C6618147B2861303F00F2E
:1082F000A9483308F6000348080013F7F70F63078F
:10830000A80C630668008507E39517FF2947B38724
:10831000E6002380A70097D7FF1F9387275F5DA8FC
:10832000411113D765001347170006C693F63500B1
:10833000058B954791CA054699476387C60009464C
:108340009D476383C600A14713F645003336C0003E
:1083500093F68503050685C2A145638BB604E14506
:10836000638AB604930580026388B604930580038C
:108370006393B600914697D5FF1F238EF57E97D560
:10838000FF1F2389C57E97D5FF1FA385D57EBE8598
:1083900017A50100130545FA97700100E780C07A20
:1083A000B240854717D7FF1FA307F77C41018280A2
:1083B0008546D1B78946C1B78D4675BF17A501005F
:1083C000130505FA177301006700037817D7FF1F1D
:1083D0001307C753BA972380B700E147E302F5F4C8
:1083E00093077002E30CF5FC82802A872380050046
:1083F000814717D5FF1F1305A5501308F00F294615
:10840000B306F50083C606006396E60297D6FF1F03
:108410009386C64FB69783C7070005452380F500AE
:108420009947636EF7029D4763FDE700E147630DDF
:10843000F7008280638506018507E393C7FC014549
:10844000C5B7238005008280B737004003C73700D7
:1084500083C7050093F70704D98F2380F500828036
:108460005D7152DC56DA5ED6716A97EBFF1F938B13
:10847000AB818D6AA6C24EDE62D486C6A2C4CAC0D3
:108480005AD866D26AD06ECEC1495E8C97D4FF1F8F
:1084900093848448130A0A20938A7ADC17E9FF1F21
:1084A00003498981B3872B0183C7070093F7F70F2F
:1084B000C9EFB787004003C76700058BE310077C4F
:1084C00003C76700118BE30D077E83C75700918BAD
:1084D00099E36F10200317D7FF1F0347077E8547D7
:1084E0006304F7006F10400197D7FF1FA385E7686B
:1084F00097D7FF1F2382074E97D7FF1F2380075A66
:1085000097D7FF1F238E076497D7FF1F238B07641E
:1085100097D7FF1FA382074C97D7FF1FA380075849
:1085200097D7FF1FA38E076297D7FF1FA38B076202
:1085300097D7FF1FA382076497D7FF1FA38F0776E4
:10854000B787004011476F0070779307190093F7C2
:10855000F70F3D476364F70617D7FF1F230EF77425
:1085600097D7FF1F93874774CA9783C707001307DE
:10857000100293F7F703638EE71E6366F704054462
:108580006385871CE38C07620947638EE710130736
:108590000002E384E74EB7E700E03707400023A07E
:1085A000E71801000100629923000900FD1923A0CA
:1085B000E71093F9F90FE39309EEE5BD97D7FF1F95
:1085C000238C076E71BF130730026388E70C63E8E2
:1085D000E71613074002638CE70A13070003E39CC6
:1085E000E7FA97D7FF1F9387276BCA9703C7070040
:1085F000A1471377F70FE31BF71483C7640097D6DF
:10860000FF1F2381F65697D7FF1F83C7573191C7A6
:10861000FD5797D6FF1F2387F65497D5FF1F83C5B5
:10862000B52F97D7FF1FA38FB75297D7FF1F83C7C9
:10863000A72E13FB07089306000493F70706639F12
:10864000D74C9307A009638DF51663EAB712930719
:10865000F0056386F54A930750096384F52A0144BF
:1086600097D7FF1F83C717501547E392E736B7E741
:1086700000E03707400023A0E71801000100B7869B
:10868000004023808602130680FC6F00500EFD57C9
:1086900017D7FF1F2307F74CFDBDFD5717D7FF1F47
:1086A0002300F74CCDBD17A501001305E5DC97703D
:1086B0000100E780406197D7FF1F9387E75DCA9766
:1086C00003C40700014B97DCFF1F938C6C3D1374B0
:1086D000F40F17AD0100130DADDA63478B04294584
:1086E00097700100E780204B854717D7FF1FA3072E
:1086F000F73A17D7FF1F2304873A17D7FF1F230D19
:10870000F74637E700E0B70640002320D7180100FE
:108710000100378600408347A60293F7370F2305F1
:10872000F6022320D71085BDB3876C0183C50700EF
:108730006A85050B97700100E780004179BF854786
:1087400017D7FF1F230CF734B9B517D7FF1F13072F
:10875000A7544A970347070097D6FF1FA38EF62614
:1087600097D6FF1F238BE62617D7FF1F2306F74058
:108770001DB5854717D7FF1F2300F72629BD93078F
:10878000400A6389F5349307200B6384F536930719
:10879000100AE396F5EC838724000144E3D207EC4A
:1087A00097D7FF1F83C7771793F63700638A061A98
:1087B0000546638AC62209466395C61A1D4755A217
:1087C00017D5FF1F03456515C94797DCFF1F83CCED
:1087D000DC1497D5FF1F83C5651417D4FF1F03440E
:1087E000F4136315F510CD476392FC1093077008DE
:1087F000639CF5021307300FB7170E006308E400FF
:108800001307900DB7B704006314E40817D7FF1FD0
:108810002320F736BE8517A501001305E5C697701E
:108820000100E780603225BD93078008639DF50055
:10883000B307804013F4F70FB7774600938787CDCF
:10884000B3D78702E1B793079008639AF500B3079F
:10885000804013F4F70F91679387C766D5B79307E6
:10886000A008639BF500B307804013F4F70FB71718
:108870003D0093870790E9B79307B008639AF50026
:10888000B307804013F4F70F9167938797D04DBFDC
:1088900093F5F5078D47639BF500B307804013F40C
:1088A000F70FB7975B00938707D859BF8947639B3A
:1088B000F500B307804013F4F70FB7770B009387E9
:1088C000071BBDBF8547639AF500B307804013F4CB
:1088D000F70FDD67938767E3A5B7D28785F9B307FD
:1088E000804093F7F70FB3D7FA020DB79700000057
:1088F000E780409FA285668597000000E780809E04
:10890000B9BB9305610017D5FF1F0345050117D4B7
:10891000FF1F0344940097000000E78040AD9305DB
:108920007100228597000000E78060AC3C0017D7FB
:10893000FF1F2329F734834761002304F100834795
:108940007100A304F100894717D7FF1F230CF720FC
:108950008357810017D7FF1F2310F7FC094409B381
:10896000154793F64700B336D00093F78703850683
:1089700085C32146638BC7066146638AC706130613
:1089800080026388C706130680036393C70091477C
:1089900017D6FF1F2300D61E97D6FF1FA38CF61CE9
:1089A00097D7FF1F2389E71C17D7FF1F034707F738
:1089B0009376070497D7FF1F83C757F68DEE13777B
:1089C000770C93067008630CD7021377F7078D4670
:1089D0006312D70CB307F040B7955B0093F7F70F1E
:1089E000938505D849A81947ADBF854755B789472D
:1089F00045B78D4771BF930670086311D7021307FF
:108A0000300FB7150E006389E7021307900DB7B555
:108A100004006383E7021307700845BF9306800CC8
:108A20006311D702B307F040B775460013F7F70F8D
:108A3000938785CDB3D5E70297D7FF1F23AAB71237
:108A4000D9BB9306900C631CD700B307F04093F595
:108A5000F70F91679387C766B3D5B702F1BF930647
:108A6000A00C631DD700B307F040B7153D0093F786
:108A7000F70F93850590B3D5F5027DBF9306B00C33
:108A8000E315D7F4B307F04093F5F70F9167938799
:108A900097D0D9B78946631BD700B307F040B775A5
:108AA0000B0093F7F70F9385051BF1B78546631A03
:108AB000D700B307F040DD6593F7F70F938565E3C3
:108AC0005DBFD28535FBB305F04093F5F50FB3D507
:108AD000BA029DB783C72400C18B99C7854717D7B2
:108AE000FF1F2304F708A5BE97D7FF1F238F070694
:108AF000BDB6854717D7FF1FA30FF7068DB63C00FD
:108B000017D7FF1F2320F7180947930700032314E3
:108B1000F10097D6FF1F2387E6042DBD6394075607
:108B2000A94763E5B742179701001307277E8A0517
:108B3000BA959C41BA97828717D4FF1F0344F4DD8E
:108B4000894C6306940D63E68C0685476303F4083D
:108B50009307F00F17D7FF1F0347C70063F6E7001F
:108B600017D7FF1F2300F70097DCFF1F83CC8CFF74
:108B70009307000413F4FC0F63F49701130400043B
:108B800097D7FF1F9387071003AD0700228626851E
:108B9000EA85B38C8C40229D97700100E78060EFDE
:108BA00097D7FF1F238097FD97D7FF1F23ACA70DF3
:108BB00045BC8D47630CF40A9947E31BF4F897977B
:108BC00001009387277B17D7FF1F232DF70AA9479B
:108BD00051B717D7FF1F0347470E97D7FF1F93873C
:108BE00067FA494697A501009385C581630687000A
:108BF000979501009385057D3E8597700100E7807C
:108C000040E917D7FF1F232FA706C947A1B797D65B
:108C1000FF1F83C6860A054797D7FF1F938787F6EE
:108C20006394E6023E8513067002979501009385D2
:108C3000E57A97700100E780C0E517D7FF1F23236F
:108C4000A7049307700239B73E8513063004979541
:108C500001009385E57297700100E78080E317D7E4
:108C6000FF1F2321A70293073004EDB597D5FF1FFF
:108C700083C5A5CA17A50100130545829770010099
:108C8000E78080EC054D97DDFF1F83CD0D0397D561
:108C9000FF1F83C585C817A50100130525806398AC
:108CA000AD0B97700100E78020EA97D7FF1F83C7BD
:108CB000C7C6B5CBE36EF4E8179401001304C4787B
:108CC000638CB701179401001304847863869701BD
:108CD0001794010013044479228597700100E780FE
:108CE000C0FF1375F50F93071500860717D7FF1FF1
:108CF000230AF7E88D4717D7FF1FA305F7E897D793
:108D0000FF1F938727E80147BE861376F70F890771
:108D10006365A60297D7FF1F23A6D7F697D7FF1F35
:108D200083C747E605BD979701009387E76A17D782
:108D3000FF1F2329F7F4914731BD3306E4000346B2
:108D40000600A380070005072380C7007DBF97703A
:108D50000100E78060DF97D7FF1F83C707BCE1D71B
:108D6000E368F4DE179401001304046B638CA7011D
:108D7000179401001304C46A6386970117940100D5
:108D80001304846B228597700100E78000F513754A
:108D9000F50F93071500860717D7FF1F2304F7DE8B
:108DA0008D4717D7FF1FA30FF7DC97D7FF1F9387B8
:108DB00067DD0147BE861376F70F8907E37CA6F4CB
:108DC0003306E40003460600A3800700050723805E
:108DD000C700D5B797D5FF1F83C525B417950100E8
:108DE0001305856C97700100E78000D697D7FF1FA9
:108DF00083C717D993E7470017D7FF1FA302F7D8F8
:108E000083C7240017D7FF1FA30AF7D689B8179581
:108E100001001305A56A97700100E780C0EA97D7A3
:108E2000FF1F9387A7D583C7070017D7FF1F230509
:108E3000F7AE17D4FF1F0344E4D2333480000DB0E3
:108E4000179501001305C56897700100E780A0E73A
:108E500097D7FF1F83C7D7D293E7070117D7FF1F05
:108E6000A300F7D283C7240017D7FF1F2308F7D02A
:108E70006FF0EFFE179501001305C56697700100AE
:108E8000E78060E403C704007D8B51EFB7870040A3
:108E900003C767021377C70B136727002383E70213
:108EA00003C7A7021377C70B136727002385E702C1
:108EB00003C7E7021377C70B136727002387E7026F
:108EC00003C727031377C70B136727002389E7021C
:108ED000854717D7FF1F2301F7B017D7FF1F230FB1
:108EE000F7BA17D7FF1F230DF7C617D7FF1F230A9F
:108EF000F7C697D7FF1FA38107AE97D7FF1FA38F92
:108F000007B897D7FF1FA38D07C497D7FF1FA38A62
:108F100007C497D7FF1FA38107C697D7FF1FA38E4C
:108F200007D86FF0CFF389476312F70297D7FF1F77
:108F300083C7C79E9146638CD70863E0F604638EAF
:108F4000E70C6369F70A05476380E70EFD5717D7FB
:108F5000FF1FA309F7C037074000B7E700E023A0D1
:108F6000E71801000100B78600401306F0FC2381DA
:108F7000C60223A0E7106FF00FE2130720086382F8
:108F8000E7086362F70213071008E391E7FC3787ED
:108F900000408347670293F7C70B93E7270023033B
:108FA000F7026FF0CFEB130730086389E70213076E
:108FB0004008E39DE7F8378700408347270393F78E
:108FC000C70B93E727002309F7026FF04FE93787B4
:108FD00000408347270393F73707F5B737870040EB
:108FE0008347E70293F7C70B93E727002307F702AE
:108FF0006FF0EFE6378700408347E70293F73707C4
:10900000F5B7378700408347A70293F7C70B93E76D
:1090100027002305F7026FF08FE43787004083476E
:10902000A70293F73707F5B73787004083476702F2
:1090300093F73707ADB7179501001305A54B977048
:109040000100E78040C897D7FF1F2387078CD5B35F
:10905000179501001305054B97700100E780A0C626
:1090600097D7FF1F239A078A97D7FF1F938787AF4A
:1090700003C40700894763F3870009441374F40F9E
:109080006FF00FDE13070002E392E7EC631B0B0A9D
:10909000638FF500930720026383F508179501009D
:1090A0001305C54997700100E78000AA45B51795DB
:1090B00001001305E54597700100E780C0C0014439
:1090C000179D0100130D0D46A14CB387840083C585
:1090D00007006A85050497700100E780E0A6E316A3
:1090E00094FF178501001305A56A97700100E780BA
:1090F00080BD17D4FF1F0344648201E897C7FF1F98
:10910000238E077E014B6FF0AFD58947E310F4E45F
:10911000854717C7FF1F2303F77E6FF04FD417C68D
:10912000FF1F0346967F97C5FF1F83C5057F1795D1
:1091300001001305A53F97700100E780E0A06FF0E4
:109140000FD26380F50693071002E399F5F497C5F3
:10915000FF1F83C5A57C179501001305253F977058
:109160000100E780609E97D7FF1F23AD97B097D788
:10917000FF1F9387E79F944383D7470017D7FF1FAD
:109180000347679F17C6FF1F2328D6781D4497C63D
:10919000FF1F2395F67897C7FF1F2382E7786FF0AC
:1091A0002FCC97C5FF1F83C5657717950100130561
:1091B000653B97700100E780209997C7FF1F238FB9
:1091C000077297C7FF1F239907746FF02FF9254780
:1091D000638FE7C89946378700406394D70223001E
:1091E0008702B7E700E0B706400023A0D7180100C8
:1091F0000100130600FC2301C70223A0D7106FF063
:109200008FB99306100A639FD70023008702B7E740
:1092100000E0B706400023A0D718010001001306A4
:1092200080FCD1BF9306A009E381D7FE9306400AD4
:10923000E38DD7FC93062002639DD700B7E700E0DB
:10924000B706400023A0D7180100010023008702C1
:10925000F9B78546E384D7FE93070008E300FBFED9
:10926000B7E700E0B706400023A0D71801000100CF
:10927000130620FC23008702BDBF17D7FF1F03473B
:10928000778E6302F71E63E7E70295476300F710E6
:109290009947630AF704B786004023800602B7E7C0
:1092A00000E03707400023A0E71801000100130683
:1092B000A0FC75B99307F005630AF70093075009FE
:1092C0006306F70093071002E317F7FCB7E700E027
:1092D0003707400023A0E71801000100B7860040CF
:1092E000130620FC69B117DBFF1F034BAB87930705
:1092F00000045A8D63F46701130D000497D7FF1F14
:109300009387479883AC07001374FD0F2286E68588
:10931000268597600100E780C077B3078B4066948D
:1093200017D7FF1F2300F78497D7FF1F23AC87941D
:10933000B7870040630C0B022380A703B7E600E069
:109340003706400023A0C6180100010003C727020A
:10935000134707042381E70203C727021377C70FC8
:109360002381E70223A0C6106FF0EFA2238007023B
:1093700037E700E0B70640002320D71801000100BE
:10938000130620FC2381C7026FF0AFB93787004076
:109390008347370097C6FF1F83C6567E93F707089B
:1093A000D58FA301F700B7064000B7E700E023A080
:1093B000D718010001001306A0FC35BD97D7FF1F89
:1093C0009387878DCA9783C7070093F7F70FC1CF9D
:1093D00097D7FF1F83C7678ED9E717C7FF1F0347BC
:1093E0007778930700026310F70883AD040017CD68
:1093F000FF1F034DAD5297CCFF1F83CC3C5217CBC0
:10940000FF1F034BCB51E6876A87DA866E8697C5C6
:10941000FF1F83C5A54E17950100130525169760FC
:109420000100E780607297C7FF1F23A3B77597C736
:10943000FF1F2381A77597C7FF1FA38D977397C73A
:10944000FF1F238A677397C7FF1FA388874AB7E761
:1094500000E03707400023A0E71801000100B786AD
:1094600000406FF04FA2B7E700E03707400023A0AD
:10947000E71801000100B786004015BD97D6FF1F11
:1094800083C6A6830547639CE60429472381E70238
:1094900009472383E7022385E70297C7FF1FA38DB0
:1094A000076C97D7FF1FA38A0780B7870040A38167
:1094B000070017C7FF1FA303076C05472383E700B7
:1094C000B640264496440649F259625AD25A425B43
:1094D000B25B225C925C025DF24D61618280294741
:1094E0002381E70209472383E7022385E7022387D5
:1094F000E7022389E70255B717C7FF1FA30FF73EFF
:109500006FE01FFF854717C7FF1F2307F74C17C7DB
:10951000FF1F2305F75817C7FF1F2303F76417C75B
:10952000FF1F2300F7646FE0BFFE854717C7FF1FCB
:109530002304F74A17C7FF1F2302F75617C7FF1F59
:109540002300F76217C7FF1F230DF76017C7FF1F20
:10955000A304074817C7FF1FA302075417C7FF1F1D
:10956000A300076097C7FF1FA38D075E828041118C
:1095700006C697000000E78080FBB7870040238085
:109580000700130740FC2386E7001307C004A386E7
:10959000E70017C7FF1F130727382398E70017C7EF
:1095A000FF1F1307673B239AE70017C7FF1F130727
:1095B000E746239CE70017C7FF1F13076752239E48
:1095C000E70029472381E70209472383E702238530
:1095D000E7022387E7022389E702A38107009306B6
:1095E00000F8A380D700930690022380D700FD5691
:1095F0002383D7002381E7009306000537E700E0C7
:10960000230BD740B70640002320D71003C717000D
:1096100013671700A380E700B24097C7FF1F239F7F
:10962000075441018280411106C697000000E7807F
:1096300000F0B787004023800700130700FC238653
:10964000E7003147A386E70017C7FF1F1307C72CA2
:109650002398E70017C7FF1F13070730239AE70077
:1096600017C7FF1F1307873B239CE7002947238168
:10967000E70209472383E7022385E702A381070066
:10968000930600F8A380D700930690022380D700AA
:10969000FD562383D7002381E7009306000537E7B3
:1096A00000E0230BD740B70640002320D71003C7A4
:1096B000170013671700A380E700B24097C7FF1F8A
:1096C000239E074A41018280F1679387072017C7CD
:1096D000FF1F232FF748854717C7FF1F231CF74895
:1096E000A14717C7FF1F2308F74897C7FF1FA38489
:1096F000074897C7FF1F2381074897C7FF1F238F7E
:10970000071E97C7FF1FA38A071E814717C5FF1FA4
:109710001305051FFD5517C6FF1F1306261F2947F2
:10972000B306F5002380B600B306F60023800600DA
:109730008507E397E7FE97C7FF1FA386074297C7F2
:10974000FF1FA384074297C7FF1F238F074097C7B8
:10975000FF1F238A074097C7FF1F2389074097C72A
:10976000FF1FA383074097C7FF1F23800740814740
:1097700017C6FF1F130646514147B306F600238064
:1097800006008507E39BE7FE828017C7FF1F03479C
:10979000C75285476316F700170300006700E3E828
:1097A000170300006700E3DC411122C406C617C797
:1097B000FF1F0347875085472E8613F4F50FAA85B0
:1097C0006317F70417C5FF1F1305452997600100AC
:1097D000E780202C97C7FF1F2382072CB787004004
:1097E00023848702B7E600E03706400023A0C618AE
:1097F0000100010003C7A7021377C70F2385E70203
:10980000B240224423A0C61001454101828017C501
:10981000FF1F1305651897600100E780802797C731
:10982000FF1F238B071AB787004023828702B7E602
:1098300000E03706400023A0C6180100010003C75E
:1098400067021377C70F2383E7025DBF411106C686
:1098500097000000E78080E7B24041011703000055
:109860006700E3F2411106C697F0FFFFE78080BF73
:1098700097C7FF1F83C75716A1CB97C5FF1F83C587
:10988000C51589C917C5FF1F1305451597E0FFFFCB
:10989000E780805D97C7FF1FA380071497C7FF1F4E
:1098A000238C072C37E700E0B70640002320D718A9
:1098B00001000100378600408347660293F7370FA7
:1098C0002303F6022320D710B2404101828041C910
:1098D000D9C597C7FF1F83C7672AD1C3011122CCFF
:1098E0004AC84EC656C25AC006CE26CA52C42E898F
:1098F000AA890144930A0004371B030063772403F9
:10990000B3078940C207C183BE8463F4FA0093049D
:109910000004C204C180130A1BD497C7FF1F83C76A
:10992000A70B9DE37D1A631C0A00F2406244D244F7
:109930004249B249224A924A024B0561828097F01D
:10994000FFFFE78020B2D1BF338589002694A6852A
:10995000420497000000E78060E5418045B78280BF
:1099600097C7FF1F9387C74718429C4383D645007C
:109970000345070083C5C700035646006396A5004C
:1099800083D5E700638DD502011106CE2386A7009B
:109990002397D700B705CF00DC4B9385757D05076E
:1099A0007D162EC2230001003AC42316C1002317DE
:1099B000D10099C30A858297F24005618280828036
:1099C000411122C417A4FF1F130484A35C4C06C6D4
:1099D00091CBC84B01C9B7E70400BC5782975C4CD8
:1099E00023AA0700B240224441018280DC4DDC4BB7
:1099F00081CFB7E70400904503A38705914517C5BC
:109A0000FF1F0345253E02838280B7E7040003A3BE
:109A10000705A14517C5FF1F0345C53C02836D71AE
:109A20003C083EC6B707E500232291103EC8AA8431
:109A30003C083285232611103ECA2324811023209E
:109A400021112E8997300000E780605A2A8497956B
:109A50000100938525B6177501001305E56E976023
:109A60000100E780600EA28517950100130545C12E
:109A700097600100E780400D294597600100E7806D
:109A80008011B705CB009385757D680097100000A5
:109A9000E780E05FA285680097300000E78080479C
:109AA000014781467000CA85268597200000E7801F
:109AB000608305CD2A84979501009385A5AF17751E
:109AC00001001305656897600100E780E007A28543
:109AD00017950100130585BB97600100E780C0065C
:109AE000294597600100E780000B8320C110032403
:109AF000811083244110032901105161828097C78E
:109B0000FF1F9387E72D18429C43797122D406D614
:109B10000348070083C807012A8483D645000355FC
:109B200046006396080183D82701638DD8022388F5
:109B3000070105072399D7003708CC00DC4B130831
:109B4000787D3ACC1307F5FF42CA23080100231E93
:109B5000E100231FD10099C7080832C62EC482979E
:109B60003246A245228597000000E78080EBB25084
:109B70002254456182807971314697750100938541
:109B8000654D280006D697600100E78080F097A712
:109B9000FF1F83D7E786231B0100231C0100231D21
:109BA0000100231E0100231F010099E3C167FD1777
:109BB000231AF10097A7FF1F83D7A78491EB97C7BC
:109BC000FF1F9387E7219C439C43DC4783D7070013
:109BD00097A6FF1F9386C682231BF100D84E83D71A
:109BE0004600231CF1005C4B91CB97A7FF1F83C756
:109BF000978181EB97000000E780C0DCB25045619F
:109C00008280FD171796FF1FA30FF67E03560701EC
:109C100083C706014C472800230FF100973000004E
:109C2000E780602C97C7FF1F9387871B9C430147E2
:109C300097960100938686A1884330004C089710C0
:109C40000000E780206A5DD975B799C9B7E70400BD
:109C500003A30705A14517C5FF1F0345A5180283E8
:109C600082805C4EDC4BB9CFB1CD411122C4177557
:109C700001001305654D2E84979501009385C598C5
:109C800006C697600100E78020ECA28517950100C9
:109C90001305C59997600100E78000EB294597609F
:109CA0000100E78040EFB7E704002244B24003A37D
:109CB000870517C5FF1F0345E512130640069145AA
:109CC000410102838280411122C41794FF1F1304B3
:109CD000E4701C4C06C689C7DC4399C34C48829784
:109CE000584CB7E70400BC57484B82975C4CB240D5
:109CF000224423AA0700410182801797FF1F130700
:109D0000E76F834707009306F00B850793F7F70F7C
:109D100063E9F6009796FF1F2382F66E034507005E
:109D20008280930700F8FDB78357450099E37D557E
:109D30008280011122CC1794FF1F1304646C5C4CC9
:109D40004AC84EC6DC4B52C406CE26CA56C2B28999
:109D50002E8A2A898DC7B7E70400FC5F829797C7D0
:109D6000FF1F9387E7059C431307301FB307F54098
:109D700071556375F70697000000E780A0C493074C
:109D8000D00D7D5563EC3705B7E404009387890057
:109D9000B858832AC401139507014181029723AA69
:109DA000AA00484C584921E7979501009385C5833F
:109DB000177501001305453997600100E780C0D889
:109DC000179501001305458F97600100E780C0D704
:109DD000294597600100E78000DC5D55F240624450
:109DE000D2444249B249224A924A0561828013878D
:109DF0004900B705CF002319E5009385757D31052E
:109E000097100000E780A028484C83456900310581
:109E100097300000E7800010484C4E86D28531050F
:109E200097300000E780200C7146CA851795FF1F08
:109E30001305055D97600100E780A0C5FC5C829773
:109E40000326C90097C7FF1F23ACA7F611CABC4C55
:109E5000854517C5FF1F0345E5F882970145BDBF3E
:109E600097000000E78060D1D5BF411106C622C42B
:109E700026C217C4FF1F1304E4F697000000E78012
:109E800060B4B7E40400FC4C0345040085458297A8
:109E900003450400224403A3C405B2409244A145F3
:109EA00041010283411126C297C4FF1F938444F3EA
:109EB0009C4006C622C44AC0D5C3DC43C5C35CC1AE
:109EC0002300B5002A84978501009385256D1775B9
:109ED00001001305652797600100E780E0C629456A
:109EE00097600100E78020CB9C4023A4070023A2B9
:109EF00007009797FF1F9387674EDC4FDC4B91C796
:109F0000295597000000E78040DC9797FF1F938753
:109F1000274FDC4FDC4B89C797000000E78020F516
:109F200037E904008327C905894517C5FF1F034585
:109F300065EB82978327C905914517C5FF1F034528
:109F400065EA82979C4003A34701630903002285C9
:109F50002244B2409244024941010283B240224469
:109F600092440249410182800111328506CE22CC01
:109F700026CA2E8497300000E7806007AA84978560
:109F800001009385E564177501001305E51B9760D3
:109F90000100E78060BB030784000356640083551B
:109FA0004400A686178501001305C56A9760010065
:109FB000E78080B9294597600100E780C0BD979789
:109FC000FF1F83C70742639D97000145970000006C
:109FD000E780A0CF81450A8597000000E780C0ECAC
:109FE000F2406244D244056182806D712324811065
:109FF000232611102322911093F745002E846387A6
:10A0000007143C083EC0B707E5003EC23C083EC40A
:10A01000231701002318010023190100231A01004E
:10A02000231B01009797FF1F83D7473B99E3C16725
:10A03000FD172316F1009797FF1F83D7473A91EB3F
:10A0400097C7FF1F9387C7D99C439C43DC4783D79F
:10A0500007001797FF1F130767382317F100544FA6
:10A06000835747002318F100DC4AA1E797850100D8
:10A070009385455A177501001305050D976001007A
:10A08000E78080AC178501001305856997600100A2
:10A09000E78080AB294597600100E780C0AF13459A
:10A0A00044008320C1100324811083244110516196
:10A0B00082809797FF1F83C7D7322555D9C3FD17D5
:10A0C0001796FF1FA30FF63003D60601834707013B
:10A0D000CC460A85230BF10097300000E780A0E012
:10A0E00097C7FF1F9387C7CF9C431797FF1F13077F
:10A0F000E72E978601009386E65288430A866C0015
:10A1000097100000E780001EAA8451D997850100AE
:10A1100093854550177501001305050397600100ED
:10A12000E78080A2A685178501001305256097604A
:10A130000100E78060A1294597600100E780A0A5A4
:10A14000268597000000E78040B891BF93F725006F
:10A150009DC7B7E70400BC47414681452808829760
:10A16000255597000000E78040B628089305F00FBA
:10A1700097000000E78040D3134524001DB793F7F4
:10A18000150081CB97000000E780209F1345140045
:10A1900009BF93F78500014589D71797FF1F03472C
:10A1A00097269797FF1F9387A7250DC3D84F584B26
:10A1B00011CF37E70400384F9047854517C5FF1F7B
:10A1C000034545C2029713458400E1BD97F0FFFFA8
:10A1D000E780407FCDBF5C4D411106C688C317C7DD
:10A1E000FF1F232FF7BEB7E7040083A70708170553
:10A1F00000001305C5DF8297B24097C7FF1F238376
:10A20000A7BE01454101828001113335A000A3079B
:10A21000A100B7E7040083A7471706CE1306F10095
:10A220008545130550308297F24005618280828017
:10A23000411122C406C697A7FF1F83C7F700054434
:10A2400089EF97B7FF1F83C76740014499E717A4B9
:10A25000FF1F034464FF134414002285970000008D
:10A26000E780C0FA178501001305055309E4178537
:10A270000100130565532244B240410117630100F8
:10A280006700838C797122D4A30F010037E40400A6
:10A290008327841726D24AD006D6AA842E8913058E
:10A2A00050309305F10132C6829732468347F1015F
:10A2B00093150601C18185CB01452EC6970000008C
:10A2C000E780C0F483274417B2454A8626858297E3
:10A2D000054597000000E78060F3B2502254925485
:10A2E000025945618280832744174A8626858297D2
:10A2F000EDB741119397050122C406C626C2C18756
:10A300002E8463D40702B7E40400FC541795FF1FA2
:10A3100003450512829719C1BC5482972165218D8E
:10A32000B240224492444101828093F715008DC7C8
:10A33000B7E7040083A7471A1796FF1F1306460EB8
:10A3400097C5FF1F9385C5AA1795FF1F0345450EA7
:10A35000829713451400E9B793F725000145E9D327
:10A3600097C7FF1F83C747AA85E7B7E7040003A87D
:10A37000871A1307401F9797FF1F83C7670B8146F4
:10A3800013064006994517C5FF1F035565A7029898
:10A390001345240071B797C7FF1F83D767A663983B
:10A3A000A70217C7FF1F231EB7A417C7FF1F231B32
:10A3B000C7A417C7FF1F2318D7A42E86178501002F
:10A3C00013050545BE85175301006700E377178520
:10A3D000010013056545176301006700C38E03572D
:10A3E000450097C7FF1F83D7A7A16318F702C1676E
:10A3F000F91717C7FF1F2325F7A097C7FF1F23A330
:10A4000007A097C7FF1F238B079E97C7FF1F238DAA
:10A41000079E170300006700E3E11785010013059D
:10A42000A540176301006700038A7D15954763E225
:10A43000A71C178701001307A7340A053A951C418A
:10A44000011122CC06CEBA972E848287178501008F
:10A450001305053E97600100E780E086A1A203C7CF
:10A46000250099476311F7022E8597000000E780C9
:10A4700040F783456400178501001305653C97503C
:10A480000100E780606C97A7FF1F238F07DA17850D
:10A4900001001305A53C7DBF03C72500954763193F
:10A4A000F702C16717C7FF1F03578795F91703D531
:10A4B000A5006309F702B7E7040083A7C7178297CF
:10A4C000178501001305853A97500100E780A07FAA
:10A4D000854717A7FF1F2309F7D617850100130526
:10A4E000653B8DBF97C7FF1F239CA79083D7E500CF
:10A4F00097C6FF1F2397F69083D7050197C6FF1FC6
:10A500002392F69083D7250197C6FF1F239DF68ED1
:10A5100097C7FF1F2384078E631BE502B7E704007C
:10A52000BC4F09661306069089451795FF1F034522
:10A5300025F082970356E4008355A4001785010097
:10A540001305053497500100E780006051B7930769
:10A55000700F2316F100B7E7040083A7870D179645
:10A56000FF1F0346E6EC6C0082974DF9854717C73D
:10A57000FF1F2305F7885DB71785010013054532D6
:10A58000D1BD83C5250091476392F502178501006F
:10A590001305853297500100E780E07297000000B4
:10A5A000E78040C9F2406244056182809947639226
:10A5B000F502228597000000E780A0E28345640051
:10A5C000178501001305C52797500100E780C05784
:10A5D000D1BF9547639AF50083471400E1F31785CF
:10A5E00001001305A52FBDB5178501001305852FA3
:10A5F000E1BF82803757315F9797FF1F938787E4CA
:10A60000130777D598C39356C50017870100130722
:10A61000E71CBA9683C5060093568500BD8ABA9694
:10A6200003C6060093564500BD8A3D89BA962A970F
:10A6300083C6060003470700238407002383D7004F
:10A64000A383E7002382B700A382C7009797FF1F69
:10A65000938747E02383B700A383C7002384D700F1
:10A66000A384E7008280411106C697000000E780BE
:10A67000A0F8B7E7040083A787141796FF1F1306F7
:10A6800066DCD54501458297B2404D469795FF1F40
:10A69000938545DC13057030410117030000670006
:10A6A000A3BE61712324811A37E4040083270408C0
:10A6B0002326111A2322911A2320211B232E31191C
:10A6C00017050000130525C382971799FF1F13096B
:10A6D00029D6994785442300A900231CF1009785BA
:10A6E00001009385A50E9307400617750100130519
:10A6F000A5A5231CF1082308910097B9FF1F938992
:10A70000490597500100E780204483D5090017854B
:10A7100001001305A50A97500100E780E042294592
:10A7200097500100E780204703D5090097000000FB
:10A73000E78080EC832744171008854513055030C7
:10A740008297832744171796FF1F1306A6D0CD457F
:10A75000130570308297832744171796FF1F13063F
:10A7600066CDB545130560308297832744173008BE
:10A77000894513051031829783274417300989458D
:10A78000130520318297832744159305000A0D4550
:10A790008297832744159305000A11458297A305E4
:10A7A00091002306910002CD23080100230C010033
:10A7B00083278416300991451305704082978327BB
:10A7C00084161306B1008545130500408297832740
:10A7D00084167000854513051040829783278416E0
:10A7E000300885451305204082978327841610087A
:10A7F0008545130550408297832704157D55829720
:10A80000832744137D5582977D559790FFFFE780FE
:10A81000C0E78327440C82979790FFFFE78020C30F
:10A82000832784141796FF1F1306C6C1D54501451B
:10A83000829789471306700F814528092306F10086
:10A840009780FFFFE780A08C8D47130600088145A5
:10A850002808230CF1089780FFFFE780408B914781
:10A86000230CF100976701009387877F984383C784
:10A8700047003AC8230AF10097C0FFFFE780E0EDE8
:10A880007000854505459790FFFFE78020E7300978
:10A890009305700F09459790FFFFE78020E6300889
:10A8A000930500080D459790FFFFE78020E510080D
:10A8B000954511459790FFFFE78040E4C16717B7C2
:10A8C000FF1F1307E753F9171CC32322070017952F
:10A8D000FF1F1305A5B59790FFFFE78000E18327D1
:10A8E000C41D17B5FF1F1305255082973C4803452B
:10A8F0000900854582978320C11A0324811A832485
:10A90000411A0329011A8329C1195D618280C16737
:10A9100017B8FF1F0358C84EF9176301F8083DCD5B
:10A92000B5CD011126CAB7E4040083A7841222CC56
:10A930002E862315B10006CE2A8401478146ED45B7
:10A94000428582972AC611ED17850100130545EA55
:10A9500097500100E7802037F2406244D2440561FD
:10A960008280FC440356A100A28582972C0017B573
:10A97000FF1F0355E5489790FFFFE780C0E369DDBF
:10A9800017850100130505E897500100E780A03303
:10A9900083A7C412ED45280082977DBF82800DC534
:10A9A00085471797FF1FA30CF7A89797FF1F2389C9
:10A9B00007A835469795FF1F9385C5A713056030F7
:10A9C000170300006700438C9797FF1FA38907A612
:10A9D000E9BF97B7FF1F83C72743A9EFC16717B721
:10A9E000FF1F0357E741F9176306F7044111854735
:10A9F00022C417B7FF1F2309F74037E404007C4C3B
:10AA000006C689451795FF1F034585A28297032334
:10AA1000841A2244B2409797FF1F83C767A117B5D6
:10AA2000FF1F0355E53D1307401F814631469945F9
:10AA30004101028382806D7123248110232611102D
:10AA400023229110328401CD8947630AF5028320C5
:10AA5000C110032481108324411051618280178525
:10AA600001001305E5E8AE8497500100E780A025BA
:10AA7000A285268597A0FFFFE780E04EC9BFB7E714
:10AA80000400FC472800829717850100130505E79D
:10AA900097500100E78020238347810039C41307C2
:10AAA000000B6380E7021387A7051377F70F8D4626
:10AAB00063EDE602A285280097B0FFFFE780E04A39
:10AAC00079B78547E3F587F883459100177501004D
:10AAD0001305859AB335B0009797FF1F2386B75C9F
:10AAE00097500100E78040069DB703479100A207F9
:10AAF000B966D98F1387E6556384E70C636DF70455
:10AB00002D671307B755638FE708636AF700296756
:10AB10001307A755638FE708A2852800A1BF3167F7
:10AB20001307C7556388E70635671307D755E395BD
:10AB3000E7FE8947E3FD87F097000000E780A0E982
:10AB40009305E4FFC205C1811305A1009780FFFFB3
:10AB5000E7800069EDBD3D671306F7556389C706B9
:10AB6000636DF6009386E665E398D7FAA285280020
:10AB700097C0FFFFE780C082D9BD9306F766638D5B
:10AB8000D7041307F777E399E7F897C0FFFFE7804B
:10AB900060AE75BD0146A285280097B0FFFFE78033
:10ABA000606875B5A285280097B0FFFFE7808073C5
:10ABB00079BDA285280097B0FFFFE780607441BD92
:10ABC000A285280097B0FFFFE780807449B597C041
:10ABD000FFFFE7800086A5BD97C0FFFFE780A08B41
:10ABE000BDB5C16717B5FF1F03558521F917630769
:10ABF000F500B7E7040003A3C7170283828017F3A9
:10AC0000FFFF670023631773FFFFE702A34B2A844C
:10AC100008452E89B28919C900C19715000093858E
:10AC2000A586610597300100E780200581447D5AA3
:10AC300097100000E780E03963C7A40481449710AF
:10AC40000000E780003A63C8A40497B7FF1F93870A
:10AC5000E71B9C43DC47B307F94091872302F400CC
:10AC6000638309048327C900B307F4409587A302CF
:10AC7000F4001C4C89C79C4799C32285829717739F
:10AC8000FFFF670063475C44139714008504BA977D
:10AC90002390470171BF1C48139714008504BA978D
:10ACA0002390070069BF832789000547B307F44055
:10ACB0009587A302F40083570400638EE7028DC3D7
:10ACC00009476384E7040D47E395E7FA9787010096
:10ACD000938787151CCC978701009387E71511A8E8
:10ACE000978701009387C7DB1CCC97870100938768
:10ACF00027DC5CC8BDBF97870100938767C71CCC62
:10AD0000978701009387C7C7EDB79787010093879F
:10AD100067161CCC978701009387C716D9BF95E5A6
:10AD20001773FFFFE702A33B0046184483479400D4
:10AD300075839D8B6317F70097100000E78060B460
:10AD400048C41773FFFF6700C33B82801773FFFF80
:10AD5000E702433713893500C16442094111AA89CA
:10AD60000144F11413590901054A2EC69710000039
:10AD7000E7802026B2456348A400014541011773CE
:10AD8000FFFF6700633783A7090013171400BA9702
:10AD900083D707006388B7006394970063742A0120
:10ADA0000504E1B70545D9BF1773FFFFE702A330DC
:10ADB000AA892E89328BB6843A8ABE8A97A000006F
:10ADC000E780C0FE71C9268597200000E780C00C8F
:10ADD0008D4763E7A7007D551773FFFF6700233199
:10ADE00083DB440097100000E780A0242A8497109A
:10ADF0000000E78040259307740031443305850245
:10AE000063CDA70297100000E780A02297100000F2
:10AE1000E78020222A8497100000E780C022930751
:10AE2000740031443305850263C3A7049710000002
:10AE3000E78020209307450029A897100000E780AD
:10AE40008020330585021307F0179307C017E35FCF
:10AE5000A7FA2D55E3C277F963040B02D686528612
:10AE6000A6854A8597200100E780C0BDB5B7971039
:10AE70000000E780401D330585029307C5FFD1BF61
:10AE8000832749001385C90083D527009700000058
:10AE9000E78000EC61F581B769553DBF97B7FF1FAB
:10AEA0002398A7F697B7FF1F938747F690438147EC
:10AEB0000C463307F500420741836393B700828055
:10AEC0005446139847008507C2962390E600D5B7ED
:10AED00097B7FF1F938787F39C4303C58700828042
:10AEE00017B5FF1F0355C5F282801773FFFFE702F6
:10AEF000031FC1671387D7FF630BE502636AA700CF
:10AF0000F1176300F50201451773FFFF6700631F28
:10AF10001387E7FF6302E502FD171D8D133515004A
:10AF2000E5B797500000E780602A7D15C5BF9750B0
:10AF30000000E780E0FED5BF97500000E78000FDED
:10AF4000EDB71773FFFFE70283194111AA8401448B
:10AF50002EC697100000E780C008B2456348A400E1
:10AF6000014541011773FFFF6700A3199C481315A2
:10AF700014003E9583570500E385B7FE0504C9BF5D
:10AF800003485500814693F7F60F63E507018147B3
:10AF90003E858280584593975600BA9703D727007D
:10AFA0006316B70003D70700E304C7FE8506E1BFB9
:10AFB0008346450001479377F70F63E4D700814745
:10AFC00011A81C45131657000507B29703D60700B2
:10AFD000E313B6FE3E8582801773FFFFE702830E00
:10AFE00093170501C18797BAFF1F938A2AE2635B13
:10AFF000F00883A70A00C0479C4703570400198D37
:10B00000420541816368F500014422851773FFFF03
:10B010006700830E12052A94CDBFDC4713944900C4
:10B02000014A3E94834744006341FA02014A834740
:10B0300054006349FA028509C20993D9090183A71B
:10B040000A009847E3EBE9FCC1B71C4413195A0006
:10B05000A6853E994A8597000000E780C0EE05E18D
:10B06000050AC9B75C4413195A00A6853E994A855A
:10B0700097000000E78020ED19E1050A4DBFE30CC1
:10B0800009FA61B7AA8481495DBF1773FFFFE70220
:10B0900003051C452A8481E79307C5001CC51C4491
:10B0A000231204001CC09307F00F63EDB70093F563
:10B0B000F50F228597200000E780C0E51773FFFF9A
:10B0C0006700230493940501C167C18063F9F5000B
:10B0D000A685228597200000E780E0E8C5B7C181FA
:10B0E00093F5F50F228597200000E780A0E2A68562
:10B0F000228597200000E780E0E3C9B797B7FF1FDC
:10B100009387C7D0884382801C4599C797B7FF1F94
:10B1100023AEA7CE014582807D55828097B7FF1F61
:10B120009387C7CE984383474500484792073E958B
:10B1300082801773FFFFE70283FA617100451C18D4
:10B140003EC6B70780013EC81C183ECA835744005C
:10B1500002CE02D002CC231EF100834784002A894C
:10B1600002D22301F1023C083ED402D6970000002F
:10B17000E78000FB835705002316F102975000007B
:10B18000E78000C82307A1025C4003556400F183F7
:10B1900013F717008347F10252055181F99BD98FAC
:10B1A000A307F10297100100E780207939CDAA8426
:10B1B0000355050097A00000E78020C083D7040056
:10B1C0002AD26800231CF10083D72400231DF1003C
:10B1D0001C4803D647008C4397200000E780A0D08E
:10B1E0008347B400CA86177601001306E6718117FB
:10B1F000A305F4006C00481097200100E7808084CC
:10B200005D611773FFFF6700C3EF2155D5BF1C4574
:10B21000B1CF03C5A700894613576500630BD7025A
:10B220008D46630ED70285466300D702130740069A
:10B230003305E50203C7B700418B15CB83C7B700C1
:10B24000BD8B3355F54082801375F5031307803E9F
:10B25000C5B709671375F50313070771D1BF372702
:10B2600009001375F5031307077CD9B701458280E0
:10B270001773FFFFE702A3E603A98500630C090427
:10B280008347B900AE8493F7070E85C30345990041
:10B29000930520030D810505B305B50288446105BA
:10B2A00097300100E78080AD35A02E859700000023
:10B2B000E78020F62A8419CD97000000E780605CC3
:10B2C0008325C900B307B54063FA87002E94B30500
:10B2D000A440E9F51773FFFF6700A3E285457DBF32
:10B2E0001773FFFFE702A3DF2A8403D505000111CE
:10B2F00032C636C43AC22EC002CA02CC02CE97A0D1
:10B300000000E78080AB82452ACA22852ECC9700B8
:10B310000000E780E0E003570500231EE10097509E
:10B320000000E780E0ADA24632469247230FA1001D
:10B3300036874C08B2862285014697000000E780D8
:10B34000E0A605611773FFFF6700A3DB1773FFFF1C
:10B35000E702E3D861711C183EC6B70780013EC8FA
:10B360001C183ECA3C0800453ED4AA8402CC02CE3A
:10B3700002D002D202D697000000E78060DA83573D
:10B38000050035592316F10297500000E78040A7C9
:10B390002307A10209C48357440081EB21594A8540
:10B3A0005D611773FFFF6700C3D503556400520545
:10B3B000518197100100E78040582A8965D1834761
:10B3C000B40093F7070E99C7130584019730010065
:10B3D000E780009D83574400231EF10083478400CB
:10B3E0002301F1025C4003550900D98313F70708D4
:10B3F00083471102231CA10093F7F707D98FA300FD
:10B40000F10283572900231DF1005C40F18313F7FB
:10B4100017008347F102F99BD98FA307F10297A088
:10B420000000E78080992AD235D9834794006800CC
:10B43000139757008347B400FD8BD98FA305F40001
:10B440001C4803D647008C4397200000E780A0A942
:10B45000A687177701001307274B740005464C1089
:10B46000268597000000E78060942A890DD98347DC
:10B47000B400A685FD8BA305F40097000000E780CB
:10B4800060DF31BF1773FFFFE70263C5832485FECA
:10B490002A844111268597000000E78080D78347E2
:10B4A00034FF93F7070E8DCB2AC626859700000040
:10B4B000E78060C809CD834734FFB245FD8BA309FF
:10B4C000F4FE91C5228597300100E780208B410171
:10B4D0001773FFFF6700E3C27DD98327C4FF26856A
:10B4E000829775F5834734FF93F7070E91C722853E
:10B4F00097300100E780C08A032584FE9700000092
:10B50000E78000E5E9B71773FFFFE70243BA9C4104
:10B5100041112A8903C7070089472E849356670083
:10B520006380F6040D466388C6049307F00763043E
:10B53000F7022E8597200000E78060ABAA8481493E
:10B54000C16B130C490097B7FF1F9387278C9C434F
:10B55000984763E4E90441011773FFFF6700E3B80C
:10B5600003D745008547E3F8E7FE2E8597200000C6
:10B57000E78040ADE1B703D74500E3FEE7FC2E8549
:10B5800097200000E780A0A6AA84228597200000CB
:10B59000E78000A8C204C98C5DB7DC470355A90049
:10B5A000139A49003E9A93170501C187635DF00025
:10B5B00083570A006397A70263E774038327CA00CF
:10B5C000034D5A002DA0A1672167A98F1307F7EF3C
:10B5D000E374F7FE6397090097000000E78020916D
:10B5E00061FD85098DB783278A00034D4A00835D7D
:10B5F000A90003576900216A138BC7003AC6814A24
:10B6000033CA4D01631E5D0197B7FF1F9387878083
:10B610009C43E1DBA2866286814526858297D1B76D
:10B62000A1679387F7EF930C4BFF63F24703B24593
:10B630005A8597F0FFFFE780A0710DC103278B00AB
:10B64000104709CE10436382C4023107D5BFEE858F
:10B65000668597000000E780008F71F993861A00D5
:10B6600093FAF60F130B0B0271BF835644005C4331
:10B67000E3E9F6F622853AC697200000E7802081AC
:10B68000A1679387D7042A8A035D4400324763E8A1
:10B6900097008347D90093E707F8A306F9001C47F2
:10B6A00066852286E2858297C1670844FD17337A52
:10B6B000FA00529508C02312A40125B797A7FF1FCF
:10B6C0009387C7749843814715C31447814763FF25
:10B6D000D500939745004C47BE9519C903C755003F
:10B6E00081476375E600DC451606B2973E85828089
:10B6F00003C745008147E37BE6FE16069C45F5B788
:10B700001773FFFFE702039CAA892E8A814497AA38
:10B71000FF1F938AAA6F83A70A00984763E6E40095
:10B720001773FFFF6700439DDC47139444000149F2
:10B730003E9413BB140083474400634BF900014956
:10B7400013BB140083475400634FF9008504E1B72D
:10B750000844931759005287DA860146A2853E9520
:10B7600082990509C9BF4844931759005287DA8660
:10B770000546A2853E9582990509E9B71773FFFF33
:10B78000E702E395814517F5FFFF1305054897A7E5
:10B79000FF1F239F076697000000E780A0F617733E
:10B7A000FFFF6700039697A7FF1F938727669C43B9
:10B7B00095C31773FFFFE7028392814517F5FFFFDB
:10B7C0001305A54497000000E780C0F31773FFFF3F
:10B7D0006700239382801773FFFFE702A38E37E48D
:10B7E00004008327841241112315E100AE893289B8
:10B7F000368A3A8681460147ED45AA8482972AC651
:10B8000021C90356A100D28597400100E780602836
:10B810008327C413CE8526858297058905C983278A
:10B82000440D2314210101462C00268582972A8489
:10B8300001C9B7E7040083A7C712ED452800829726
:10B84000228541011773FFFF6700038B4944D5B779
:10B850006554FDB75C41FD175CC182801773FFFF23
:10B86000E702E387B7E70400FC5F8297954733055B
:10B87000F50281450D811773FFFF670083881773F9
:10B88000FFFFE702C385B7E70400FC5F8297954797
:10B890003305F5020D811773FFFF67008386177369
:10B8A000FFFFE702C383B7E7040083A7870B0355B5
:10B8B000050082971773FFFF6700A3841773FFFFCC
:10B8C000E702E381035505003287AE861786FF1F26
:10B8D000035666BE97A5FF1F938505549700000089
:10B8E000E780A0EF1773FFFF6700A3811763FFFFD7
:10B8F000E702E37EB7E7040083A7C71782971773B1
:10B90000FFFF670003801763FFFFE702437DB7E790
:10B91000040083A7871397A5FF1F9385E54F8297A0
:10B9200001451763FFFF6700C37D1763FFFFE70251
:10B93000037BB7E7040083A7C71F81451785FF1F57
:10B94000035565B382971763FFFF6700837B176317
:10B95000FFFFE702C378B7E7040083A7871397A523
:10B96000FF1F9385654C829701451763FFFF6700B2
:10B9700043791763FFFFE7028376B7E7040083A7E5
:10B98000C71F81451785FF1F0355E5B482971763CD
:10B99000FFFF670003771763FFFFE70243742E85FD
:10B9A00097800000E78080B397800000E78080F0F8
:10B9B0001763FFFF6700E3741763FFFFE70223725B
:10B9C00097800000E78080FA1763FFFF67006373CA
:10B9D0005C49E1175CC95CC583572501A1072319A0
:10B9E000F50083570501A1072318F5008280F14770
:10B9F0003305F50297A7FF1F938707459C433E95A4
:10BA000082808D476315F60803D74600854763F0AB
:10BA1000E7081763FFFFE702836C368536842E89BB
:10BA200097100000E780A05C29C983574400931455
:10BA30000501C18063E39704228597100000E78029
:10BA4000005BFD14231294009307A0026300F5022B
:10BA50009307B0026307F50293079002631FF50096
:10BA6000228597000100E780608901A80146CA8508
:10BA7000228597A00000E78000B41763FFFF6700EE
:10BA80004368228597100000E7806007FDB7828039
:10BA900097A6FF1F9386863B9C42014599CF98430A
:10BAA000D44217A6FF1F2323E63A6396D70097A632
:10BAB000FF1F23AFE6381385C7FE82801763FFFFA1
:10BAC000E702E36197000000E780A04B7144330573
:10BAD0008502914597900000E780C0EC11E565551F
:10BAE0001763FFFF6700E36197A7FF1F23ACA7342D
:10BAF00097000000E780E048330585029145979064
:10BB00000000E78020EA61DD97A7FF1F23AEA73280
:10BB100097000000E780E04697A7FF1F239EA7300D
:10BB200097000000E780E04597A7FF1F2397A73005
:10BB300097770100938787E217A7FF1F2322F7302B
:10BB400097070000938707E917A7FF1F2328F72E01
:10BB5000014579B71763FFFFE7026358AA8517A568
:10BB6000FF1F1305652D97100000E780605F1763C6
:10BB7000FFFF670003591763FFFFE7024356970073
:10BB80000000E78060FD97100000E780E05E97A767
:10BB9000FF1F9387A72B9C4391CF1387C7FE19CB19
:10BBA00083D5C7FF17A5FF1F1305C52A97200100DE
:10BBB000E780C01C1763FFFF6700A3541763FFFFF4
:10BBC000E702E35197000000E780C0EC09CD83470E
:10BBD00085002A8493F7070499EB0355E500970045
:10BBE0000000E78080F91763FFFF670083518347F8
:10BBF000C5009304450117A9FF1F1309292585E3F3
:10BC0000832709005CC997A7FF1F23A197248327D7
:10BC10004900F1FB97A7FF1F23AC9722E9B7FD1757
:10BC20002306F500610597800000E78060DA83074E
:10BC3000840063CB07048347840093E707F8230459
:10BC4000F400B7E704009C5F82974205A947418151
:10BC50003375F5028347840093F707FCC98F2304EB
:10BC6000F4008347D4003E951C402318A40089CFDC
:10BC7000984319CB8347C40050408145850733055D
:10BC8000F502420541810297832709005CC897A706
:10BC9000FF1F23AD971A8327490089E797A7FF1F46
:10BCA00023A8971A8347C4009DDF8355040117A575
:10BCB000FF1F1305251A97200100E780200C25B7E8
:10BCC0001763FFFFE702A34197A7FF1F9387C73DB5
:10BCD0009C4701448583858B85E3AE84B2853A8693
:10BCE00097100000E780204F2A8419C597100000A4
:10BCF000E7806045829408CC22851763FFFF6700C8
:10BD000043401763FFFFE702E33B41112E8932C630
:10BD1000AA8997000000E780C03132471306050268
:10BD2000CA86970500009385C5CC17A5FF1F13058C
:10BD3000A51097000000E780E0F82A8425C9930445
:10BD4000C50097000000E780E0411946AA852685D6
:10BD500097100000E7802019854526859710000080
:10BD6000E780001517750100130505BD4E95834545
:10BD70000500268597100000E780C0195C48314611
:10BD80008145A1075CC85CC483572401E1172319CE
:10BD9000F40083570401E1172318F4001C4C3E857E
:10BDA0009760FFFFE780A036A304250122854101AB
:10BDB0001763FFFF670043341763FFFFE702233277
:10BDC0004111AA842EC632C497100000E780003AC1
:10BDD000004DB2452246834784000CC050C093F703
:10BDE000F70393E707042304F400231804002685CF
:10BDF00097100000E780203583479400A946231759
:10BE0000A40013D7370005073307D7029D8B85079A
:10BE10002306F400A306E40083C70401D84885077D
:10BE2000230FF7FE17A7FF1F130747025843232AC4
:10BE300004009307440129E317A7FF1F232AF700F3
:10BE400017A7FF1F2324F70017A4FF1F1304840064
:10BE5000228597200100E780A0E41C44858B5D8D3E
:10BE600019E58145228597200100E78020F14101F5
:10BE70001763FFFF6700E3281CC317A7FF1F2329D1
:10BE8000F7FCD9B71763FFFFE702632597050000AA
:10BE9000938565B7014597000000E78000B0014534
:10BEA0001763FFFF6700E3251763FFFFE702232304
:10BEB00097000000E78080B01763FFFF67006324EE
:10BEC0008347C500A5E31763FFFFE70243212A84E8
:10BED0000355E50097000000E78000C821C18347B3
:10BEE000840093F7F7FB2304F4001C4091C7DC4364
:10BEF00081C74C400145829797000000E78080B9D8
:10BF000017A5FF1F130505F597200100E78040E9FD
:10BF10000355E40097000000E78020C61763FFFF89
:10BF20006700231E82801763FFFFE702431B97A76A
:10BF3000FF1F9387A7F197050000938565C817A594
:10BF4000FF1F130525F123A0070023A20700972058
:10BF50000100E78080D21763FFFF6700831A1C4D42
:10BF600091CFDC4381CF1763FFFFE702431783457F
:10BF7000070082971763FFFF6700A318828097A7C7
:10BF8000FF1F938767EF9C4303C50700828097A735
:10BF9000FF1F938767EE9C4303C51700828097A716
:10BFA000FF1F938767ED9C4303C52700828097A7F7
:10BFB000FF1F938767EC9C4303C54700828097A7C8
:10BFC000FF1F938767EB9C4303C53700828097A7C9
:10BFD000FF1F938767EA9C4303C55700828097A79A
:10BFE000FF1F938767E99C4303C56700828097A77B
:10BFF000FF1F938767E89C4303C57700828097A75C
:10C00000FF1F938767E79C4303C58700828097A73C
:10C01000FF1F938767E69C4303C59700828097A71D
:10C02000FF1F938767E59C4303C5A700828097A7FE
:10C03000FF1F938767E49C4303C5B70011E11D45CB
:10C04000828097A7FF1F938727E39C4303C5C70000
:10C05000828097A7FF1F938727E29C4303C5D700E1
:10C06000828097A7FF1F938727E19C4303C5E700C2
:10C07000828097A7FF1F938727E09C4303D5070182
:10C08000828097A7FF1F938727DF9C4303C5270163
:10C09000828097A7FF1F938727DE9C4303D5470124
:10C0A000828097A7FF1F938727DD9C4303D56701F5
:10C0B000828097A7FF1F938727DC9C4303D58701C6
:10C0C000828097A7FF1F938727DB9C4303C5A701A7
:10C0D000828097A7FF1F938727DA9C4303C5B70188
:10C0E000828097A7FF1F938727D99C4303C5C70169
:10C0F000828097A7FF1F938727D89C4303C5D7014A
:10C10000828097A7FF1F938727D79C4388578280F9
:10C1100097A7FF1F938747D69C4303D5C70282800A
:10C1200097A7FF1F938747D59C4303D5E70219E1E3
:10C130001305800C828097A7FF1F9387E7D39C434A
:10C1400003C50703828097A7FF1F9387E7D29C430D
:10C15000C85B828097A7FF1F938787D1884382801F
:10C1600097A7FF1F938707D18843828019E17D55E8
:10C170008280F5DE984265DFFDD917A7FF1F130700
:10C18000A7F21847AA877155058B631D072403C5BD
:10C1900007001547E37DA7FC03C737001305F0052B
:10C1A0007D171377F70FE364E5FC03C35700E30043
:10C1B00003FC83C86700E38C08FA03C7770049458E
:10C1C00079171377F70FE364E5FA03C7A70011485F
:10C1D0001305F7FF1375F50FE36BA8F803CE97006F
:10C1E0000D481305FEFF1375F50FE362A8F803C8A9
:10C1F000B7006309080065181378F80F1305600D80
:10C20000E36705F703C5C700794879151375F50F7E
:10C21000E36FA8F403C8D7000D457D181378F80F15
:10C22000E36705F503D80701930E4017511842083C
:10C2300013580801E3ED0EF303C8E7007D181378E7
:10C24000F80FE36605F303C827017D181378F80F8C
:10C25000E36F05F103C88700C54E75181378F80F12
:10C26000E3E70EF103D86701856E938EBEE06D188B
:10C27000420813580801E3EC0EEF03D847016D188C
:10C28000420813580801E3E40EEF03D88701791838
:10C29000420813580801E36C05ED03C8A7017D1897
:10C2A0001378F80FE36505ED03C5B7011D487D154B
:10C2B0001375F50FE36DA8EA03C5D7017148791529
:10C2C0001375F50FE365A8EA03D5E7011308E00F3E
:10C2D0007D1542054181E36CA8E803C50702494882
:10C2E00079151375F50FE364A8E8C85301C937C879
:10C2F00034005915130858BFE36BA8E603A887025A
:10C3000037C53400130555BF5918E36205E717A573
:10C31000FF1F2321C5B603C6050117A5FF1F232D47
:10C32000F5B40545E375C5E403D82501D049337656
:10C330000603E31E06E203C61501E30A06E217A69A
:10C34000FF1F2327B6B283C5270001466387A500D8
:10C3500003C61700F1453306B60283C707039305EA
:10C36000C00272971A071307C70516031A97960893
:10C370004697B387B70241553E97329742074183AC
:10C380006362E8061763FFFFE70263D5368597808F
:10C390000000E780406C97000100E780C04B2A84D2
:10C3A00097A00000E780205E2A9497F00000E780C5
:10C3B000002A2A9497900000E78040852A9497F0FD
:10C3C000FFFFE780E06F2A9497400000E780009726
:10C3D0002A9497700000E78040A022951763FFFF22
:10C3E000670023D282801763FFFFE70243CF41112A
:10C3F000A307A10097A00000E78040C99305F100C2
:10C40000170500001305E5B597F0FFFFE780802FC3
:10C41000014541011763FFFF6700A3CE1763FFFFCC
:10C42000E70263C917A4FF1F130404C8032884008C
:10C4300079599368180097A4FF1F23AB14C713788A
:10C44000180063100802BA84BE89368B328A2E899E
:10C45000AA8A97F0FFFFE780E0A77D15269519E5EA
:10C4600031594A851763FFFF670063C897F0FFFFE4
:10C47000E78040A67D152695A167E353F5FE97A7B3
:10C48000FF1F938727F998433E8C814B01CB0145D1
:10C4900097F00000E780C047933B15004A85DA8695
:10C4A0005686D28597900000E78060512A8911CD89
:10C4B0001C44F99B17A7FF1F232CF7BE83270C00F2
:10C4C000CDD3E3800BFA829769BF268597A7FF1F1C
:10C4D00023AE07BC97F0FFFFE780809C4146CE85E6
:10C4E00017A5FF1F1305C5C597300100E780605AE7
:10C4F00097D00000E780E09C0325040B97D0000054
:10C50000E780A0A0054597D00000E780A0A70545DB
:10C5100097000000E78060EDA9B797A7FF1F9387FA
:10C52000A7B89C47858BEDC71763FFFFE70223BBC6
:10C5300017A5FF1F130505BF97A7FF1F23A607B663
:10C5400097A7FF1F23A407B697A7FF1F23A207B62D
:10C5500097200100E780C08497500000E78080F9B1
:10C5600097100100E780405097100100E780405687
:10C5700097A7FF1F9387C7B19C4391C70545978035
:10C580000000E780E02397A7FF1F9387279A9C432B
:10C5900099C741657D1597700000E780E0A597F089
:10C5A0000000E780804197D00000E780209397A7A4
:10C5B000FF1F938727C49C431397170163560700F7
:10C5C00097F00000E780A0B097A7FF1F23AA07B647
:10C5D00097A7FF1F23A807B697A7FF1F23A607B695
:10C5E00097A7FF1F23A407B697000000E780008CE1
:10C5F00097000000E780A07597F0FFFFE7804018E4
:10C6000097F00000E780E0D91763FFFF670063AF92
:10C61000828097A7FF1F938727A98843828097A7C7
:10C62000FF1F938767A8C8438280B7E7B00093874E
:10C63000075063E1A70297A7FF1F9387E7A6D84398
:10C64000FD576367E50097A7FF1F23A1A7A68147B2
:10C650003E858280B957EDBF1763FFFFE70223A82D
:10C6600097800000E780607597800000E780C077C2
:10C670001763FFFF6700E3A81763FFFFE70283A4C8
:10C680002A849304140201112E85B289A6852146BD
:10C6900036C63A8997300100E780403D0DE9B24641
:10C6A00038082686CE851305940497500000E7804D
:10C6B000604121462C084A8597300100E780003B05
:10C6C0001335150005611763FFFF6700E3A20145FD
:10C6D000D5BF1763FFFFE70283A0930545061795B3
:10C6E000FF1F1305A57997100100E78020691763E4
:10C6F000FFFF670003A11763FFFFE702439E41119D
:10C700002EC697F0FFFFE780C017B24588C14101F0
:10C710001763FFFF6700E39E1763FFFFE702839A3B
:10C72000AA842E8497800000E780006CAA89854542
:10C73000228597000000E780E07D83C7E40113892C
:10C74000940899E313890403CE852285970000009D
:10C75000E780407C2146930519022285970000005E
:10C76000E780607897A7FF1F938707948C43228503
:10C7700097100000E780C0822146938584022285BD
:10C7800097000000E78020761763FFFF6700C396DD
:10C790001763FFFFE7022392397197F00000E780EB
:10C7A000E0B49305400661E997800000E7800060EF
:10C7B000630205149797FF1F83C7076E13B717000F
:10C7C0009796FF1F238AE66C014499CFC16417A98D
:10C7D000FF1F1309698D9309400EFD149700000097
:10C7E000E78020836342A40A97F0FFFFE780600997
:10C7F0004169B7290900096AFD7A2A8B81447D19AC
:10C800009389F97B130A0A71938A8AC797000000FB
:10C81000E780208063D7A4041304400EB38784020A
:10C8200017A7FF1F130747880324070B3E9483575E
:10C83000C4016382270B18403307EB4063EAE90029
:10C84000834744008507B3874703D6976365F70896
:10C8500001468145094597F0FFFFE780C04AAA8B52
:10C8600029E597400000E780808385476317F50638
:10C870008965938505711795FF1F1305256097102E
:10C880000100E780A04F95A0B30734030327090BED
:10C89000BA9703D7C7016308970003C75700A3825D
:10C8A00007002382E700050415BF9305C500228514
:10C8B00097000000E78080E65E852286976501008C
:10C8C0009385C50897F0FFFFE780404F5E8597107E
:10C8D0000000E780608A850415BF9797FF1F938744
:10C8E000A77C9C478D83858BC1F721611753FFFF80
:10C8F0006700E37F01468545094502D002D202D494
:10C9000002D697F0FFFFE7800040AA8479DD97F018
:10C910000000E780E09C1389C4002A8481454A8591
:10C9200097000000E780005F0C4041464A85970071
:10C930000000E780405B832944006385090C4E8535
:10C9400002D802DA02DC02DE97300100E780E0382C
:10C950002ACE141005462C0808184ECC975000001B
:10C96000E780E00A1375F50F51ED8355840093E5D8
:10C9700025004A8597000000E780E05E11460C1014
:10C980004A8597000000E780005601469765010040
:10C99000938545FC268597F0FFFFE780204226859A
:10C9A00097000000E780407D5C40A1D301468545AB
:10C9B0000D4597F0FFFFE7800035AA841DD548405C
:10C9C0001389C40097300100E78020312AC64A85C8
:10C9D00097000000E780404C3246636FC5004C4032
:10C9E0004A8597000000E780005001468145268572
:10C9F00097F0FFFFE780803C268597000000E780E6
:10CA0000A077E5B583558400ADB71753FFFFE70264
:10CA1000036D9797FF1F938727699C471DC193E775
:10CA200087001795FF1F130565451797FF1F2321E3
:10CA3000F76897100100E78040321753FFFF670047
:10CA4000436CDD9B1797FF1F2324F7669730000088
:10CA5000E780E0647DF11795FF1F130525429710CD
:10CA60000100E780E033D1BF1753FFFFE702A36463
:10CA70004169AA892E8AB28A368BBA8B8144179C67
:10CA8000FF1F130C6C62930C400E7D1997F0FFFF93
:10CA9000E780205863C4A40001443DA0338494037C
:10CAA00083270C0B3E948357C401638627055A875E
:10CAB000D6865286CE851305040397000000E780D2
:10CAC000E0BB01C923800B0022851753FFFF6700DD
:10CAD00003628347F40185C35A87D6865286CE8582
:10CAE0001305940897000000E78040B909C5854701
:10CAF0002380FB00D1BF850451BF8357450063806D
:10CB0000071E1753FFFFE702E35B01112A8497001A
:10CB10000000E780C04D09C985476309F506056136
:10CB20001753FFFF6700435D97E00000E780007C3C
:10CB30007DF5835744004947ED9BE392E7FEC145ED
:10CB4000228597000000E7804033AA842285970061
:10CB50000000E780204F0357440002CE91472A8906
:10CB6000631AF700228597000000E780A0513C0877
:10CB70002ACC3ECE97E00000E78080765C55C5D396
:10CB800074084A86A6850545829751BF035744001D
:10CB9000D147E3F6E7F8032A0400C1690149979AEF
:10CBA000FF1F938A6A50130B400EFD1997F0FFFF89
:10CBB000E7802046634FA90E2285032A04009700D0
:10CBC0000000E780C042A1452A8922859700000025
:10CBD000E780A02AAA84228597000000E780804A87
:10CBE00014402A86AA8978082685CA8597000000FD
:10CBF000E780C0E7AA8405D503C7F4018947631518
:10CC0000F7008347C10181DF5546D2851385640053
:10CC100097300100E780E0E7014597800000E7805A
:10CC2000C01901C583D7C401A5E79797FF1F938754
:10CC3000A7479C4793551900858913D73700058B63
:10CC400001CF8983858B6399B70001452EC6970074
:10CC50000000E780C0DBB2454E8597800000E7808A
:10CC6000601F0346C1012A84937519002685979099
:10CC70000000E780E03935C1268597800000E78015
:10CC8000E018268511C0014597800000E780004C20
:10CC900097300000E780A0408547E312F5E883C79E
:10CCA00054001307F00FE38CE7E68507A382F40036
:10CCB000BDB5B304690383A70A0BBE9483D7C4012F
:10CCC000638B37015546D285138564009730010088
:10CCD000E780C0D955DD0509D1BD5DD86DB782802B
:10CCE0001753FFFFE702033E97800000E780000C28
:10CCF00005C1C16401441799FF1F1309E93A93095B
:10CD0000400EFD1497F0FFFFE780A030634EA400B3
:10CD10001795FF1F1305851697100100E780E003A4
:10CD20001753FFFF6700433D330534038327090B87
:10CD30003E958357C50163889700231205009780AD
:10CD40000000E780A00C050475BF9797FF1F93872D
:10CD5000A7359C478D83858B8DE31753FFFFE70233
:10CD600003381795FF1F1305651197100100E78021
:10CD700020031753FFFF6700C33882801753FFFF5C
:10CD8000E702E335970500009385C5A01795FF1FBF
:10CD90001305C50E97100100E78020EE1753FFFF23
:10CDA000670023361753FFFFE70263338841B7E775
:10CDB0000400BC5B050542054181829709C5854792
:10CDC0002300F50005051753FFFF6700833383C772
:10CDD000F5FF2E858507A38FF5FE828083C7F5FFBB
:10CDE000FD1793F7F70FA38FF5FE99EF1753FFFF8A
:10CDF000E702E32EB7E70400BC571385F5FF8297DF
:10CE00001753FFFF6700E32F82801C410357450043
:10CE10008D8FBA951CC12312B5003E85828093D7B1
:10CE20008500A2051441DD8D835745001387E6FF79
:10CE300018C189072312F50013D685004111238FED
:10CE4000B6FEA38FC6FE4101828018419307F7FF0B
:10CE50001CC18357450085072312F500A30FB7FEB9
:10CE60008280835745008D8F2312F5001C41BE95AB
:10CE70000CC12E858280AA8703D7470008410D8FF9
:10CE8000AA952392E7008CC3828018410845330598
:10CE9000A740828083574500035765001D8F1C41C2
:10CEA00008453385A7403305A74082801753FFFF0D
:10CEB000E702E32241112EC62A8497000000E78092
:10CEC000A0FDB2456373B50001A08357440008403C
:10CED000BE952312B4003E9541011753FFFF670032
:10CEE00043221753FFFFE702831F41112E84B285AF
:10CEF00032C697000000E780A0FB3246A28597303B
:10CF00000100E78000B941011753FFFF6700631F6D
:10CF10001753FFFFE702A31C2E84854597000000EE
:10CF2000E78000F9230085001753FFFF6700631DAA
:10CF30001753FFFFE702A31A41112317B1008945D8
:10CF400097000000E780C0F68347E1002300F5006A
:10CF50008347F100A300F50041011753FFFF67006D
:10CF6000431A1753FFFFE702831793D78500A205E3
:10CF70004111DD8D2317B100894597000000E7803E
:10CF800020F38347E1002300F5008347F100A3006D
:10CF9000F50041011753FFFF6700A3161753FFFF6A
:10CFA000E702E3131397850193D78501C166938642
:10CFB00006F0D98F13D78500758FD98FA205370753
:10CFC000FF00F98D4111DD8D2EC6914597000000BF
:10CFD000E78000EE6C00114697300100E78060ABFF
:10CFE00041011753FFFF6700C3111753FFFFE7020B
:10CFF000030F1C41854503C4070097000000E7802C
:10D0000080E622851753FFFF6700A30F1753FFFF2A
:10D01000E702E30C1C414111894503C7070083C7A0
:10D0200017002307E100A307F10097000000E78045
:10D0300080E30355E10041011753FFFF6700630CD4
:10D040001753FFFFE702A3091C414111894503C79C
:10D05000070083C717002307E100A307F10097002B
:10D060000000E78040E08357E100410113D58700CD
:10D07000A2075D8D420541811753FFFF67006308DA
:10D080001753FFFFE702A3050C4141112A84114603
:10D09000680097300100E780C09F91452285970086
:10D0A0000000E78040DCB247C166938606F0139724
:10D0B000870113D58701598D13D78700758F598D37
:10D0C000A2073707FF00F98F5D8D41011753FFFF5E
:10D0D000670023031C45BE950CC18280AE87944334
:10D0E00091E6584101EF0CC15CC1828003C7570033
:10D0F00013671700A382E700B687D5B70CC3EDB757
:10D10000AA87084119CD1841D44398C36313D500A9
:10D11000D8C32A87034657009376160081E623205A
:10D1200007008280944381CA8C4203A847008CC3C5
:10D1300063930601CCC3799A14C3A302C700368750
:10D14000D1BF1C45DC471D8DB777DBB6938777DBF6
:10D1500009853305F502420541818280F147B38597
:10D16000F50248452E9582808347450085072302B6
:10D17000F50082801753FFFFE70263F62A8409E473
:10D180001753FFFF6700E3F783474400F5DBFD1704
:10D1900093F7F70F2302F400E5F71C4403D72700A9
:10D1A00005072391E700DC4399C3228582974C4809
:10D1B00089CD83475400898B99E71C4422859C477D
:10D1C0009C439C478297232A0400004023200400AC
:10D1D0007DB71753FFFFE70283F083572500411106
:10D1E0002EC681EB0144228541011753FFFF6700E2
:10D1F00043F1035705008147F146E305F7FEB38588
:10D20000D702404585072E948345440008C4F5F5B0
:10D21000B247AA8481E7232A040009A81C456C00B0
:10D2200022859C439C43829748C84DDD8547231245
:10D23000F400B24723200400231804002319F4004B
:10D240005C485CC483D72400FD172391F40061BFC0
:10D250001753FFFFE702A3E89797FF1F938707C4C1
:10D26000884323260500232405004105971001006B
:10D27000E78000B31753FFFF6700A3E81753FFFFD2
:10D28000E702E3E51794FF1F130444C11C4041115A
:10D2900099CF9C472300B5002AC65CC197000000C7
:10D2A000E78040FB1C40DC4399C332458297410133
:10D2B0001753FFFF6700E3E40347450029E3584D98
:10D2C000AA877D551DCF1753FFFFE70243E11CC31B
:10D2D000DC479796FF1F23A3E6BCF1561305070111
:10D2E0002390D70097050000938505029710010051
:10D2F000E780A09801451753FFFF670083E07D5545
:10D30000828082801753FFFFE70263DD01116146CF
:10D31000814528009750FFFFE78060DF9797FF1F48
:10D320009387C7B79C4328009305F00FDC473EC6A0
:10D3300097000000E780C0F405611753FFFF670006
:10D3400043DC9797FF1F938767B59C43D847A16736
:10D350009387C702631EF70A397106DE22DC26DADC
:10D3600080004AD84ED652D456D23285B284970025
:10D370000000E780C0C7AA89268597000000E780E3
:10D3800020C92318A4FC268597000000E78040C828
:10D390002319A4FC268597000000E78060C783D787
:10D3A00044000A8A231AA4FC858393F7F70F230EFF
:10D3B000F4FC8607BD0793F7073F3301F1408A8AE3
:10D3C00001498347C4FD6367F902CE85130584FCD8
:10D3D000232C54FD97000000E78080EA528113015E
:10D3E00004FCF2506254D2544259B259225A925A11
:10D3F00021618280268597000000E78060C1931735
:10D400001900D69705092390A7001379F90F55BF86
:10D4100082809797FF1F938767A89C43D847A1678F
:10D420009387A702631AF70A397106DE22DC26DA2F
:10D4300080004AD84ED652D456D23285B284970054
:10D440000000E780C0BAAA89268597000000E7801F
:10D4500020BCFD572318A4FC26852319F4FC970053
:10D460000000E780E0BA83D744000A8A231AA4FCAC
:10D47000858393F7F70F230EF4FC8607BD0793F718
:10D48000073F3301F1408A8A01498347C4FD63673E
:10D49000F902CE85130584FC232C54FD970000006F
:10D4A000E78000DE5281130104FCF2506254D25432
:10D4B0004259B259225A925A216182802685970098
:10D4C0000000E780E0B493171900D6970509239070
:10D4D000A7001379F90F55BF82809797FF1F938795
:10D4E000E79B9C43D847A16789076310F70A397106
:10D4F00006DE22DC26DA80004AD84ED652D456D236
:10D500003285328997000000E78060AEAA894A859B
:10D5100097000000E780C0AF835749000A8A2318AC
:10D52000A4FC858393F7F70F230CF4FC8607BD0753
:10D5300093F7073F3301F1408A8A8144834784FD92
:10D5400063E7F402CE85130584FC232A54FD97007B
:10D550000000E780E0D25281130104FCF2506254D3
:10D56000D2544259B259225A925A216182804A8534
:10D5700097000000E780C0A993971400D697850410
:10D580002390A70093F4F40F55BF82809797FF1F55
:10D590009387C7909C43D847A1679387E704631E8E
:10D5A000F70A397106DE22DC26DA80004AD84ED628
:10D5B00052D456D23285B28497000000E78020A36F
:10D5C000AA89268597000000E78080A42318A4FC80
:10D5D000268597000000E780A0A3231AA4FC2685D7
:10D5E00097000000E780C0A283D744000A8A23196D
:10D5F000A4FC858393F7F70F230EF4FC8607BD0781
:10D6000093F7073F3301F1408A8A01498347C4FDFC
:10D610006367F902CE85130584FC232C54FD970023
:10D620000000E780E0C55281130104FCF25062540F
:10D63000D2544259B259225A925A21618280268587
:10D6400097000000E780C09C93171900D697050942
:10D650002390A7001379F90F55BF82809797FF1F7A
:10D660009387C7839C43D847A1679387C704631AEE
:10D67000F70A397106DE22DC26DA80004AD84ED657
:10D6800052D456D23285B28497000000E7802096AB
:10D69000AA89268597000000E7808097FD57231808
:10D6A000A4FC2685231AF4FC97000000E78040962E
:10D6B00083D744000A8A2319A4FC858393F7F70FC4
:10D6C000230EF4FC8607BD0793F7073F3301F140B3
:10D6D0008A8A01498347C4FD6367F902CE85130531
:10D6E00084FC232C54FD97000000E78060B9528130
:10D6F000130104FCF2506254D2544259B259225AD6
:10D70000925A21618280268597000000E780409030
:10D7100093171900D69705092390A7001379F90FDD
:10D7200055BF82809787FF1F938747779C43D847D1
:10D73000A167DD076317F7041753FFFFE702239A7A
:10D7400079713285328497000000E780408A2AC6CA
:10D75000228597000000E780A08B2311A10222857B
:10D7600097000000E780A088B2452300A1022808A6
:10D7700097000000E780C0B045611753FFFF6700C6
:10D78000439882809787FF1F938747719C43D847B0
:10D79000A167938787046317F7041753FFFFE70216
:10D7A000039479713285328497000000E7802084E9
:10D7B0002AC6228597000000E78080852311A102F8
:10D7C000228597000000E7808082B2452300A102F5
:10D7D000280897000000E780A0AA45611753FFFFC3
:10D7E0006700239282809787FF1F9387276B9C4354
:10D7F000D847A1679387A7046312F7021753FFFF67
:10D80000E702E38D01112800814597000000E780C1
:10D8100020A705611753FFFF6700A38E82809787BB
:10D82000FF1F9387A7679C43D847A1679387570239
:10D830006319F7021753FFFFE702638A011132856C
:10D8400097F0FFFFE780A07A2308A1008145280018
:10D8500097000000E780C0A205611753FFFF670033
:10D86000438A82809787FF1F938747639C43D847EB
:10D87000A1679387E702631BF7041753FFFFE702D3
:10D88000038601113285328497F0FFFFE7804078EC
:10D89000AA84228597F0FFFFE7808077854709E912
:10D8A000228597F0FFFFE78080744205B337A00020
:10D8B00028008145231891003ECA97000000E780A8
:10D8C000209C05611753FFFF6700A3838280978721
:10D8D000FF1F9387A75C9C43D84799476313F708BA
:10D8E0001743FFFFE702A37F79713285328497F0F7
:10D8F000FFFFE780C06F2AC6228597F0FFFFE78011
:10D9000020712310A102228597F0FFFFE780206E8F
:10D910002301A102228597F0FFFFE780406DA3015C
:10D92000A102228597F0FFFFE780606C2302A1022D
:10D93000228597F0FFFFE780806B2313A1022285E9
:10D9400097F0FFFFE780A06AB2452314A1022808E0
:10D9500097000000E780C09245611743FFFF670012
:10D96000437A82809787FF1F938747539C43D8470A
:10D97000A1679387C7036313F7081743FFFFE70205
:10D98000037679713285328497F0FFFFE780206655
:10D990002AC6228597F0FFFFE78080672310A10247
:10D9A000228597F0FFFFE780A0662311A102228560
:10D9B00097F0FFFFE780A0632302A102228597F082
:10D9C000FFFFE780C062A302A102228597F0FFFF5C
:10D9D000E780E0612303A102228597F0FFFFE78043
:10D9E0000061B245A303A102280897000000E78068
:10D9F000208945611743FFFF6700A37082801743AA
:10DA0000FFFFE702C36D01112A8497F0FFFFE78053
:10DA1000005EAA84228597F0FFFFE780605F228581
:10DA200097F0FFFFE780C05E035744008D4763F720
:10DA3000E700228597F0FFFFE780805D228597F061
:10DA4000FFFFE780E05C2800A68597000000E780E4
:10DA5000208305611743FFFF6700A36A9787FF1FB5
:10DA60009387C7439C43D847A167FD07631FF7000F
:10DA70001743FFFFE702A366328597000000E780A7
:10DA800040F81743FFFF6700C36782809787FF1F37
:10DA90009387C7409C43D847A167E5076315F708FC
:10DAA0001743FFFFE702A36379713285328497F051
:10DAB000FFFFE780C0532AC6228597F0FFFFE7806B
:10DAC0002055228597F0FFFFE78080542310A102A4
:10DAD000228597F0FFFFE780A05352055181231163
:10DAE000A10222852302010297F0FFFFE780205068
:10DAF000A302A102228597F0FFFFE780404F230396
:10DB0000A102228597F0FFFFE780604EB245A30394
:10DB1000A102280897F0FFFFE78080764561174350
:10DB2000FFFF6700035E82809787FF1F9387073799
:10DB30009C43D847A1679387E703631FF700174308
:10DB4000FFFFE702C359328597000000E78060EBD2
:10DB50001743FFFF6700E35A82809787FF1F938771
:10DB6000E7339C43D847A16793874704631EF702B6
:10DB70001743FFFFE702A35679713285328497F08D
:10DB8000FFFFE780C0462AC6228597F0FFFFE780A7
:10DB90002048B245280897F0FFFFE780606E456196
:10DBA0001743FFFF6700E35582809787FF1F938726
:10DBB000E72E9C43D847A167938787026310F70439
:10DBC0001743FFFFE702A35179713285328497F042
:10DBD000FFFFE780C0412AC6228597F0FFFFE7805C
:10DBE0000041B2452300A102280897F0FFFFE7801B
:10DBF000206945611743FFFF6700A35082801743E8
:10DC0000FFFFE702C34D011197F0FFFFE780203EC1
:10DC1000AA85280097F0FFFFE7808066056117431B
:10DC2000FFFF6700034E9787FF1F938727279C43BB
:10DC3000D847A167D107631FF7001743FFFFE7022B
:10DC4000034A328597000000E780A0FB1743FFFFDF
:10DC50006700234B82809787FF1F938727249C436D
:10DC6000D847A167C507631FF7001743FFFFE70207
:10DC70000347328597000000E780A0F81743FFFFB5
:10DC80006700234882809787FF1F938727219C4343
:10DC9000D847A167B907631FF7001743FFFFE702E3
:10DCA0000344328597000000E780A0F51743FFFF8B
:10DCB0006700234582809787FF1F9387271E9C4319
:10DCC000D847A167AD07631FF7001743FFFFE702BF
:10DCD0000341328597000000E780A0F21743FFFF61
:10DCE0006700234282809787FF1F9387271B9C43EF
:10DCF000D84789476318F7021743FFFFE702233E1F
:10DD00000111328532C897F0FFFFE780402EAA85C7
:10DD1000280097F0FFFFE780A05605611743FFFF3B
:10DD20006700233E82809787FF1F938727179C43B6
:10DD3000D847A1678D076311F7041743FFFFE70278
:10DD4000033A01113285328497F0FFFFE780202AE1
:10DD500013066100AA844C00228597300000E780FA
:10DD6000C0232800A68597F0FFFFE780605105617A
:10DD70001743FFFF6700E33882809787FF1F938771
:10DD800027129C4381CFDC4391CB1743FFFFE7026F
:10DD9000033582971743FFFF6700A336828017433E
:10DDA000FFFFE702C33379713C08AE843ED2A16520
:10DDB000B7070A002A843ED448103C08DD053ED649
:10DDC00036C432C63AC297D0FFFFE780402C1247D4
:10DDD0004810BA8597F0FFFFE780C013324648101D
:10DDE000B28597F0FFFFE780E014A2464810B685A1
:10DDF00097F0FFFFE7800012501001478146A6858B
:10DE0000228597D0FFFFE780E04D45611743FFFF74
:10DE10006700232F1743FFFFE702632C01117C00EB
:10DE20000329C501AE843ECAA165B70707002A844D
:10DE30003ECC48087C00C5053ECE97D0FFFFE7806A
:10DE400000258345D900480897F0FFFFE780800C44
:10DE5000500801478146A685228597D0FFFFE780BD
:10DE6000604805611743FFFF6700A3291743FFFFC1
:10DE7000E702E32683C7950093F7F707A384F5002D
:10DE800097000000E78040F91743FFFF6700632712
:10DE90001743FFFFE702A32479713C08AE843ED20A
:10DEA000A165B70709002A843ED448103C08938531
:10DEB00045043ED632C636C497D0FFFFE780201D0A
:10DEC000A2464810B68597F0FFFFE780A0043246CF
:10DED0004810B28597F0FFFFE780C005501001475A
:10DEE0008146A685228597D0FFFFE780A03F456148
:10DEF0001743FFFF6700E3201743FFFFE702231EDE
:10DF000083C7950041112A8493F7F707A384F5008E
:10DF100032852EC697F0FFFFE780800F85672AC401
:10DF20006370F50297700000E78020E92246B24551
:10DF300009ED11478146228597000000E78060E6E1
:10DF400041011743FFFF6700C31B01478346F501EB
:10DF5000DDB71743FFFFE702E31601113C003ECA9D
:10DF6000B7070A003ECC3C003ECE83C79500AA8985
:10DF7000328593F7F707A384F5002E8497F0FFFF0F
:10DF8000E78000098567637DF504A165AA84938510
:10DF90008504480897D0FFFFE780600F26859770BB
:10DFA0000000E78080E12A8929E19145480897F03F
:10DFB000FFFFE78020F6A685480897F0FFFFE7807F
:10DFC00060F7CA85480897F0FFFFE780A0F4014793
:10DFD00081465008A2854E8597D0FFFFE7808030AC
:10DFE00005611743FFFF670023118145480897F03B
:10DFF000FFFFE78020F20349090275BF1743FFFFC7
:10E00000E702430C79711C103ECAB7070F003ECCE3
:10E01000404D1C10AA84AE894808994532C63689FD
:10E020003ECE97D0FFFFE780800632464808B28593
:10E0300097F0FFFFE78000EE630C0902A545480852
:10E0400097F0FFFFE780C0E62546CA8597200100CC
:10E05000E78020A4500801478146CE85268597D0C9
:10E06000FFFFE780202845611743FFFF6700C308D3
:10E070008355C402480897F0FFFFE780A0EB0355E3
:10E08000E402814505C5854785456301F502C16701
:10E09000FD179305F00F630BF5007D1597700000D9
:10E0A000E780208E9305150093F5F50F480897F04B
:10E0B000FFFFE78020E683450403480897F0FFFF51
:10E0C000E78040E583451403480897F0FFFFE780A9
:10E0D00060E483552403480897F0FFFFE78080E55C
:10E0E00083554403480897F0FFFFE780A0E49DB7FD
:10E0F0001743FFFFE702A3FE83C795008146014651
:10E1000093F7F707A384F50097000000E78040EF3E
:10E110001743FFFF6700E3FE1743FFFFE70223FCFF
:10E1200079713E841C103ECA2E89B7070F00A16585
:10E130003ECCFD051C10AA84480842C03AC23ECE1F
:10E1400036C432C697D0FFFFE78060F432464808F5
:10E15000B28597F0FFFFE780E0DBA2464808B6856E
:10E1600097F0FFFFE78000DD12474808BA8597F077
:10E17000FFFFE78020DC0248630C08029145480855
:10E1800097F0FFFFE780C0D21146A28597200100DB
:10E19000E7802090500801478146CA85268597D0A0
:10E1A000FFFFE780201445611743FFFF670063F519
:10E1B0008945480897F0FFFFE78080CF8347040038
:10E1C0002300F50083471400A300F500E1B71743CF
:10E1D000FFFFE70223EF83C7950001112A8A93F717
:10E1E000F707A384F5003285AE8432C697F0FFFFAF
:10E1F000E78000E232462A89328597F0FFFFE78008
:10E2000000DF85676373F902AA894A859770000069
:10E21000E780A0BA2A8419ED114781464A86A6856F
:10E22000528597000000E780C0B705611743FFFFE4
:10E23000670083EC9387E9FF93F7F70F0547E366E1
:10E24000F7FE8347F50195EB8947E380F9FE8346A6
:10E25000F401528501474A86A68597000000E780B1
:10E2600040B4A167D90748083ECC230A010002CE7A
:10E2700097000000E780A0B04DBF639EE70089478C
:10E28000639EF90093071020231FF500977000008C
:10E29000E780C0B76DBF0947E39BE7FA8D47E39876
:10E2A000F9FA228597700000E78080DF9787FF1FCB
:10E2B000938707DE9C4399E79787FF1F938707C7DC
:10E2C0009C4399C703D5040097800000E780A0CE47
:10E2D000231F040022855DBF1743FFFFE70223E0F1
:10E2E00001113C003ECAB7070B003ECC3C003ECEBD
:10E2F00083C795002A89328593F7F707A384F50031
:10E30000AE8497F0FFFFE780A0D093170501C18787
:10E31000635AF006A1652A849385E502480897D0E0
:10E32000FFFFE780C0D6A285480897F0FFFFE7808F
:10E3300060C09787FF1F938767BF9C43A9EB014489
:10E340009375F40F480897F0FFFFE780A0BC935542
:10E35000844093F5F50F480897F0FFFFE78080BBF6
:10E360009355044193F5F50F480897F0FFFFE780B8
:10E3700060BA014781465008A6854A8597D0FFFFBD
:10E38000E78040F605611743FFFF670083D74165CB
:10E3900085460546A2857D1597500000E78060BD43
:10E3A00059DD510597000100E780808F1304400676
:10E3B0003344850271B71743FFFFE70243D20111CF
:10E3C000B70706003EC683C7950021642A8993F7E4
:10E3D000F707A384F500AE8428009305A4040AC4BB
:10E3E0000AC897D0FFFFE78080CA30000147814606
:10E3F000A6854A8597D0FFFFE780C0EE97E0FFFF34
:10E40000E780E01113049404480822CC230A010099
:10E4100002CE97000000E780809605611743FFFF5A
:10E42000670023CE1743FFFFE702C3C9C1642A89EF
:10E4300001449789FF1F938929C7130A8002FD149D
:10E4400097E0FFFFE780E0BD6347A4000145174365
:10E45000FFFF670063CAB307440303A7C90ABA975B
:10E4600003D707006306970083D72700638427013B
:10E470000504F9B70545E1BF1743FFFFE70283C471
:10E480002A8A2E8999C123A0050081498144978A4F
:10E49000FF1F938A2AA1614B97E0FFFFE780A0BE90
:10E4A00063C7A4004E851743FFFF6700E3C43384AE
:10E4B000640383A70A003E948357040099E763042A
:10E4C0000900232089008504C1BF4146D285130578
:10E4D000440097100100E780605975F5A289E5B7FF
:10E4E0001743FFFFE70203BE39717C083ED4B7072C
:10E4F0000A003ED67C083ED883C795002A8A32851A
:10E5000093F7F707A384F5002E8932C697F0FFFF33
:10E51000E78000B085676373F5083246AA843285C8
:10E5200097F0FFFFE780A0AC8547AA8963E8A706BC
:10E53000A16593858504281097D0FFFFE78020B55B
:10E54000268597700000E78040872A8429ED914551
:10E55000281097F0FFFFE780E09BA685281097F032
:10E56000FFFFE780209DCE85281097F0FFFFE78012
:10E57000609A014781463010CA85528597D0FFFFC7
:10E58000E78040D6A1679387770448183EDC230ACA
:10E59000010202DE97F0FFFFE780607E21611743F2
:10E5A000FFFF670063B58145281097F0FFFFE78004
:10E5B0006096A685281097F0FFFFE780A0979787C1
:10E5C000FF1F9387E7E49C4381CB22856389090081
:10E5D00097D00000E78040248345040271B797D0AC
:10E5E0000000E780C022CDBF1743FFFFE70283ADE5
:10E5F00083C795004111AA8993F7F707A384F50013
:10E600003285AE84328A97F0FFFFE78060A085678D
:10E61000637FF5022A8997600000E780007A2A84E8
:10E62000914631C58347F50105476387E70291C7E6
:10E630000D476366F704AD461DA893050503032542
:10E640000A00414697100100E78040420DE9410170
:10E650001743FFFF670043AA9305950803250A00A7
:10E66000414697100100E7806040814669F54A867F
:10E67000A6854E8597000000E780C081C9BF83252D
:10E680000A001305940897700000E780A02919C1BB
:10E69000C146F1BF9787FF1F9387879F9C4399E7E8
:10E6A0009787FF1F938787889C4399C72285978008
:10E6B0000000E780208A69FD8547A30FF4002285CA
:10E6C00097B00000E7806084228597600000E780B3
:10E6D000E0734E8581464A86A68597F0FFFFE78066
:10E6E000607BA1679387570448003EC42302010062
:10E6F00002C697F0FFFFE780806891BF1743FFFFD6
:10E70000E702639B83C795004111AA8993F7F70736
:10E71000A384F50032852E89B28A97F0FFFFE78047
:10E72000208F85676374F50EAA8497600000E780E8
:10E73000C0682A840DED416B014A978BFF1F938BB4
:10E74000AB96130C400E7D1B19A833048A0383A7D4
:10E750000B0B3E948357C40163836705050A97E05A
:10E76000FFFFE780008BE342AAFE95460DA083578A
:10E77000C501639697029305050303A50A00414668
:10E7800097100100E780802E994611E18146268688
:10E79000CA854E8597F0FFFFE780C06F85A883A5E7
:10E7A0000A001305040397700000E780A017C14614
:10E7B00079FD2285231E940097A00000E780E07475
:10E7C000228597600000E78060649787FF1F93872A
:10E7D00027C49C43A9C323000402228597D00000CC
:10E7E000E78040F04E8581462686CA8597F0FFFF78
:10E7F000E780406AA1679387070448003EC423026C
:10E80000010002C697F0FFFFE78060574101174300
:10E81000FFFF6700C38D89472300F402E1B7397118
:10E8200006DE22DC4AD8800052D456D25AD026DAEC
:10E830004ED65ECE2E8A32892A8B97D0FFFFE78094
:10E84000407A0605710541998A8A3301A140232245
:10E8500024FC231404FC97D0FFFFE78080788347D3
:10E860009A000605350593F7F7072315A4FCA304C2
:10E87000FA004A85232624FC97E0FFFFE7804079D1
:10E8800093170501C1876340F0025681130104FC10
:10E89000F2506254D2544259B259225A925A025BEF
:10E8A000F24B21618280AA844A8597E0FFFFE780CE
:10E8B0002076AA894A8597E0FFFFE7806075A16509
:10E8C0009385C5022A89130544FC97C0FFFFE780A2
:10E8D000007C268597C0FFFFE7804070854511C901
:10E8E0004A86CE8597C0FFFFE780C069AA8B21E9E1
:10E8F0008945130544FC97E0FFFFE780A061A685EA
:10E90000130544FC97E0FFFFE780C062CE85130546
:10E9100044FC97E0FFFFE780E061CA85130544FCF3
:10E9200097E0FFFFE780006101478146130644FC42
:10E93000D2855A8597D0FFFFE780C09AB9B7814545
:10E94000130544FC97E0FFFFE780C05CA685130534
:10E9500044FC97E0FFFFE780E05DCE85130544FCB3
:10E9600097E0FFFFE780005DCA85130544FC97E050
:10E97000FFFFE780205C814497D0FFFFE78060665F
:10E98000E3D4A4FA83A70B0113971400BA9783D595
:10E99000070099C5130544FC97E0FFFFE780805905
:10E9A0008504D9BF797106D622D44AD000184ECE3C
:10E9B00052CC56CA26D25AC8AE893289AA8A97D072
:10E9C000FFFFE78000620605690541990A8A330165
:10E9D000A140232A24FC231C04FC97D0FFFFE780DE
:10E9E000406083C7990006052D0593F7F707231D9F
:10E9F000A4FCA384F9004A85232E24FC97E0FFFFA2
:10EA0000E780006193170501C187634FF0005281D1
:10EA1000130104FDB250225492540259F249624A41
:10EA2000D24A424B45618280AA844A8597E0FFFF23
:10EA3000E780005EA1659385A5022A89130544FD40
:10EA400097C0FFFFE780A064268597C0FFFFE7809F
:10EA5000E058854509C9CA8597C0FFFFE780805502
:10EA60002A8B29E18945130544FD97E0FFFFE780E4
:10EA7000604AA685130544FD97E0FFFFE780804BC1
:10EA8000CA85130544FD97E0FFFFE780A04A0147D0
:10EA90008146130644FDCE85568597D0FFFFE7805B
:10EAA0006084B5B78145130544FD97E0FFFFE7801B
:10EAB0006046A685130544FD97E0FFFFE780804789
:10EAC000CA85130544FD97E0FFFFE780A046814417
:10EAD00097D0FFFFE780E050E3DBA4FA83270B0128
:10EAE00013971400BA9783D5070099C5130544FD01
:10EAF00097E0FFFFE78000448504D9BF1733FFFF8D
:10EB0000E702E35D83474500404DD5EFFD575DC407
:10EB10008346940009476363D70A0346B4008546D9
:10EB200063EEC6088306E40063CA06085C45F9562E
:10EB30002390D7009777FF1F83C7073799E3A30474
:10EB4000E4009777FF1F9387673E9C4381E78947DF
:10EB5000A306F4009787FF1F9387878B9C4381E769
:10EB600089472306F4009705000093854506AA848B
:10EB70001305040197F00000E7802010FD57231AC9
:10EB8000F40281471CDC01489777FF1F23AA8730D6
:10EB90009777FF1F93870731232E040304C0804318
:10EBA00097D0FFFFE780204E61463306C5028145BE
:10EBB00022859730FFFFE780805581473E851733D8
:10EBC000FFFF67000354FD57D5BF1733FFFFE70270
:10EBD00003512A840355450297600000E780E01D39
:10EBE00019E5231E04001733FFFF67008351835785
:10EBF000E401F5DB930504FF174501001305450FFC
:10EC000097E00000E780E014F9BF1733FFFFE70249
:10EC1000034D2E89A16541119385E5032A8436C4ED
:10EC200032C6BE843AC297C0FFFFE7804046124713
:10EC30002285BA8597E0FFFFE780C02D3246228506
:10EC4000B28597E0FFFFE780E02EA2462285B685D9
:10EC500097E0FFFFE780002E6303090291452285BC
:10EC600097E0FFFFE780C0241146A68597100100BA
:10EC7000E78020E241011733FFFF670083488945A1
:10EC8000228597E0FFFFE780A02283C704002300CE
:10EC9000F50083C71400A300F500E9BF1733FFFF99
:10ECA000E702E34383C79500444D054793F7F70711
:10ECB000A384F5001C42411183C707006367F70670
:10ECC0002E842A89B1C003C7D400630FF7021777D7
:10ECD000FF1F1307A725184305C3A386F40097A0B9
:10ECE0000000E780404A83C7D40099E741657D155D
:10ECF00097400000E780403083D72403918B89C779
:10ED000097E00000E780C0134A85A28597F0FFFFD7
:10ED1000E7808010A167C10748003EC423020100BC
:10ED200002C697F0FFFFE780800541011733FFFF20
:10ED30006700233D1733FFFFE702633A03D745001F
:10ED40008D47AA8441112E8432892E8563E3E70220
:10ED500097E0FFFFE780C02BAA85230009002685E6
:10ED600097C0FFFFE780002541011733FFFF6700D1
:10ED7000433997E0FFFFE780A0292AC6228597E064
:10ED8000FFFFE780E028B24585472A862300F90087
:10ED9000268597C0FFFFE780E01EF9B7397106DED0
:10EDA00022DC26DA80004ED652D456D24AD85AD027
:10EDB0005ECEAE89B284AA8A97D0FFFFE780602139
:10EDC00006051305250241990A8A3301A140232231
:10EDD00024FC231404FC97D0FFFFE780801F83C727
:10EDE000990006054D0593F7F7072315A4FCA384A6
:10EDF000F9002685232624FC97E0FFFFE7804021C9
:10EE000093170501C1876340F0025281130104FC8E
:10EE1000F2506254D2544259B259225A925A025B69
:10EE2000F24B21618280AA8B03AB040097C0FFFFE5
:10EE3000E780C01A51E583D7440001498544F117A2
:10EE400093B71700A301F4FC834734FCA165C9C73D
:10EE50009385E504130544FC97C0FFFFE78020235A
:10EE6000A685130544FC97E0FFFFE780A00ADE8536
:10EE7000130544FC97E0FFFFE780C00B834734FC99
:10EE8000114691E30946DA85130544FC97E0FFFF3C
:10EE9000E78060058144630A0900416B7D1B97D0C0
:10EEA000FFFFE780001363CCA402014781461306ED
:10EEB00044FCCE85568597C0FFFFE780A042B1B7DE
:10EEC000A685130634FC97000000E780E0E6933443
:10EED00015002A8986048DBF9385C504A5BF8327A5
:10EEE000C90013971400BA9783D50700638865019A
:10EEF000130544FC97E0FFFFE780C003850445B796
:10EF00001733FFFFE702231B79711C103EC4B707BC
:10EF10000F003EC61C103EC883C79500AA8A3285E2
:10EF200093F7F707A384F500AE89328497E0FFFFDB
:10EF3000E780000E93170501C187635AF0062A8AFD
:10EF4000228597E0FFFFE780A00C2A895285032BDA
:10EF5000040097C0FFFFE780600839ED8357440045
:10EF600081440544F11793B71700A303F1008345CB
:10EF70007100DA872287CA8652862800970000002F
:10EF8000E780E0C8014781463000CE85568597C0AE
:10EF9000FFFFE7802035A1679387D70348083ECC61
:10EFA000230A810026CE97F0FFFFE78040DD456110
:10EFB0001733FFFF6700A313A285130671009700A4
:10EFC0000000E78060D7AA84094455D13544E300A6
:10EFD00055FB4A8597F0FFFFE78000450D4441D976
:10EFE000014497D0FFFFE780C0FE634DA400C16BD2
:10EFF0000144FD1B97D0FFFFE780A0FD634EA400F6
:10F000001544B5B7DC4413171400BA9783D707002B
:10F01000638327030504F1B7D84493171400BA9704
:10F0200003D70700631B770123902701268597A04C
:10F030000000E78080DB01441DBF050465BF173376
:10F04000FFFFE702230883C7950041112A8A93F73F
:10F05000F707A384F50032852E89328497E0FFFFFD
:10F06000E78000FB93170501C1876353F006AA8967
:10F07000228597E0FFFFE780A0F92311A1004E85CC
:10F08000832A040097C0FFFFE78040F539E58357E6
:10F09000440085440144F11793B71700A300F10021
:10F0A0000348110003572100D6875285CE86268655
:10F0B000CA8597F0FFFFE7806006A167F107480067
:10F0C0003EC42302910022C697F0FFFFE78020CBC9
:10F0D00041011733FFFF67002302A28513061100C9
:10F0E00097000000E78040C52A84894455D983579A
:10F0F000210011678544BA97C2071167C1831307BE
:10F10000F7EFE36FF7F89777FF1F938767F89C4354
:10F1100081CB85451305210097500000E7802075BD
:10F12000835521002285814497C0FFFFE780A0E13D
:10F1300025D923100500228597A00000E78040CD47
:10F1400085B71733FFFFE70203F783C79500411127
:10F150002A8B93F7F707A384F50032852E8A328431
:10F1600097E0FFFFE780C0EA93170501C18763516D
:10F17000F006AA8A228597E0FFFFE78060E92A89E6
:10F180005685832B040097C0FFFFE78020E531E51B
:10F190008357440081440544F11793B71700A30136
:10F1A000F10003483100DE875A854A87D6862286D9
:10F1B000D28597F0FFFFE78060F6A167ED07480072
:10F1C0003EC42302810026C697F0FFFFE78020BBE4
:10F1D00041011733FFFF670083F1A2851306310059
:10F1E00097000000E78040B5AA8409445DD9916783
:10F1F000CA97C2071167C1831307F7EF0544E3629B
:10F20000F7FACA8597C0FFFFE780E0D3014451F9C0
:10F21000814997D0FFFFE780C0DC63DBA9009848F5
:10F2200093971900BA9703D7070005EF239027019A
:10F2300097D0FFFFE780E0DA1544E384A9F626853E
:10F2400097A00000E780C0BC9777FF1F938747E433
:10F250009C430144B9D74A8597500000E780C058C5
:10F2600089B785097DB71733FFFFE702A3E57971F9
:10F270003E847C083EC82E8AB7071400A1653ECAAA
:10F28000E5057C08AA89080836C4428932C6BA8ACC
:10F29000C6843ECC97C0FFFFE78060DFCA850808C0
:10F2A00097E0FFFFE78000C732460808B28597E085
:10F2B000FFFFE78020C8A246630A09049D450808AD
:10F2C00097E0FFFFE780C0BE1D4681459730FFFFF6
:10F2D000E780E0E363890A089145080897E0FFFFAB
:10F2E000E78000BD1146A68597000100E780607A9F
:10F2F000100801478146D2854E8597C0FFFFE78001
:10F3000060FE45611733FFFF670003DFB68508081D
:10F3100097E0FFFFE78000C21C400808D8439355E0
:10F32000C701858912075183B205D98D97E0FFFF88
:10F33000E78040C01C40080883C5870097E0FFFFB6
:10F34000E78040BD1C40080883C5A70097E0FFFF89
:10F35000E78040BC1C40080883C5970097E0FFFF8A
:10F36000E78040BB85BF8945080897E0FFFFE7803D
:10F3700020B483C704002300F50083C71400A30052
:10F38000F500BDB71733FFFFE702C3D383C795006E
:10F390004111AA8993F7F707A384F5003285AE845B
:10F3A000328497E0FFFFE780A0C693170501C1876D
:10F3B000635DF0042A89032A040097C0FFFFE780F9
:10F3C000E0C119E9835744000548F11793B71700C6
:10F3D000A307F100814631A81306F100A28597002A
:10F3E0000000E78060951DC51C459DC783D647007A
:10F3F00001480347F10093078500D2884A86A68515
:10F400004E8597000000E78040E641011733FFFF7B
:10F41000670083CE09487DBF1D486DBF1733FFFFCE
:10F42000E70243CA65715C083EC4B7077B013EC66C
:10F430005C083EC883C795002A8A328593F7F70790
:10F44000A384F500AE8997E0FFFFE78040BA8357B9
:10F45000E100E1C78945280097C0FFFFE78020C38E
:10F460008145280097E0FFFFE780C0AA97C0FFFF13
:10F47000E78000C99777FF1F938787F99C4317742C
:10F48000FF1F034464A2AA843334800099C3136429
:10F4900024009777FF1F938767A99C4399C3136440
:10F4A00044009777FF1F9387A7BE9C4399C31364BB
:10F4B000840083D504002800014997E0FFFFE7801E
:10F4C00060A783D52400280097E0FFFFE78080A68F
:10F4D00083D54400280097E0FFFFE780A0A597D0E0
:10F4E000FFFFE78000AB93150501C181280097E07D
:10F4F000FFFFE78020A4A285280097E0FFFFE780B8
:10F5000060A39C446360F902014781463000CE85C8
:10F51000528597C0FFFFE780E0DC59611733FFFF9A
:10F52000670083BDDC441314490028003E9497E033
:10F53000FFFFE78060968347440003475400890734
:10F540000607BA978607E36AF5FC8355240028006E
:10F55000814A97E0FFFFE780E09D83454400280053
:10F5600097E0FFFFE780009B83455400280097E069
:10F57000FFFFE780209A8347440063C9FA00814A6D
:10F580008347540063C1FA020509A5BF1C441397C1
:10F590005A002800BA9783D50700850A97E0FFFF35
:10F5A000E7804099C9BF032BC40093975A002800F5
:10F5B0003E9B83552B00850A97E0FFFFE7808097ED
:10F5C00083550B00280097E0FFFFE780A0964DBF12
:10F5D0001733FFFFE702A3B05C4993E717005CC94C
:10F5E00097A00000E78020B61733FFFF670063B1E4
:10F5F0001733FFFFE702A3AE2E84814597F0FFFF8C
:10F60000E780C0E705C583570500FD172310F50007
:10F6100009C4835725002310F40097000000E780F9
:10F6200060FB01451733FFFF6700A3AD31457DD86F
:10F6300023100400C5BF1733FFFFE702A3A883C749
:10F64000950041112A8A93F7F707A384F5003285C4
:10F650002E89328497E0FFFFE780809B9317050196
:10F66000C1876356F006AA89C145228597E0FFFF4E
:10F67000E780A0802A8B4E85832A040097C0FFFF75
:10F68000E780C09531E98357440023110100054408
:10F69000F11793B71700A300F1008144034811004C
:10F6A00003572100D6875285CE862286CA8597F0D9
:10F6B000FFFFE780A0A6A1679387170248003EC41A
:10F6C0002302810026C697E0FFFFE780406B4101DF
:10F6D0001733FFFF670043A213061100A28597F0BE
:10F6E000FFFFE7806065AA8409E523110100094452
:10F6F00075B7930521005A8597000000E78080EFD9
:10F70000835721002A84D9DB9777FF1F9387479877
:10F710009C4381CB85451305210097500000E7806D
:10F720000015835521002685314497C0FFFFE780EF
:10F7300080812DD523100500268597900000E78055
:10F74000206D0144A1BF1733FFFFE7024399411128
:10F750002E896C00AA8402C697F0FFFFE78000D2D2
:10F760000DC10357050005072310E50097000000B1
:10F77000E78040E681473E8541011733FFFF670080
:10F7800043983247954765DBCA8526859730000048
:10F79000E780400DC147E34005FE324485474146BE
:10F7A0002310F40083570900A68513054400231194
:10F7B000F40097000100E780C02D228545BF173374
:10F7C000FFFFE702239083C795004111AA8A93F7B0
:10F7D000F707A384F5003285AE89328497E0FFFFF6
:10F7E000E780008393170501C1876356F0062A8AD4
:10F7F000C145228597D0FFFFE7802068AA84528503
:10F80000032B040097B0FFFFE780407D31E9835769
:10F810004400231101008544F11793B71700A3009A
:10F82000F10001440348110003572100DA8756858F
:10F83000D2862686CE8597F0FFFFE780208EA167CF
:10F840009387070248003EC42302910022C697E036
:10F85000FFFFE780C05241011733FFFF6700C389F4
:10F86000A2851306110097F0FFFFE780E04C2A8481
:10F8700009E523110100894475B726859305210008
:10F8800097000000E78060ECAA8449FD83552100C1
:10F89000228597B0FFFFE780006B49F5014997C0CB
:10F8A000FFFFE7800074635DA900184893171900F3
:10F8B000BA9703D707000DEF035721002390E70005
:10F8C00097C0FFFFE780E071630625039767FF1F7E
:10F8D0009387077C9C4399C70355210097500000EC
:10F8E000E78080F0228597900000E78060521DBF7E
:10F8F000050975B795443DB705C19307F00F630F30
:10F90000F500C547630CF5009307F5FF0545331572
:10F91000F5004205418182800145828041657D1567
:10F920008280B9E91723FFFFE702637B03450603E3
:10F93000328497000000E78060FC9305803EB305A9
:10F94000B502C205C18181CD0357E402854763F842
:10F95000E7001305040197E00000E7802042835789
:10F96000E40241677D176385E700FD172317F40262
:10F970001723FFFF6700E37882801723FFFFE7026A
:10F980008373004283C79500444D0349140093F7E5
:10F99000F707A384F5008347040022091167336940
:10F9A000F900A167B347F90041112A8BAE8A63ECD5
:10F9B000E70E834724001307C00EB91793F7F70F1C
:10F9C0006373F71003473400C14763EEE70E8347C4
:10F9D00044001307E00793C707086371F70C8349D6
:10F9E000840083477400A209B3E9F900856763F7CF
:10F9F000F90A034A6400834754004E85220A336A99
:10FA0000FA0097500000E780403B61C12396240331
:10FA1000834B3400137AFA00239A34032388740347
:10FA20002399440393890401631C090023A604025B
:10FA3000239804024E8597E00000E78060363DA0E1
:10FA4000034924004A8597000000E78020EB2397B4
:10FA5000A402834744004E85A388F402E38D0BFC87
:10FA6000E30B09FC97E00000E780202F979000004F
:10FA7000E780007381460146D6855A8597E0FFFFEF
:10FA8000E7800058A167938797033EC423020100D3
:10FA9000480002C697E0FFFFE780602E4101172370
:10FAA000FFFF6700C3648544A2862686D6855A85F3
:10FAB00097E0FFFFE780C054A167938797033EC498
:10FAC00023029100F1B7BD44C5B79144F1BF17239C
:10FAD000FFFFE702235F01111C08404D3EC2B7073C
:10FAE0000F003EC41C083EC62A89AE8997C0FFFF9E
:10FAF000E78000D7585C1C5C6346B70E6394E50052
:10FB000063E2A70E3385A740B3B7A700B305B7409C
:10FB10001306803E81469D8D97000100E78080B7E7
:10FB200093140501C180A1659385C503480097B072
:10FB3000FFFFE780C0558145480097D0FFFFE78071
:10FB4000603D83550404480097D0FFFFE780803E66
:10FB500083552404480097D0FFFFE780A03D8145EE
:10FB600089CCC167FD179305F00F6388F4002685E3
:10FB700097500000E780E0E0AA85480097D0FFFF9B
:10FB8000E780403903554404814501CDC167FD1725
:10FB90009305F00F6307F50097500000E78060DEE3
:10FBA000AA85480097D0FFFFE780C03683456404EC
:10FBB000480097D0FFFFE780E03583457404480094
:10FBC00097D0FFFFE7800035500001478146CE8582
:10FBD0004A8597B0FFFFE780E07005611723FFFFBC
:10FBE00067008351814481B71723FFFFE702234F4A
:10FBF00083C7950093F7F707A384F50097000000EB
:10FC0000E78020ED1723FFFF6700A34F1723FFFFB7
:10FC1000E702434B83C795004111404D93F7F70727
:10FC2000A384F5002A8A3285B284AE8997D0FFFF7B
:10FC3000E780003E2A8B268597D0FFFFE780403D76
:10FC40002A89268597D0FFFFE780603A93170B013A
:10FC500063CA0702E177CA97C207C183116763E3EA
:10FC6000E70293070910C207C1831307B00F637B34
:10FC7000F70093170901C187AA8A634AF000C547B4
:10FC800063FE570141011723FFFF6700E34697B06A
:10FC9000FFFFE7802025E31725FFD5B763080B0298
:10FCA00063060902814463890A02B7077F002310B3
:10FCB0006405231124057CC0568597000000E78069
:10FCC000E0C39304803EB304950239A0B7077F00D8
:10FCD000232004047CC081440355240497E00000E1
:10FCE000E780A0A3A1C497C0FFFFE78060B7269577
:10FCF00093D7F44133379500AE97BA9708DC5CDCB4
:10FD0000CE85528597000000E780A0DC99E0232291
:10FD10000404A1679387B70348003EC4230201008F
:10FD200002C697E0FFFFE7808005A9BF8147014831
:10FD30001CDC232E0403E9B71723FFFFE702233A55
:10FD400097C0FFFFE7802034E1473305F502914576
:10FD500097500000E78000C5E55711C59767FF1F62
:10FD600023A2A71481473E851723FFFF670063394D
:10FD700085471767FF1F2309F71282801723FFFFAC
:10FD8000E702E3359767FF1F9387871180433DC0E4
:10FD9000835704046390A70683572404639CB70425
:10FDA0003689B28497C0FFFFE78080AB5C5C63C399
:10FDB000B7046395B7001C5C63EEA7028347640435
:10FDC00063F3F400A6872303F4048347740463F306
:10FDD0009700A687A303F4048357440441677D1763
:10FDE0006385E70085072312F4043C4481C7CA8574
:10FDF000268582971723FFFF6700A3309767FF1FB1
:10FE00009387070A9C43014599C303C587008280F5
:10FE10001723FFFFE702A32C0111B70707003EC617
:10FE200083C79500584D0AC493F7F7070AC8A384FF
:10FE3000F5002A89AE8411CB1C4283C70700230436
:10FE4000F70097900000E780003421649305540286
:10FE5000280097B0FFFFE780802397000000E7802D
:10FE600020FAAA85280097D0FFFFE780A00A30007B
:10FE700001478146A6854A8597B0FFFFE780804607
:10FE800013044402480822CC230A010002CE97E062
:10FE9000FFFFE780C0EE05611723FFFF67006326C1
:10FEA0001723FFFFE702A32301117C003ECAB70717
:10FEB00007003ECC7C003ECE83C795002E84AA84EA
:10FEC00093F7F707A384F500A165938555024808C9
:10FED00097B0FFFFE780A01B97000000E78040F28B
:10FEE000AA85480897D0FFFFE780C0025008014765
:10FEF0008146A285268597B0FFFFE780A03E056179
:10FF00001723FFFF6700E31F9767FF1F938747F9DA
:10FF10009C43094599C303C5970082809767FF1FDB
:10FF2000938707F89C43094599C303C5D70082808E
:10FF30009767FF1F9387C7F69C43014599C303C585
:10FF4000A70082801723FFFFE702C3170111B7073D
:10FF500008003EC683C79500404D0AC493F7F707D3
:10FF60000AC8A384F5002A89AE8429C414428547AF
:10FF700003C7060063E0E70A834794000946814906
:10FF80006380C702B307F740A304E400B339F0006D
:10FF900083C716002305F40097900000E780A01E99
:10FFA00003572403058B19C76386090097D0000007
:10FFB000E78000E9216493058402280097B0FFFFE1
:10FFC000E780E00C97000000E78040F4AA85280055
:10FFD00097D0FFFFE78000F497000000E78080F5EE
:10FFE000AA85280097D0FFFFE780C0F2014781462D
:10FFF0003000A6854A8597B0FFFFE780A02E130446
:020000040001F9
:100000007402480822CC230A010002CE97E0FFFFC9
:10001000E780E0D605611723FFFF6700E30D172394
:10002000FFFFE702C30B01117C003ECAB7070800BF
:100030003ECC7C003ECE83C795002E84AA8493F7E5
:10004000F707A384F500A16593858502480897B05A
:10005000FFFFE780C00397000000E78020EBAA8540
:10006000480897D0FFFFE780E0EA97000000E780AC
:1000700060ECAA85480897D0FFFFE780A0E9500808
:1000800001478146A285268597B0FFFFE78080253E
:1000900005611723FFFF6700C3069767FF1F93875C
:1000A00027E09C43014599C303C5B700828017230D
:1000B000FFFFE702C3020111B70707003EC683C76F
:1000C0009500404D0AC493F7F7070AC8A384F500CA
:1000D0002A89AE8405C81C42054783C707006368A8
:1000E000F7060347B400630FF700A305F4009790E9
:1000F0000000E78040098347B400B9CF97D0FFFFE5
:10010000E78040BE21649305B400280097B0FFFF4C
:10011000E780E0F797000000E78060F8AA852800F4
:1001200097D0FFFFE78000DF014781463000A685BA
:100130004A8597B0FFFFE780E01A2904480822CCDF
:10014000230A010002CE97E0FFFFE78040C305616C
:100150001723FFFF6700E3FA97D0FFFFE78020BF78
:1001600055B71723FFFFE70283F701117C003ECA52
:10017000B70707003ECC7C003ECE83C795002E8497
:10018000AA8493F7F707A384F500A165AD05480895
:1001900097B0FFFFE780A0EF97000000E78020F016
:1001A000AA85480897D0FFFFE780C0D650080147CE
:1001B0008146A285268597B0FFFFE780A0120561E2
:1001C0001723FFFF6700E3F39767FF1F938747CD70
:1001D0009C43094599C303C5C70082801723FFFFCD
:1001E000E702E3EF01117C00AE843ECAA165B707C8
:1001F00007002A843ECCD1057C0048083ECE97B04B
:10020000FFFFE780C0E897000000E78020FCAA8598
:10021000480897D0FFFFE780E0CF500801478146AC
:10022000A685228597B0FFFFE780C00B05611723E5
:10023000FFFF670003ED1723FFFFE70243EA83C7D1
:10024000950093F7F707A384F50097000000E78077
:1002500020F91723FFFF6700C3EA1723FFFFE70218
:1002600063E683C795000329C501411193F7F7079A
:10027000A384F5001C4283C90700854763E637075E
:100280009767FF1F9387C7189C432E84AA8485CF46
:1002900097000000E78080F389476306F502630456
:1002A00009028347C9006380370323063901979009
:1002B0000000E78040ED83572903898B89C797D0D9
:1002C0000000E780E0B72685A28597000000E78060
:1002D00020F1A167CD0748003EC42302010002C6F9
:1002E00097E0FFFFE780A0A941011723FFFF670008
:1002F000A3E09767FF1F9387A7BA9C431D4599C347
:1003000003C5E70082801723FFFFE70243DD0111E9
:10031000B70707003EC683C79500584D0AC493F738
:10032000F7070AC8A384F5002A89AE8415C71C42C2
:1003300083C7070093968701E18663C40606854656
:100340006381D7068346E7006388F6002307F7003A
:1003500097900000E78020E321649305E4002800E3
:1003600097B0FFFFE780A0D297000000E780A0F8D9
:10037000AA85280097D0FFFFE780C0B901478146D2
:100380003000A6854A8597B0FFFFE780A0F53504C9
:10039000480822CC230A010002CE97E0FFFFE78045
:1003A000009E05611723FFFF6700A3D51723FFFFFA
:1003B000E702E3D201117C003ECAB70707003ECC3A
:1003C0007C003ECE83C795002E84AA8493F7F7075E
:1003D000A384F500A165B905480897B0FFFFE78041
:1003E00000CB97000000E78000F1AA85480897D06D
:1003F000FFFFE78020B2500801478146A28526858D
:1004000097B0FFFFE78000EE05611723FFFF67004D
:1004100043CF1723FFFFE702E3CAAA840144176909
:10042000FF1F130929A8E14997C0FFFFE780A0C576
:100430006344A400014519A8330534038327090048
:100440003E95835725006397970011051723FFFFFB
:10045000670083CA0504C9BF032E8500630A0E1214
:100460001763FF1F1303C3C20323030063150300B5
:1004700029436390061203234E01631503001D43B5
:10048000639907101723FFFFE702E3C2C689428A78
:100490003E89BA8AB684328BAE8B2A84B5E1035585
:1004A0004E0019E501431A851723FFFF670023C497
:1004B000A167A98F116763FBE70097000000E78041
:1004C00080F5814597F0FFFFE780C0120844B70729
:1004D00000E05841F98F18455CC1B707001FF98F3C
:1004E0001CC55C4991C7610597E00000E780408B1F
:1004F000E38A09FA228597900000E78060C65DB71D
:10050000328597C00000E78040430D4349DD1C441D
:10051000116703D54700A167A98F63FBE700970028
:100520000000E78040EF814597F0FFFFE780800CF7
:100530000323840093164B01D1828347B3000356F3
:1005400063008588FD8BA305F300FD777D8E558EB6
:10055000FD76FD16B204F18E83274301C58E23126A
:1005600073012313D3002304530123052301A304A0
:100570004301BDDF228597B0FFFFE78080C9AA85D0
:100580000844B5D1610597D00000E780207F8DB782
:100590001D431A8582801723FFFFE702A3B2056976
:1005A000AA84AE89328A0144FD5A7D1997C0FFFFA3
:1005B000E78020A26347A40001451723FFFF6700DF
:1005C000A3B3D84493171400BA9703D70700631F47
:1005D00037032390570163070A0026859790000090
:1005E000E780A0809C449DC383D76700B3F72701B1
:1005F000639E3701D2880148814701478146014601
:100600008145268597000000E78040E5050479BF15
:100610001723FFFFE70203AB79711C103EC4B70735
:100620000F003EC61C103EC883C79500AA8A3285BB
:1006300093F7F707A384F5002E89328497D0FFFF44
:10064000E780009D93170501C187635AF006AA89C8
:10065000228597D0FFFFE780A09B2A8A4E85032B37
:10066000040097B0FFFFE780609739ED835744009F
:1006700081440544F11793B71700A303F1008345A4
:100680007100DA872287D2864E86280097E0FFFF26
:10069000E780E057014781463000CA85568597B00C
:1006A000FFFFE78020C4A1679387F70348083ECC8B
:1006B000230A810026CE97D0FFFFE780406C45617A
:1006C0001723FFFF670043A3A2851306710097E07D
:1006D000FFFFE7806066AA84094455D1528597E000
:1006E000FFFFE78060D40D4459D90546D2852685A1
:1006F00097000000E78060EA2A8451B71723FFFFC4
:10070000E702E39D835507000346270041112A8431
:100710002E8532C62EC497E0FFFFE780E0D001C9E6
:100720003246A245228597000000E78000E741019C
:100730001723FFFF6700E39C1723FFFFE702A39740
:1007400083C795004111AA8A93F7F707A384F500A0
:100750003285AE89328497D0FFFFE780608B931794
:100760000501C1876357F00AC1452A8A228597C0CF
:10077000FFFFE78080702A8D228597D0FFFFE780FA
:1007800020892A89228597D0FFFFE780408693073A
:1007900005F893F7F70F1307E007AA8B637BF706BB
:1007A000228597D0FFFFE78080842A8C228597D00E
:1007B000FFFFE780C083AA8C5285032B040097B00B
:1007C000FFFFE780A08139E983574400231101002E
:1007D0008144F11793B71700A300F10005440347C4
:1007E000110083562100938784005685DA88228879
:1007F0005286CE8597F0FFFFE78020A7A167E90723
:1008000048003EC42302810026C697D0FFFFE78040
:10081000005741011723FFFF6700638D1306110086
:10082000A28597E0FFFFE7802051AA8409E5231104
:10083000010009446DB7930521006A8597F0FFFF19
:10084000E780A0F02A8441FD835521009356C9001A
:100850001316490185486688E2875E87858A51823A
:10086000268597000000E78060BF2A848DBF17238C
:10087000FFFFE702438483C7950041112A8B93F75A
:10088000F707A384F5003285AE89328497C0FFFF55
:10089000E780007893170501C1876352F00A2A8A1E
:1008A000228597C0FFFFE780A076AA8A228597C09D
:1008B000FFFFE780E0752A89228597C0FFFFE78068
:1008C0000073930705F893F7F70F1307E0072A8CD7
:1008D0006377F706228597C0FFFFE7804071AA8CF7
:1008E000228597C0FFFFE78080702A8D5285832B79
:1008F000040097A0FFFFE780606E39E5835744004E
:1009000085440144F11793B71700A301F100034791
:100910003100930784005A85DE882688D686528661
:10092000CE8597F0FFFFE78040948D4748003EC496
:100930002302910022C697D0FFFFE7804044410187
:100940001713FFFF6700A37AA2851306310097E013
:10095000FFFFE780603E2A84894455D99356C90039
:100960001316490185486A88E6876287858A51821D
:10097000D68597000000E78060AEAA8449BF1713B0
:10098000FFFFE70223742A8981440144617A916A56
:10099000175BFF1F130BCB6F97B0FFFFE7806064FF
:1009A00063C7A40022851713FFFF6700E374832742
:1009B000090093991400CE9703D50700330745012A
:1009C000420741836364570305C103270B0019C71E
:1009D00085453E8597400000E78060E98327090050
:1009E0000504CE972390070085047DB7970000008B
:1009F000E78060A2832709000504CE9723900700B3
:100A000065D5814597F0FFFFE780C0BEF1BF1713A2
:100A1000FFFFE702236B83C7950041112A8A93F7F2
:100A2000F707A384F50032852E89328497C0FFFF33
:100A3000E780005E93170501C187635AF004AA8915
:100A4000832A040097A0FFFFE780405931E58357D0
:100A5000440085440144F11793B71700A301F10046
:100A600003483100D68752850147CE862686CA853F
:100A700097D0FFFFE780806AA167F50748003EC472
:100A80002302910022C697D0FFFFE780402F41014B
:100A90001713FFFF67004366A2851306310097E036
:100AA000FFFFE78060292A8489445DD99757FF1F9B
:100AB0009387075E9C4381CF044997B0FFFFE7808F
:100AC0004052AA85268597400000E78040DA13054A
:100AD000040197000000E780C0EA228597800000AB
:100AE000E78000338144ADBF1713FFFFE702A35C2B
:100AF00083C795004111AA8A93F7F707A384F500ED
:100B00003285AE8932842311010097C0FFFFE78050
:100B1000205093170501C1876354F0062A8AC14506
:100B2000228597C0FFFFE7804035AA8B5285032BB3
:100B3000040097A0FFFFE780604A21E98357440043
:100B400085440144F11793B71700A300F10003484F
:100B5000110003572100DA875685D2862686CE8576
:100B600097D0FFFFE780805BA1679387270248004B
:100B70003EC42302910022C697D0FFFFE7802020C9
:100B800041011713FFFF67008356A285130611006A
:100B900097E0FFFFE780401A2A8489444DD9975790
:100BA000FF1F9387E74E98433E8901CF044997B0D2
:100BB000FFFFE7800043AA85268597400000E78075
:100BC00000CB1305040197000000E78080DB97B09D
:100BD000FFFFE780004195443DD9930521005E85E4
:100BE00097F0FFFFE78060B6AA8435F11C480357F1
:100BF000210022852390E70097800000E7804021B4
:100C000083270900A9D70355210097400000E780FA
:100C1000A0BD35BF1713FFFFE702E34983C7950067
:100C20004111AA8A93F7F707A384F5003285AE89AC
:100C3000328497C0FFFFE780A03D93170501C1876D
:100C40006351F0062A8A228597C0FFFFE780403C67
:100C50002A895285032B040097A0FFFFE780003804
:100C600031E58357440085440144F11793B71700D9
:100C7000A301F10003483100DA8756854A87D286FE
:100C80002686CE8597D0FFFFE7804049A167F90708
:100C900048003EC42302910022C697D0FFFFE780A0
:100CA000000E41011713FFFF67006344A28513067E
:100CB000310097E0FFFFE78020082A8489445DD94E
:100CC0009167CA97C2071167C1831307F7EF85447D
:100CD000E362F7FA9757FF1F9387873B9843BE8BD2
:100CE00001CF044997B0FFFFE780A02FAA85268592
:100CF00097400000E780A0B71305040197000000AB
:100D0000E78020C897B0FFFFE780A02D95443DD134
:100D10001C48228581442390270197800000E780AA
:100D2000200F83A70B00B9D74A8597400000E780C2
:100D3000A0AB89B71713FFFFE702633A2A84410586
:100D4000B28497000000E780C0C311C52285978058
:100D50000000E780E00B81460146A685228597804A
:100D60000000E780C04E1C4C89C7DC4799C3228530
:100D700082971713FFFF6700C3389757FF1F9387AA
:100D800027129C43014599C3138507018280975719
:100D9000FF1F9387E710884382801713FFFFE70246
:100DA00003349317C600DD8DC2054111C1812A8429
:100DB00032C697C0FFFFE780E017324622851182D6
:100DC0009375F60F97C0FFFFE780C014410117131A
:100DD000FFFF670003331713FFFFE702A32E7971AC
:100DE0003C083ED2B7070C003ED43C083ED683C731
:100DF0009500AE842A8993F7F707A384F500A165CF
:100E000093853504481097A0FFFFE7804028C1650F
:100E1000FD150144175AFF1F130A0A29930A400EB1
:100E2000AE892E8B2EC697B0FFFFE780801E42054D
:100E3000931704014181C183B24563E9A702C167E9
:100E4000FD176387F500481097C0FFFFE780800E0D
:100E5000501001478146A6854A8597A0FFFFE7808D
:100E6000604845611713FFFF6700032933075403E8
:100E700083270A0BBA9703D6C701630A3601638A30
:100E80003501481097000000E78060F1DA8505041D
:100E900051BFB285EDBF1713FFFFE702C321797180
:100EA0007C083EC8B70711003ECA7C083ECC83C709
:100EB0009500AA89328593F7F707A384F5002E8958
:100EC00097C0FFFFE780C01485676378F504A165CC
:100ED000AA848905080897A0FFFFE780401B2685A4
:100EE00097400000E78060ED133415000A04A285E6
:100EF000080897C0FFFFE780E001A685080897C0B3
:100F0000FFFFE780200325CC014781461008CA85F2
:100F10004E8597A0FFFFE780E03C45611713FFFF78
:100F20006700E31CB30754030327CA0ABA9703D721
:100F30000700631C970003D6270063806505080837
:100F400097000000E780A0E5DE8505042EC697B077
:100F5000FFFFE780000D4205931704014181C18323
:100F6000B245E3E1A7FCC167FD17E38FF5F8080878
:100F700097C0FFFFE78000FC41BFB285F9B7C165AC
:100F8000FD150144175AFF1F130A0A12930A800223
:100F90002E8BAE8B65BF1713FFFFE702431418417A
:100FA0008347170083460700A207D58FD207D18356
:100FB0002390F50083472700034717008D45A207BC
:100FC000D98F91832310F60097C0FFFFE780A0E937
:100FD0001713FFFF6700E3121713FFFFE702830EEB
:100FE000C16401441759FF1F1309090C93098002BA
:100FF000FD1497B0FFFFE780C0026347A4000145DE
:101000001713FFFF6700430F330534038327C90A13
:101010003E9583570500E38597FE0504D9BF171356
:10102000FFFFE702230A2A8AAE89B284B68A974074
:101030000000E78080D819E591473E851713FFFF30
:101040006700830B2A894E8597C00000E780E08EF9
:101050002A84638E0A048D476DD103570500C54766
:10106000E31D47FD0347F9018546AD47E317D7FC6C
:101070008347450081CF4146A6855D0597F0000076
:10108000E780C09E814755D9AD4745BF130965012B
:101090002302E500CA85268597100000E78060627C
:1010A00031C1A547E38B0AF82302040079B705C1D3
:1010B00083570500E39247F94146A685190597F045
:1010C0000000E780A09A81472DD99947BDB74E858A
:1010D00097000000E78080F02A84954739DD1309E6
:1010E00055004DBF4146A68523104401231134010C
:1010F0001305190097F00000E780A09922859780DA
:101100000000E780A0EA81470DBF1713FFFFE70249
:1011100003FD79717C003ECCB7070A003ECE7C000F
:101120003ED083C79500B2842E8493F7F707A3843B
:10113000F5001306A1002A892C00268597000000DF
:10114000E780A0E5A16528088D0597A0FFFFE7804F
:1011500000F490408355A100035581008546970017
:101160000000E78000ECAA84AA85280897C0FFFF4A
:10117000E78040DA0356A1008355810028089700D4
:101180000000E780C0C1300801478146A2854A853A
:1011900097A0FFFFE7800015854748103ED4230243
:1011A000910202D697D0FFFFE78060BD456117131B
:1011B000FFFF670003F51713FFFFE70243F27971A2
:1011C0007C003ECCB7070A003ECE7C003ED083C7F1
:1011D0009500B2842E8493F7F707A384F5001306D5
:1011E000A1002A892C00268597000000E780E0DA1C
:1011F000A16528088D0597A0FFFFE78040E9904092
:101200008355A10003558100814697000000E780C7
:1012100040E1AA84AA85280897C0FFFFE78080CF15
:101220000356A10083558100280897000000E7803D
:1012300000B7300801478146A2854A8597A0FFFF85
:10124000E780400A48102302910202D402D697D0C8
:10125000FFFFE780C0B245611713FFFF670063EA35
:101260001713FFFFE702A3E797000000E78060DBAA
:101270001713FFFF6700E3E89757FF1F938787C2A5
:10128000884382801713FFFFE70263E58357250039
:101290004111AE842A842307B10017F5FFFF13051F
:1012A00025466C002316F10097A0FFFFE7808045DC
:1012B00091C4228597800000E780E0D6FD57231077
:1012C000F400130620028145130554009710FFFF18
:1012D000E780E0E341011713FFFF670083E2171384
:1012E000FFFFE70223DE79717C003ECCB7070A00DE
:1012F0003ECE7C003ED083C79500AA89AE8493F78A
:10130000F7073285A384F5001306A1002C0097008F
:101310000000E78080C80355810011449740000019
:10132000E780A0A915C50355A100014497B00000AE
:10133000E780A06011CD0357050083578100454425
:101340006318F700854597000000E780E0F301444B
:10135000216993053900280897A0FFFFE78020D373
:10136000A285280897C0FFFFE780C0BA0356A100F6
:1013700083558100280897000000E78040A23008CC
:1013800001478146A6854E8597A0FFFFE78080F53F
:1013900048104AD42302810202D697D0FFFFE7808B
:1013A000009E45611713FFFF670003D51713FFFF6A
:1013B000E70243D19757FF1F938787AE2A8488435C
:1013C0002E8915C5035745038357C4016311F702DE
:1013D0002326050223180502410597D00000E78067
:1013E000209C6306090097800000E78060DB814451
:1013F0009759FF1F938949CB130A800297B0FFFFCB
:10140000E78020C263C4A4049757FF1F938707B2E5
:101410009C4399C70355C40197200000E780C0BDD5
:1014200063070900228597800000E780C0A01306AB
:10143000400E814522859710FFFFE78040CDFD5784
:10144000231EF4001713FFFF670003CB338544030B
:1014500083A7C90A3E95035705008357C401631744
:10146000F700CA8597000000E78000E2850479B79D
:101470001713FFFFE70203C583C795004111AA892F
:1014800093F7F707A384F5003285AE8497C0FFFF7A
:10149000E78000B885676378F5042A8997400000E3
:1014A000E780A091014401CD83D7040031446388D3
:1014B0002701854597000000E78080EF01444E85B5
:1014C000A2864A86A68597D0FFFFE780A09CA167E9
:1014D0009387170448003EC42302810002C697D0B8
:1014E000FFFFE780C08941011713FFFF6700C3C0FA
:1014F0001713FFFFE70203BD9757FF1F9387479A14
:10150000804329C4014597C00000E780002181473E
:101510000148C1641CDC232E040323200404175952
:10152000FF1F130969B801449309400EFD1497B0D9
:10153000FFFFE78000AE634FA400814517F5FFFF72
:101540001305857F97A0FFFFE780C01B1713FFFFE0
:10155000670083BA330534038327090B3E9583570D
:10156000C50163879700854597000000E78040E448
:10157000050475BF9357050113D78700A380F500B5
:1015800093170501C183A1832380E5002381F50022
:10159000A381A50082801713FFFFE70243B4230055
:1015A000050083C71500A300F50083C725002301AC
:1015B000F50083C73500A301F50083C7450023026A
:1015C000F50083C75500A302F50083C765009305A6
:1015D0009500A30305002303F500230405003285CD
:1015E00097000000E78040F91713FFFF670063B121
:1015F0001713FFFFE70203AD4111E9540DCD85CD6F
:1016000093F9C5FF2E842A89AA84338AA900B7EAF0
:10161000040063189A020D88854411CCB7E70400D2
:101620009C5F82972AC622866C003305390197E0B9
:101630000000E7800046268541011713FFFF670081
:10164000A3AB83A78A039104829793170501C183F3
:10165000A183A38EF4FE93570501238FF4FEA1838B
:10166000238EA4FEA38FF4FE6DB763E6D502171395
:10167000FFFFE702C3A6B28741113686BE8536C694
:1016800097E00000E780E040B2464101368517133D
:10169000FFFF670003A781463685828083870500A8
:1016A0001387F5003D05FD8793F77708834607000C
:1016B0007D158606B58FA300F5006307B7007D177B
:1016C000834717009D83DDB782801713FFFFE70272
:1016D00003A1B7E7040083A7070932872A863A8562
:1016E0008297133515001713FFFF670083A115C1FB
:1016F00081478DC11713FFFFE702639E414697E0C4
:101700000000E780003985473E851713FFFF67001B
:10171000439F81473E8582801DCD1713FFFFE7025F
:10172000039C414681452A849710FFFFE780209E55
:1017300041468145130504039710FFFFE780209D74
:101740000147C1672322040438C87CC80545171324
:10175000FFFF6700039B0145828081473DCDB5CDEA
:101760001713FFFFE702A397B2842E8913068005A3
:1017700081452A849710FFFFE7806099CA8524C4B9
:10178000268597000000E780C0F641468145228506
:101790009710FFFFE780A0973044A285228597002D
:1017A0000000E780C0F293040401A285268597001B
:1017B0000000E780E0EEA685130504029700000014
:1017C000E78000EE228597000000E78020F585473E
:1017D0003E851713FFFF6700C3923E858280171373
:1017E000FFFFE702238E4111E9540DCD85CD93F91A
:1017F000C5FF2E842A89AA84338AA900B7EA040087
:10180000639844030D88814411CCB7E704009C5FC2
:1018100082972AC622866C003305390197E00000C2
:10182000E7802027268541011713FFFF6700C38C3F
:1018300083A78A039104829793170501C183A1832B
:10184000A38EF4FE93570501238FF4FEA183238E0C
:10185000A4FEA38FF4FE6DB765CD1713FFFFE7025B
:101860006386B28411E605451713FFFF6700C3883E
:101870002A842E890145EDD93C487848B3E6E70033
:10188000E5D69386F7FFB3B7F6007D17032A440425
:10189000BA9734C87CC863050A06C14913050A0310
:1018A000B38949412295637D3601B2862E86A6858D
:1018B00097000000E780A0DB7C40BE9464C065B761
:1018C000CE862E86CE8597000000E78040DAC114D0
:1018D000D2944E9923220404A2879306040103C7DD
:1018E000070003C607038507318FA38FE7FEE39840
:1018F000F6FE3044A285228597000000E78020DDB7
:101900002699C1493306994063EC9900A9DCA68663
:10191000A6851305040397000000E78040D579BF32
:101920008147B306F4003307F6000347070083C579
:10193000060085072D8F2380E600E39437FF3044AF
:10194000A285228597000000E78060D8C1145DBFA2
:10195000014582800DC11703FFFFE702437813069C
:10196000800581459700FFFFE780607A05451703F2
:10197000FFFF6700037901458280814749C5C1C5E2
:101980001703FFFFE702A375FC4141462E84AA849A
:101990006399C70413860501A2878146C14503C721
:1019A000070003C507038507298F3305D6000345C4
:1019B00005008506298FA38FE7FEE392B6FE30442B
:1019C000A285268597000000E78060D022859700D9
:1019D0000000E78060F885473E851703FFFF67003A
:1019E0004372138507031D8E814522959700FFFFE3
:1019F000E780E0717C40130700F813060402A29709
:101A00002388E70251BF3E8582801703FFFFE7026C
:101A1000036D6D712E84B284AA85901028003689DA
:101A200097000000E780A0D309EDD55725A05040CE
:101A30000C40280097000000E78040E27DD5FD14AF
:101A40002104F5F42C004A8597000000E78020F37C
:101A5000814761DD3E8551611703FFFF6700636ABF
:101A60001703FFFFE702A36741112EC432C62C0003
:101A7000054697000000E78080F941011703FFFF4A
:101A8000670023681703FFFFE702636501112A84DB
:101A90002EC602C802CA02CC02CE97E00000E78040
:101AA000C023B2462A86A285080897000000E78076
:101AB00060FB1375F50F05611703FFFF6700636493
:101AC0001703FFFFE702A3617971B2872A842146D9
:101AD0002308B10013051101BE853AC436C697E04C
:101AE0000000E78000FBB246930591013685970020
:101AF0000000E78060A82285141035460C08970086
:101B00000000E78020F62A84224701E921460C10D4
:101B10003A8597E00000E780C0F72285456117030A
:101B2000FFFF6700035E1703FFFFE702435B71716E
:101B3000AE84AA850A85328497000000E78060BBE6
:101B400011C90A86A685228597000000E78020B883
:101B5000814711E1C5473E854D611703FFFF6700CF
:101B6000435A1703FFFFE70283541D712A8AB28983
:101B7000BE8435468547130511012E8CB68A3A8BF3
:101B8000C28C468D2308F10097E00000E78060F0EA
:101B900010100C085285231F010097000000E780F9
:101BA000C0F82A843DEDA1476313FD089307900513
:101BB00091E0E5473546E2851305110113990A01C5
:101BC0002308F1001359090197E00000E78060EC59
:101BD0001357890093978A00D98F90080C08528573
:101BE000231FF10097000000E78020F42A8415E904
:101BF000A1E49387FA0091831379F9003EC6631339
:101C000009004149668B8144C14B854DB247639FB2
:101C1000970C6A868C0033855C0197E00000E780B2
:101C200040E7228525611703FFFF6700034C9307F8
:101C30009004C9F0A547BDBF834701050947C14BC3
:101C40002308F10083471105A58FA308F1009387AE
:101C50002400814463E1FB04014714083386E60055
:101C60008C08B386E400BA95DA9683C6060083C56D
:101C700005000507AD8E2300D600E390E7FE41473F
:101C8000639CE70490080C08528597000000E780E9
:101C9000C0E925D181A0B3069B00BA871008B3051F
:101CA000F60090083E9603C5060003460600850729
:101CB0008506298E2380C500E39277FF998F9008CF
:101CC0000C085285BE9497000000E78000E6894723
:101CD000014749D12A84B1B790083E9603460600D1
:101CE0001408BE962380C600850759BFB2478504F5
:101CF0006387971481471808B306F70098083E9742
:101D00003386F90003470700034606008507318F35
:101D10002380E600E39177FF90080C085285970036
:101D20000000E78080E05DF53546E285130511018E
:101D30002308B10197E00000E780A0D513970401C4
:101D40004183939784002183D98F10180C08528502
:101D5000231FF10097000000E78020DD25FD81476B
:101D600010183387F9003E96034707000346060024
:101D7000B306FB008507318F2380E600E39277FFEF
:101D800065A81808B306F70098083E973386F9004F
:101D900003470700034606008507318F2380E600CE
:101DA000E3E127FFCA87639E770990080C085285F4
:101DB00097000000E78060D711FD81479800B306C7
:101DC000F700900818103E973E9603470700034619
:101DD00006008507318F2380E600E39177FF3546C3
:101DE000E285130511012308B10197E00000E780A7
:101DF00040CA139704014183939784002183D98FAC
:101E000010180C085285231FF10097000000E7808E
:101E1000C0D1E31105EC814710183387F9003E96D5
:101E20000347070003460600B306FB008507318F12
:101E30002380E600E3E227FFC109410BC1BB8147D4
:101E400085B79408BE9683C6060018083E972300FF
:101E5000D700850789BF638006321703FFFFE702BB
:101E6000032559712A84BE89B28B854735461305EF
:101E700011022E8B468C4289BA8A368A2300F102DF
:101E800097E00000E780E0C010180C1022852317AF
:101E9000010297000000E78040C963180512A147BE
:101EA000631FFC069307900563930900E5473546D9
:101EB000DA851305110293140A012300F102C1808F
:101EC00097E00000E780E0BC93178A0013D78400F6
:101ED000D98F90080C1022852317F102970000007B
:101EE000E780A0C47DE1639209049307FA00BD88EE
:101EF000918391E0C144C207C183DE8C814A3EC612
:101F0000414DB24763E2FA0E6286B3854B018810F9
:101F100097E00000E78080B54DC93D557DA093074F
:101F20009004E39609F8A54759B783470105094787
:101F3000C14C2300F10283471105B3C7F900A30088
:101F4000F10293872900814963E1FC04814618105E
:101F50003306D7008C083387D900B69556970347C8
:101F6000070083C5050085062D8F2300E600E3905A
:101F7000D7FE41476390E70690080C102285970032
:101F80000000E78080BA35D189A0B3863A01BA87CC
:101F90001010B305F60090083E9603C506000346F0
:101FA000060085078506298E2380C500E39297FFEA
:101FB0003387EC4090080C102285BA9997000000F6
:101FC000E780A0B68947014741D165611703FFFF4C
:101FD0006700A31190083E96034606001410BE96B3
:101FE0002380C600850779B7B247850A93990A010D
:101FF000939D8A0093D909016391570F8547354610
:10200000DA85130511022300F10293D9890097E0C4
:102010000000E78000A8B3ED3D0190000C10228580
:102020002317B10397000000E78020B059FD8147D6
:10203000A68963EA970626860C084A8597E0000081
:10204000E78020A581471810B306F700100898080C
:102050003E973E9603470700034606008507318FEB
:102060002380E600E3E197FE639FA90590080C102A
:10207000228597000000E78040AB21F98147981046
:10208000B306F700900818183E973E9603470700DE
:10209000034606008507318F2380E600E391A7FF02
:1020A0004109C10CB9BD18089000B306F7003E966F
:1020B0003387FC0003470700034606008507318F7E
:1020C0002380E600B5B798084E97034707001C1019
:1020D000CE972380E700850941BF85473546DA85DD
:1020E000130511022300F10293D9890097E0000043
:1020F000E780209AB3ED3D0190000C102285231754
:10210000B10397000000E78040A2E31005EC81478F
:1021100018089000B306F7003E963387FC0003478B
:102120000700034606008507318F2380E600E39110
:10213000A7FF41460C084A8597E00000E7806095BC
:1021400081471810B306F700100898083E973E968E
:1021500003470700034606008507318F2380E6000A
:10216000E391A7FF90080C10228597000000E780FC
:10217000C09B1DD599BD7D5582801703FFFFE702E7
:1021800003F601112A842E8593055100328902C07D
:1021900002C202C402C69304740097F0FFFFE780F6
:1021A000A03D1D46A6851305910097E00000E7803D
:1021B000408E10088A854A8597000000E780E096E7
:1021C00019ED93071400180883C60700034607009B
:1021D00085070507B18EA38FD7FEE397F4FE05614F
:1021E0001703FFFF6700E3F11703FFFFE70283ED2B
:1021F0002E848C414111AA8983871500328991442C
:1022000063D30700A1449747FF1F938767209C4330
:10221000A1C7C1CA8D472310F10083C725004A8595
:102220002301F10083C73500A301F10083C74500F6
:102230002302F10083C75500A302F10083C76500A4
:1022400093059100A30301002303F100230401007F
:1022500097F0FFFFE78040320C404A860A8597F0EE
:10226000FFFFE78080330328040083564400A688DC
:102270001D0881470147E51642868A854E859700ED
:102280000000E780408E2A8919E5A685228597B04F
:10229000FFFFE780E0C14A8541011703FFFF6700A8
:1022A000A3E54A860A8597F0FFFFE780002F6DB708
:1022B0001703FFFFE70203E12E848C414111AA8935
:1022C000838715003289914463D30700A14497475F
:1022D000FF1F9387E7139C43A1C7C1C68D472310F7
:1022E000F10083C725004A852301F10083C735002B
:1022F000A301F10083C745002302F10083C7550005
:10230000A302F10083C7650093059100A3030100B8
:102310002303F1002304010097F0FFFFE780C025AD
:102320000C404A860A8597F0FFFFE7800027835616
:102330004400032804008A85858EC2061D08C182D8
:102340002312D400A68881470147E51642864E85B0
:1023500097000000E78060B041011703FFFF6700AE
:10236000A3D94A860A8597F0FFFFE78000234DBF77
:102370001703FFFFE702A3D6B335B00001118505AF
:102380002A891315F601336515012308B100930559
:10239000110136843AC632C03EC442C297F0FFFFF4
:1023A000E780801DA2471248425593D68700230B31
:1023B000F1009305910193578800A30AD100A30B64
:1023C000F100230C010197F0FFFFE780E01A32478C
:1023D000024603280400B337E00083564400920706
:1023E000914411C2A1444A85A68842860C0897F000
:1023F000FFFFE78040772A8919E5A685228597B0F7
:10240000FFFFE780E0AA4A8505611703FFFF670029
:1024100043CF1703FFFFE702E3CA01113EC6864719
:10242000B335B0008505AA891315F6015D8D230823
:10243000B1009305110136843A89B28442C446C280
:1024400097F0FFFFE78040132248924816459357C4
:102450008800A30AF1009305910193D78800230B0C
:102460000101A30BF100230C110197F0FFFFE7809E
:10247000A0103247104083564400B337E000920763
:1024800003280900914891C0A1480C084E85970087
:102490000000E780809CAA8401E9835544004A85B6
:1024A00097B0FFFFE780C0A0268505611703FFFFF7
:1024B000670083C4AA959307F00F1717010013074D
:1024C000A7866317B50013C5F7FF1375F50F828054
:1024D00005058346F5FFB58FBA9783C70700D5B7C3
:1024E0000357450014419307F00F17160100130618
:1024F000A683369742074183139506014181631BEA
:10250000E500AD8FB29703C50700130515F313352A
:1025100015008280850603C5F6FFA98FB29783C791
:102520000700D9BF1703FFFFE70263BBB2873684FA
:102530002E86BA86AA853E85BA8497F0FFFFE7808B
:102540006052634F0500228597D00000E780E07855
:102550002A86A686A285268597F0FFFFE780805011
:102560001703FFFF6700E3B91703FFFFE70283B517
:102570005D712A8BAE8A17050100130565782C0062
:10258000B284368ABA893E8997F0FFFFE780C04F50
:102590002A845DE134104146DA85280097F0FFFF78
:1025A000E780404C2A8449E98547A303F100A6C28D
:1025B000930771002408BEC4A68685470D462C18D3
:1025C000281002DC02DED6C0BEC697F0FFFFE7800F
:1025D00000442A8435E183477102A6860D4693F7AD
:1025E000F7072300FA00C1473EDE2C188947281060
:1025F00026DCA303F10097F0FFFFE78040412A8427
:1026000005ED4146A6854E8597D00000E7806048DD
:102610008D47A6860D462C182810A303F10097F0CD
:10262000FFFFE780C03E2A8401E94146A6854A852E
:1026300097D00000E780E045228561611703FFFF26
:10264000670083AB1703FFFFE70263A997F700005A
:10265000938787A1984383C7470079712A89AE84FD
:10266000170501001305456A0C083AC42306F1005A
:1026700097F0FFFFE78040412A8405ED14104146A2
:10268000CA85080897F0FFFFE780C03D2A8415E15E
:10269000140815462C00081097F0FFFFE780803CD7
:1026A0002A8401E921462C08268597D00000E7807E
:1026B000403E228545611703FFFF670083A417038F
:1026C000FFFFE702C3A197F700009387E7999C47B4
:1026D0007971AA842E8417050100130565630C081F
:1026E0003EC697F0FFFFE780203A0DE914104146FF
:1026F000A685080897F0FFFFE780C03605E11408BB
:1027000011466C00081097F0FFFFE780A03519E52F
:102710008347F10193F7F7032300F40045611703A2
:10272000FFFF6700039E1703FFFFE702439B368806
:10273000A14881470147E54697F0FFFFE780A042A7
:102740001703FFFF6700E39B1703FFFFE7022399CF
:102750003688A14881470147E54697F0FFFFE780AB
:10276000C06F1703FFFF6700C3991703FFFFE7025E
:10277000039701112A842E850C0832C697F0FFFFBB
:10278000E780803009ED3247970601009386C656F0
:102790001008C145228597000000E780E0D8056158
:1027A0001703FFFF6700E3951703FFFFE70223937B
:1027B0004111C1472EC032C48A8509463EC23EC679
:1027C00097F0FFFFE780A02441011703FFFF670098
:1027D00043931703FFFFE70283904111AE86130670
:1027E0001009AA850A8502C002C202C402C697F077
:1027F000FFFFE780202741011703FFFF6700639079
:102800001703FFFFE702A38D328797060100938627
:10281000A6502E869305000297000000E780C0D0E6
:102820001703FFFF6700E38D1703FFFFE702238B0A
:102830007971C1472ACC2ED032D42C080D462800FD
:102840003ECE3ED23ED602C402C602C802CA97F0AD
:10285000FFFFE780C01B45611703FFFF6700638A26
:102860001703FFFFE702A3870111AA842E8417052F
:1028700001001305E54A8A8597F0FFFFE780C02035
:1028800015E514084146A6850A8597F0FFFFE78005
:10289000601D09ED8347E1010347F101A207D98FCC
:1028A000CA07C9836177D98F2310F4000561170324
:1028B000FFFF6700038515CD1703FFFFE7022382A3
:1028C0009737FF1F9387876290439735FF1F938544
:1028D00025621735FF1F1305655D97D00000E7805F
:1028E00000C51735FF1F1305655C1703FFFF670061
:1028F00043811735FF1F1305655B82808DCD17F36C
:10290000FEFFE702C37D9737FF1F9387275E94433F
:1029100001112E840A869735FF1F9385655D97D038
:102920000000E78040C60A8502940145056117F35F
:10293000FEFF6700037D7D55828017F3FEFFE702EF
:10294000037A97D00000E78080D19737FF1F23AF2D
:10295000A75817F5FFFF1305E5C997B00000E780FA
:10296000C07417F3FEFF6700C3791737FF1F130703
:10297000275A9317150008433E95FD572310F5007D
:10298000828017F3FEFFE70283752A84084009E579
:1029900017F3FEFF6700E3761C4158401CC0631329
:1029A000E5005CC08347550023200500F99BA30286
:1029B000F50097A0FFFFE780207CC9BF17F3FEFF5B
:1029C000E70243709737FF1F9387875698432A84FF
:1029D00011CB8347350093F7070289C703550500DC
:1029E000894502971305440197B00000E780403BFA
:1029F000835504000355E40097300000E780A00CE5
:102A0000485819C597A0FFFFE7800077232A0402E2
:102A10001305840397000000E780E0F68144B14984
:102A20009790FFFFE780206A63CBA40283473400BE
:102A30002320040493F727FCA301F4000048979097
:102A4000FFFFE7804069131615008145228597F046
:102A5000FEFFE780C06B17F3FEFF6700E369B387F3
:102A600034030329040385043E994A859700000036
:102A7000E78060F12304090065B78347350093F7C9
:102A8000070299E3014582808357E500E39CB7FE86
:102A9000C167FD176316F60005458280054599A8B4
:102AA00017F3FEFFE702A36393170601C187B28401
:102AB0002A8401496359F002835705009DCB0145E3
:102AC0006367F600034584003E953325A600137521
:102AD000F50F0DA01C4813171900BA9783D70700EC
:102AE000E38E97FA05099790FFFFE780C05EE34306
:102AF000A9FE014517F3FEFF6700A36017F3FEFF71
:102B0000E702435CAE89AA849790FFFFE78060529A
:102B10002A8497D0FFFFE780A02EAA8601471306DC
:102B2000840197050000938585E41735FF1F130581
:102B3000653E9790FFFFE780E0182A8925C98C44FD
:102B40001304C50022859E0593F5050897A0FFFF95
:102B5000E780403CCC4083877400E18163DD07045B
:102B600093E50508228597A0FFFFE780A03A0D4670
:102B700093854400228597A0FFFFE780C03683D568
:102B80000400228597A0FFFFE780E03D83D5240065
:102B9000228597A0FFFFE780003D03D6490083A56B
:102BA0000900228597A0FFFFE780E0334A8517F3ED
:102BB000FEFF6700635493F5F5076DB717F3FEFF4B
:102BC000E702E35101112A84328532C697A0FFFF44
:102BD000E780E0279780FFFFE780C030835704003D
:102BE0001737FF1F1307474C3246231BF10093078B
:102BF00000F8A30DF1001C471843231AA100898394
